:1000000000100020F576030835D4020849D4020810
:100010005DD4020871D4020885D4020800000000F3
:1000200000000000000000000000000099D4020859
:10003000ADD4020800000000915500087F3F010880
:10004000797803087D78030881780308CB3F01089D
:1000500089780308E7DD020805D70208EDD8020811
:10006000B3D90208A5DA0208A1780308A578030825
:10007000A9780308AD780308B1780308B5780308B8
:10008000B9780308BD780308C1780308C578030868
:10009000C9780308CD780308D17803080FDC02087B
:1000A000D9780308DD780308E1780308E5780308C8
:1000B000E9780308ED780308F1780308F578030878
:1000C000F9780308FD78030801790308C5D402080C
:1000D000097903080D7903081179030815790308D4
:1000E00089DB0208EFDC020821790308257903087F
:1000F000297903082D790308317903083579030834
:10010000397903083D7903084179030845790308E3
:10011000497903084D790308517903085579030893
:10012000597903085D790308617903086579030843
:10013000697903086D7903087179030875790308F3
:10014000797903087D7903088179030885790308A3
:10015000897903088D790308917903089579030853
:10016000997903089D790308A1790308A579030803
:10017000A9790308AD790308B1790308B5790308B3
:10018000B9790308BD790308DFF85C0B0078704784
:100190002DE9F04798B002F04DFC0446DFF84C0B17
:1001A000856BDFF84C6B376826E098F81910D8F8A3
:1001B0001000D8F804208018D7F820215269904701
:1001C000002802D0384602F073FD00213846D9F8E5
:1001D000042092699047022802D1012088F8160075
:1001E00001213846D9F8042092699047022802D1AB
:1001F000384602F053FE3F68B74243D097F90800F3
:100200001A28F8D01B28F6D00728F4D00B2807DBD3
:100210000E2805D00F2803D0102801D01828EAD1C5
:100220000628E8D007F10808D8F84800002805D5C6
:1002300004F1780109690818C8F8480007F59079B1
:100240004FF0FF313846D9F8042092699047824632
:10025000BAF1010F05D198F84C00D7F820110969BF
:100260008847BAF1020FB0D197F9080001289CD154
:10027000687A002899D0A87F012896D1384602F0E4
:1002800017FDA2E7D4E91E01002901D100280DD0F5
:100290000A208DF8020002208DF8000004F1780099
:1002A0000069ADF8580000A803F0B2FA012018B0B8
:1002B000BDE8F08730B585B004460D46CA208DF8FC
:1002C00000002888ADF801000220ADF80300BDF859
:1002D0000100001D03F0F2FBCDF8090002220DF130
:1002E000030103F013FC02222946DDF80900801CFB
:1002F00003F00CFC2A882146DDF80900001D03F0FC
:1003000005FC0020288000A9DFF8E80903F01CFCA8
:1003100005B030BD42F23411081A322801DA01204A
:1003200070470020704780B503F04FFC407B0028E9
:1003300004D002F08BFBDFF8C019086001BD80B566
:1003400002F084FBDFF8B419086001BD80B502F04B
:1003500086FBDFF8AC29C2E9000101BDDFF89C098A
:1003600000687047DFF89829D2E90001704770B53E
:1003700082B004460020009004F10C05FFF7EEFF68
:10038000E96F401A0090E96AC968DFF878295118C6
:1003900008180090687DAB7DEE68E4686968891B89
:1003A000994205D1042200A9001903F0AFFB73BDE7
:1003B000042200A934191B19C01803F0A7FB73BD50
:1003C00070B582B0044600200090054604F1900606
:1003D000307A012834D104F10800016C01290CDBCA
:1003E0008168827E91FBF2F1012908D0006BC06820
:1003F0004FF47A714843009001E00120009094F995
:1004000008000C2801D011280ED1FFF7A7FFD4E96E
:100410002423801A0090DFF8EC1808180090014699
:100420000FF2681003F03AFC2846C4F81401782251
:10043000014604F19C0004F043F92846307288E03C
:1004400094F908000C2801D0112821D1FFF786FF6C
:10045000D4E92423801A0090FFF780FF2946D4E9CD
:100460002423994209D801D3904206D264200090F7
:1004700001460FF2301003F011FC0098DFF88418E9
:100480000818009001460FF2301003F007FC26E038
:10049000FFF768FFD4E9242300F096F8009004F1F8
:1004A0000800006BC0680099002914D09DED000A77
:1004B000B8EE400A00EE900AF8EEE00A9FED5B1AF3
:1004C00060EE810AB7EE081A60EE810AF4EE400A87
:1004D000F1EE10FA03D54FF47A714843009094F985
:1004E00008000C282CD011282AD0D4F81401411C63
:1004F000C4F8141104EB80000099C0F89C10284641
:1005000005E004EB8001D1F89C104D19401CD4F893
:1005100014118842F5DBB5FBF1F00090D4F814011A
:100520001E280DDB1D20C4F81401002006E004EB9A
:100530008001D1F8A020C1F89C20401C1D28F6DBCA
:1005400004F58A700179012903D10021017150203D
:10055000009004F10800042200A9437E0569406868
:100560002818181803F0D2FA94F908000C2801D0C2
:10057000112805D1FFF7F2FE0021C4E9240173BD63
:10058000FFF7F0FEC4E9240173BD000046697273F1
:10059000742054696D652064696666203D20256479
:1005A0000000000054696D655F646966665F6F7680
:1005B0006572203D2025640054696D655F6469663D
:1005C00066203D202564000038B52DED028B0446E1
:1005D0000D4610461946A94205D801D3A04202D2C1
:1005E0009FED138A01E09FED138A04F073F800EE8B
:1005F000100A30EE088A2046294604F06BF800EE17
:10060000100A38EE400ABCEEC00ADFF8FC16B8EE5D
:10061000C00AD1ED010A20EE200ABCEEC00A10EE9D
:10062000100A0860BDEC028B32BD000000007A4465
:10063000000080460000000030B41488651C15805E
:10064000052565541488651C1580635413885C1C4B
:100650001480007A585430BC704732B515461C4699
:1006600021884A1C228037224A5521884A1C228030
:10067000007A4855022200A92088401903F046FA62
:100680002088801C208031BD2DE9F04105461646AA
:100690001F4605F10808069CA4B298F81A0004FB4E
:1006A00000F2D8F8040009183888801903F02EFAEF
:1006B000388898F81A10614311FA80F03880388829
:1006C000FFF728FE002803D039463046FFF7F2FD39
:1006D00095F9080016280AD1D8F81000D8F80410A7
:1006E000415C0FF21000BDE8F04103F0D7BABDE85D
:1006F000F08100002323205368616B65202564008E
:1007000030B400F110039B7C914203D1006990FB4F
:10071000F3F00DE00C46154603D2281B90FBF3F0D6
:1007200006E00069001B90FBF3F095FBF3F108185D
:1007300080B230BC704700F110018A688B7CD218FF
:100740008A600069824201D100208860002088739D
:10075000704770B582B004460D461E4692B289B20B
:10076000FFF7CEFF0090069B324629462046FFF752
:100770008BFF73BDF8B5044615461E462269002D51
:1007800000D11546069F0097FFF7E3FF20698542D9
:1007900006DA009733462A4600212046FFF7D9FFA4
:1007A000F1BD2DE9F04184B004460F469046A169A1
:1007B0006069002816D500250A4692B289B2204603
:1007C000FFF79EFF064643463A4631462046FFF76E
:1007D00044FFA269CDF800803B4611462046FFF752
:1007E000C9FF39E0814217DA01250A4692B2014673
:1007F00089B22046FFF784FF064643463A46314613
:100800002046FFF72AFFCDF800803B46A2696169C8
:100810002046FFF7AFFF1FE00225884206D00A46B8
:1008200092B2014689B22046FFF76AFFA26992B2EE
:10083000616989B22046FFF763FF064643463A46A0
:1008400031462046FFF709FFCDF800803B46A269FC
:1008500061692046FFF77DFFA06B80680290A06968
:100860000190606900902B46324694F908100FF20F
:100870000C0003F013FABDE8FF8100005061636BC8
:10088000203D2564202564202564202564202564DE
:100890002025640070B582B004460D461646A06C53
:1008A000012811DAA07F012811D133462A460121FF
:1008B0002046FFF7D2FE0120009033462A46A16968
:1008C0002046FFF7E1FE02E02046FFF76AFF012322
:1008D000324629462046FFF7AFFE00206061A06146
:1008E000A36CE26C94F908100FF20C0003F0D6F937
:1008F000A06CE06473BD0000666C757368202564AD
:1009000020256420256400002DE9F84304460D46A7
:10091000164602F08FF8814603F057F9804604F13D
:100920000807B87D00280ED02046FFF749FD94F94E
:1009300008000C2807D1012084F81901D4F81C0103
:10094000401CC4F81C01386C0128C0F2DC8098F807
:100950000E00002848D0B87D002800F01C81786C7B
:10096000D9F88810401A7864B87E3969FA68531A41
:10097000834205D0002A33D1BA68511A81422FD15F
:1009800094F90820397E0FF2142003F087F9397E9C
:1009900000291ED094F908200FF2182003F07EF9E8
:1009A0003869B97E421892B2F96889B22046FFF7D9
:1009B000A7FE33462A4601462046FFF74EFE009624
:1009C0002B463869B97E4218F9682046FFF7D2FEF7
:1009D00006E04FF0FF30F860FFF7C0FCC4F8880075
:1009E0002046BDE8F243A6E698F80E00002840F045
:1009F000D280786CD9F88810401A7864F96811F1BF
:100A0000010F10D1B87D002802D02046FFF793FED9
:100A10002046FFF7ACFC324629462046FFF7C1FED0
:100A20003869F860B7E001284CDA386C7864386BC4
:100A3000D0F80C8094F908308268396C0FF290106D
:100A400003F02CF994F908000C281FD0B868B97E7F
:100A500090FBF1F0396C91FBF8F1814202DB4FF031
:100A6000FF30F860B87D0028204607D0FFF763FE0E
:100A7000324629462046FFF794FE20E0FFF7A0FC0F
:100A8000324629462046FFF78CFE18E094F81901FB
:100A9000012814D1D4F81C01B968BA7E91FBF2F197
:100AA000884202D14FF0FF30F86032462946204696
:100AB000FFF777FE0020C4F81C0184F8190138699B
:100AC000F86068E094F908000C2815D1D4F81C01EE
:100AD000B968BA7E91FBF2F188420DD14FF0FF3038
:100AE000F860324629462046FFF75BFE0020C4F836
:100AF0001C0184F819014EE0B87D00284BD0204637
:100B0000BDE8F24317E6B87D002844D094F9080008
:100B100098F80A1000291FD0072807D00D2805D003
:100B2000162803D01A2801D01B282FD133462A4675
:100B300001212046FFF791FD0120009033462A460F
:100B400039692046FFF7A0FD7A7894F908100FF272
:100B5000940003F0A3F819E0092809D194F8721061
:100B6000012905D10FF28C00BDE8F44303F096B8DB
:100B700033462A4601212046FFF76FFD01200090F1
:100B800033462A4639692046FFF77EFD2046FFF7A7
:100B9000D2FD3869F860BDE8F183000073757370A9
:100BA000656E64206669666F2066756C6C202564CE
:100BB0002025640073757370656E64206669666FC6
:100BC0002066756C6C2032202564202564000000AE
:100BD0006669666F2066756C6C3320256420256419
:100BE000202564004150205375732025642025641E
:100BF00000000000233E6C75785F736174202564EB
:100C000000000000F8B504460D463848466896F8DE
:100C1000730001281DD1002086F873002888411C2C
:100C20002980082101550020ADF8000007460EE09C
:100C300006EB8700006EADF80000022200A92888AC
:100C4000001902F063FF2888801C28807F1C032F76
:100C5000EEDBF1BDF8B504460D46FFF7D3FF244E99
:100C6000376805E02A4621463846FFF74DFE3F68C3
:100C7000B742F7D1F1BD2DE9F04104460D461B4EB8
:100C8000F76907F10C0898F81510D8F80C00FA6805
:100C90008018D7F820215269904700280AD00120F7
:100CA00088F81200787A002804D02A46214638466F
:100CB000FFF72AFEB66906F10C07797DF868F2683D
:100CC0008018D6F8202152699047002809D00120C9
:100CD000B874707A002804D02A4621463046FFF7BF
:100CE00013FE0120BDE8F081F5560120AC4901203A
:100CF0002C400020A0AC0020885601208C560120FA
:100D00000856012000CA9A3B54AA00200288D21C2F
:100D100002800A80704780B50B889B1AADF80030BE
:100D2000BDF80030002B09D01018012100F8031C79
:100D3000022200A9801E02F0E9FE01BD0888C01E43
:100D4000088001BD2DE9F04FADF68C2D04460D460F
:100D500001F070FE064602F038FF804610A840F60B
:100D6000482103F0EBFC00208DF8020006A82821A2
:100D700003F0E4FC01A8142103F0E0FC0020ADF82E
:100D800000000746D6E91E01002902D1002800F024
:100D90002C8598F9090004F06EF9002800F02585EB
:100DA00000A92846FFF7B2FFB8461CE0D6E91E01AD
:100DB000424604F0C7FB00F0010011F0000101D130
:100DC00000280ED0C8EB0810DFF8441E01EB8002AB
:100DD00092F90300012804D10DF1020110A8526B11
:100DE000904708F10108B8F13C0FDFDBBA461BE081
:100DF00029884A1C2A80807808552888FFF78AFAB3
:100E000000280DD0BDF8002029462046FFF783FFBB
:100E100029462046FFF74EFA00A92846FFF776FF3D
:100E20000AF1010A4FFA8AFA9DF80200824580F21F
:100E3000D4842988481C288040F2491010FB0AF00D
:100E400010AA825C0A5529884A1C2A8010AA861892
:100E5000707808552988481C2880701C42780A55EB
:100E60004178032927D0092900F09A810C2900F044
:100E700075811A2900F091821B2900F0A4811C2998
:100E800000F0BB821D2900F0AE811E2900F0A68271
:100E9000262900F0DE822C2900F00A832F2900F099
:100EA000E782302900F06183312900F08C833429F6
:100EB00000F0EA839CE77178032904D129884A1C51
:100EC0002A8082780A5529884A1C2A80C2780A55C5
:100ED000C178C0290FD106F22708B8F82E20D8F81B
:100EE00030102888001902F011FE2888B8F82E105A
:100EF0000818288081E70846E0284AD106F205064E
:100F0000002035E056F820100A0222F0FF12090AEC
:100F100001F0FF11114346F820104FEA314146F825
:100F2000201006EB80014A68130223F0FF13120A17
:100F300002F0FF121A434A604FEA32424A608A685E
:100F4000130223F0FF13120A02F0FF121A438A6001
:100F50004FEA32428A60CA68130223F0FF13120A72
:100F600002F0FF121A43CA604FEA3242CA60001D03
:100F70001428C7DB50210FF67C0002F08FFE5022B0
:100F800031462888001902F0C1FD28885030288099
:100F900033E7791C000647D401A8321D52783A5431
:100FA000C9B2B2790A54491CC9B200220A544A1C77
:100FB00006F20601D2B24B781354521CF389D2B216
:100FC0001F0A1754521CD2B21354521C06F20E03BD
:100FD000D2B29F781754521CD2B2DB781354521CF1
:100FE000D2B2B37C1354521CD2B2F37C1354521CB1
:100FF000D2B28B781354521CD2B2C9781154511CFE
:10100000C9B2B27A0A54491CC9B2F27A0A544F1CC6
:10101000FFB23A4601A92888001902F077FD288816
:1010200050FA87F02880E8E6D6F8052006A8130CC9
:101030003B54C9B2130A0B54491CC9B20A54491C87
:10104000D6F80920C9B2130C0B54491CC9B2130AB3
:101050000B54491CC9B20A54491CD6F80D20C9B218
:10106000130C0B54491CC9B2130A0B54491CC9B2C6
:101070000A54491CD6F81120C9B2130C0B54491C50
:10108000C9B2130A0B54491CC9B20A54491CD6F8F8
:101090002720C9B2130C0B54491CC9B2130A0B54B4
:1010A000491CC9B20A54491C06F22708C9B298F86B
:1010B00004200A54491CC9B298F805200A54491C56
:1010C000B8F80620C9B2130A0B54491CC9B20A5415
:1010D000491CC9B298F808200A54491CD6F81520B2
:1010E000C9B2130C0B54491CC9B2130A0B54491C46
:1010F000C9B20A54491CD6F81920C9B2130C0B54B2
:10110000491CC9B2130A0B54491CC9B20A54491CE0
:10111000D6F81D20C9B2130C0B54491CC9B2130ACE
:101120000B54491CC9B20A54491CD6F82120C9B233
:10113000130C0B54491CC9B2130A0B54491CC9B2F5
:101140000A544F1CFFB23A4606A92888001902F03B
:10115000DDFC288850FA87F028804EE6F11CB1F9B2
:101160000300C0F3072242EA0020A1F80300B1F90E
:101170000700C0F3072242EA0020A1F80700B1F9F6
:101180000500C0F3072242EA0020A1F80500092269
:101190002888001902F0BAFC2888093028802CE63B
:1011A00029880B467278032A08D10222F11C1819EB
:1011B00002F0ACFC2888801C28801EE6491C29808F
:1011C0008078185519E629884A1C2A8080780855A5
:1011D000707805287FF411AE2888411C2980311DC4
:1011E0004978015509E606F103087078012840F0B6
:1011F000C4802888411C298098F8041001554FF0BC
:101200000009A1E0C9EB491000EB080BDBF818005E
:10121000010221F0FF11000A00F0FF100843CBF893
:1012200018004FEA3040CBF8180004220BF11801E7
:101230002888001902F06AFC2888001D2880DBF845
:101240000800010221F0FF11001200F0FF10084316
:10125000CBF80800C0F30F4141EA0040CBF808008A
:1012600004220BF108012888001902F04FFC28889D
:10127000001D2880DBF80C00010221F0FF11001294
:1012800000F0FF100843CBF80C00C0F30F4141EA17
:101290000040CBF80C0004220BF10C012888001947
:1012A00002F034FC2888001D2880DBF810000102C1
:1012B00021F0FF11001200F0FF100843CBF81000DE
:1012C000C0F30F4141EA0040CBF8100004220BF1BB
:1012D00010012888001902F019FC2888001D2880B8
:1012E000DBF81C00010221F0FF11000A00F0FF10E2
:1012F0000843CBF81C004FEA3040CBF81C00042216
:101300000BF11C012888001902F000FC2888001D40
:101310002880BBF81600010A41EA0020ABF816004D
:1013200002220BF116012888001902F0EFFB288831
:10133000801C2880411C298080B2DBF820100155D8
:1013400009F101095FFA89F998F804008145FFF66F
:1013500059AFB6F84321D6F845112888001902F094
:10136000D5FB2888B6F8431108182880B6F8431131
:101370000FF2904002F092FC3FE505287FF43DAD6E
:101380002888411C298098F8021001552888411CA2
:10139000298098F8031001552FE5F11C7078032877
:1013A00004D12888421C2A80B27A0255D1F8010063
:1013B000020222F0FF12000A00F0FF101043C1F8F1
:1013C00001004FEA3040C1F80100072228880019C7
:1013D00002F09CFB2888C01D28800EE5F11C0888BF
:1013E000020A42EA0020088002222888001902F03E
:1013F0008DFB2888801C2880FFE4F11C7278012A6C
:101400007FF4FBAC8078012815D12888421C2A8003
:1014100009780155B288D6F806102888001902F01C
:1014200075FB2888B18808182880B1880FF2E83049
:1014300002F034FCE1E402287FF4DFAC2888421C8F
:101440002A800A7802552888421C2A80C9790155C9
:10145000D3E4F11C0888020A42EA00200880022234
:101460002888001902F052FB2888801C2880C4E4D8
:10147000F01C29884A1C2A8001220A5529884A1C06
:101480002A8005220A5529884A1C2A80C1220A5529
:1014900029884A1C2A8042790A5529884A1C2A80B0
:1014A00042780A5529884A1C2A8080780855A4E485
:1014B000F61C29880B463078020727D5481C28805F
:1014C000307818552888411C2980F17901552888E1
:1014D000411C2980317A0155D6F80900010221F01A
:1014E000FF11000A00F0FF100843C6F809004FEA98
:1014F0003040C6F80900042206F1090128880019C5
:1015000002F004FB2888001D288076E4400721D5DE
:10151000481C2880307818552888411C298071780B
:101520000155D6F80300010221F0FF11000A00F076
:10153000FF100843C6F803004FEA3040C6F8030026
:101540000422F11C2888001902F0E0FA2888001D06
:10155000288052E4B278D6F80D10181902F0D6FAA5
:101560002888B1784018288047E4F61C30680102CA
:1015700021F0FF11001200F0FF1008433060011449
:1015800041EA00403060042231462888001902F008
:10159000BDFA2888001D28807068010221F0FF1123
:1015A000001200F0FF1008437060011441EA00408F
:1015B00070600422311D2888001902F0A7FA2888DB
:1015C000001D288019E4F61C3068010221F0FF118B
:1015D000001200F0FF1008433060C0F30F4141EAF1
:1015E00000403060042231462888001902F08EFA4B
:1015F0002888001D28807068010221F0FF11001268
:1016000000F0FF1008437060C0F30F4141EA004052
:1016100070600422311D2888001902F077FA2888AA
:10162000001D2880B068010221F0FF11001200F0B7
:10163000FF100843B060C0F30F4141EA0040B060C2
:10164000042206F108012888001902F05FFA2888B0
:10165000001D2880F068010221F0FF11001200F047
:10166000FF100843F060C0F30F4141EA0040F06012
:10167000042206F10C012888001902F047FA288894
:10168000001D2880FFF7B9BBF61C3068010221F06D
:10169000FF11001200F0FF1008433060011441EA0E
:1016A00000403060042231462888001902F02EFAEA
:1016B0002888001D28807068010221F0FF110012A7
:1016C00000F0FF1008437060011441EA00407060B0
:1016D0000422311D2888001902F018FA2888001DFC
:1016E0002880B068010221F0FF11001200F0FF1005
:1016F0000843B060011441EA0040B060042206F1E2
:1017000008012888001902F001FA2888001D2880A5
:10171000F2683369F06831691B0243EA126312020E
:1017200022F0FF1223F0FF13000A40EA0160090AC9
:1017300000F0FF1001F0FF1110431943F060316118
:10174000D6F80C80D6F81090F06831694FEA094954
:1017500049EA1849DFF8BC24134602EA084209EABC
:1017600003039046000C40EA01404FF6FF72104020
:101770004246104353EA1141F0603161F268336927
:10178000F06831691346084600211943F060316161
:10179000F0683169082206F10C012888001902F06E
:1017A000B5F92888083028807069010221F0FF11FE
:1017B000001200F0FF1008437061011441EA00407C
:1017C0007061042206F114012888001902F09EF9C4
:1017D0002888001D2880FFF710BBBDF8002029468F
:1017E0002046FFF798FA03F074FC0DF68C2DBDE847
:1017F000F08F000050442053462053656E742564DA
:10180000000000004F4A483A204154424420736986
:101810007A653A20256400004F4A483A20415044F6
:10182000522073697A653A20256400002DE9F04161
:1018300005460E4602F0C9F90746DFF8DC4320787A
:10184000401C20706078F021084202D0992003F0FB
:101850008DFE03F001FF6078401C607097F81C80DB
:10186000B8F1000F27D03088404480B2FEF752FD17
:10187000002803D031462846FEF71CFD3088411C65
:101880003180032141553088411C318000F80580AA
:10189000424607F11D013088401902F037F93088BF
:1018A000404430804FF4FA72002107F11D0002F02D
:1018B00007FF002038776078F021084202D0992095
:1018C00003F054FE6078401E6070C0B2002801D161
:1018D00003F0BCFEBDE8F04104F0A8B938B50446F9
:1018E0000D4602F072F9817A002909D1417B002965
:1018F00006D129884A1C2A8006220A5501214173F3
:1019000031BD38B504460D46288800280CD0204645
:10191000FFF78CFF29462046FFF7E0FF29462046C7
:10192000BDE83440FEF7C6BC31BD14B585B00491A6
:1019300001A90022134614461CC10A21ADF800106B
:1019400004218DF804108DF805000A4605A90DF153
:10195000060002F0DBF8042204A90DF10A0002F0EF
:10196000D5F800A901A8FEF7A5FC06B010BD80B50A
:1019700002F02BF94FF4967102F08AFB07208DF8E4
:1019800002000120ADF8000000A90DF10200FEF7F1
:1019900091FC01BD2DE9F04383B005460F4690460A
:1019A00002F013F981460026D5F80900041D2878B5
:1019B000014601297CD00F2939D035294AD0362952
:1019C0003FD040294FD07F2936D0802900F09C801D
:1019D000812900F0A380822900F0A080852900F0F1
:1019E0009D80862900F09A80882900F097808A29B6
:1019F00000F09C808B2900F0B7808C2900F0C38018
:101A00008D2900F0CE80DD2900F0D880DF2900F09C
:101A1000EC80F0292CD0F42934D0F6293DD0F829D7
:101A20005BD0F92949D0FF2900F0C08073E099F814
:101A30001A00207001206FE099F812022070012036
:101A40006AE004F09DFE15220146204602F05EF891
:101A5000012061E0012006F0D6FD304606F0D7FDFA
:101A60000120207058E0204606F0F0F8012053E0F5
:101A700004226A49204602F049F8012008F024F9BE
:101A8000012049E0484602F0ADFA082209F11001B0
:101A9000204602F03BF801203EE00322214630467A
:101AA0005F4B9B68D3F820311B6A9847012033E0D5
:101AB000204608F0C3FA01202EE0B5F80120B5F861
:101AC0000300C010C0EB0011D5F8050000EB811138
:101AD000204602F01BF801201EE03046ADF804005D
:101AE00001206979012900D1032007F0D6FB07F016
:101AF00010FCADF8040007F023FC022201A92046E7
:101B000002F004F8012007E0D5F805002070214616
:101B1000304601F086FA3046BDE8FE83314621703A
:101B2000214600F07F0001F07CFAF4E701202070EC
:101B30003B4845683746287F002801D13046EBE70F
:101B4000687A002804D1D5F820014068804707460C
:101B50002046D5F82011C9698847002FDBD0D5F879
:101B6000200180688047D6E70120B5F80310C1F353
:101B7000C101091D884040F002002070214601206B
:101B800001F04FFAC7E799F800002070012060705B
:101B900099F80500A07099F80600E0700120207106
:101BA000BAE7204608F05EFA0646B4E704F10802F8
:101BB000211D204608F028F90120ADE76879184971
:101BC00051F82050687A00280BD042463946284602
:101BD000FEF760FE1349082008F006FB0120207084
:101BE00001E030462070012096E768790C4951F8F1
:101BF0002050286995F8221090FBF1F0401E0090CB
:101C0000042200A9204601F081FF012084E70000A2
:101C1000ACE200200000FFFF28A8002068AA0020F6
:101C2000AC490120F0E100202DE9F041B6B00646B4
:101C300001F0CBFF054600F0FDFE8046D6F8090016
:101C4000041D3078002102914FF0FF3119910F46A9
:101C50000146312900F04D81322900F054813329A9
:101C600000F06081342900F06781372978D07D2920
:101C700000F0A680A12900F07B81A22900F0C78195
:101C8000A42900F0D281B12900F04984B22900F0E2
:101C90002086B82900F0E481C12900F00382CD2913
:101CA00000F0A680CE2900F0BB80D02932D0D12907
:101CB00028D0D22933D0D32937D0D42939D0D62926
:101CC0005AD0D72958D0D8295ED0D9295CD0EC2950
:101CD00000F08080F1295FD0F22900F0BA80F52968
:101CE00000F0DB80F72900F0F080FA2900F03F8651
:101CF000FB2900F03F86FD2900F0DB80FE2900F083
:101D00004386F2E00021284602F0CFF90020A873B4
:101D10000120EBE0002007F0D7FF0120E6E00121E1
:101D2000284602F0C2F90120E0E00020A87201205C
:101D3000DCE00120A872002068730120A873DFF89E
:101D40005C0C016808E08A6B92F91420012A02DB1E
:101D5000012281F8182109688142F4D10120C5E0EF
:101D6000002221461046DFF8383C1B68D3F82031AA
:101D70001B6A98470120B9E0D62801D1012000E074
:101D80000020E8720120B1E0D92801D1012000E053
:101D9000002028730120A9E000200DE000EB0801DD
:101DA000025D81F88C20022805D108F18C01025DCA
:101DB000CA70025D0A71401C0328EFDB012095E028
:101DC000207802F0EFF808F18C01487088F88C0058
:101DD00001208BE0237840F27672DFF8C81BDFF831
:101DE000C80B01F05BFF207806F0FAF901207DE0D6
:101DF000002511E0DFF8A80B466806EB85060222F5
:101E000004EB450106F1600001F080FE316EDFF861
:101E10009C0B01F043FF6D1C032DEBDB012065E003
:101E2000002512E0DFF8780B066806EB4506022273
:101E300004EB450106F1580001F068FEB6F95810B0
:101E4000DFF86C0B01F02AFF6D1C032DEADB01208B
:101E50004CE0D5E9040100F0800011F0000103D14D
:101E6000002801D1012041E008F18C01207862783E
:101E700012EB0020C880A078E27812EB00200881E5
:101E800004212046DFF8182BD269D2F8202192696C
:101E90009047002829D0012028E003222146012074
:101EA000DFF8FC3A9B68D3F820311B6A9847012081
:101EB0001CE01B2221460720DFF8E43A9B68D3F898
:101EC00020311B6A9847012010E0DFF8D40A8669A8
:101ED000D6F8200180688047002806D001222146DC
:101EE0000520D6F820311B6A9847002036B0BDE89F
:101EF000F08106F090FB012801D10120F6E7204691
:101F000006F000FBF1E706F086FB012801D1012075
:101F1000ECE7204606F023FB20780028E5D006F009
:101F20005BFBE2E706F077FB012801D10120DDE74A
:101F3000207806F058FBD8E706F06DFB012801D1A8
:101F40000120D3E7DFF86C0A01F0A8FE002006F0BC
:101F50005AFB012006F030FA04F0E3FD012006F000
:101F600056FB207806F05AFB06F090FA0120BDE7F8
:101F700094F900500422611C02A801F0C7FDB6F8D4
:101F80000100062806DB0422611D19A801F0BEFD30
:101F900094F909702846DFF8081A042802D10A6962
:101FA0000023937251F8206000F044FDD0E91E2315
:101FB000C2F3401800F03EFDD0E91E23C2F380209A
:101FC000804400F037FDD0E91E23C2F3800000EB0F
:101FD000080296F90800072804D1717A002901D077
:101FE000002A04D0182809D1707A002806D0717A06
:101FF000DFF8C40901F052FE012077E70097199B32
:1020000000220299284601F079F820706DE794F9D2
:1020100000500422611C02A801F078FD00231A463A
:102020000299284601F03CF960E794F90050042237
:10203000611C02A801F06AFDB6F80100062806DB63
:102040000422611D19A801F061FD94F9097000973F
:10205000199B00220299284601F0A1F9207044E75B
:1020600020780146032904D01A2910D02C290ED03B
:1020700011E060780DF10D025070012805D1A078B3
:102080008DF80F00204601F059FB01202EE7204675
:1020900001F054FBF9E794F9011040B20020C0466A
:1020A000C0B223E720780146491E51D00D390DD02A
:1020B000C91E55D0491E032921D9091F00F0A68049
:1020C000491E00F0048119393AD010E20E208DF833
:1020D0000C0060780DF10D025070A1788DF80F1092
:1020E000E2780DF10F035A700023ADF8113052B2AF
:1020F00049B240B202F02AF801F01EFBF7E18DF878
:102100000C000146122903D10DF10D0062784270D6
:10211000132902D160788DF80F00142903D10DF135
:102120000F0062784270152903D10DF10D0061781E
:10213000417062782178DFF8840801F0AFFDD6E1C4
:1021400030208DF80C000DF10D0061784170CEE16A
:1021500001208DF80C000DF10F0061784170C6E18F
:102160000DF10D0061784170A0788DF80F000DF130
:102170000F00E178417020798DF81100002802D01D
:1021800001281FD030E06079A179090401EB0060DB
:10219000E17900EB0120217A4018CDF812000DF111
:1021A0001206607AA17A11EB0020B080E07A217BE0
:1021B00011EB0020F080607BA17B11EB0020ADF8DB
:1021C0001A0011E06079A17911EB0020ADF812003E
:1021D0000DF11206E079217A11EB00207080607A0F
:1021E000A17A11EB0020B0801AA80DF10E010E2289
:1021F00008F02CF81AA80FC802F0CBF802F030F95A
:10220000012840F0748101F0ECFA70E16078A17867
:10221000090401EB0060E17800EB0120217940180E
:10222000CDF80E006179A279120402EB0161E27926
:1022300001EB0221227A8918CDF81210627AA37A72
:102240001B0403EB0262E37A02EB0322237BD21826
:102250000DF112067260637B8DF81A30A37B8DF846
:102260001B300DF11B03E57B5D70257C9D70657C4B
:10227000DD70A57CE67C16EB05252DB29D80267DC4
:1022800005EB0625667DAD19DD80A57D1D72002854
:1022900003D1002901D1002A0CD00DF10E0184B028
:1022A0006846162207F0D2FF0FBC02F0FFF802F0DA
:1022B000DFF801E002F0E1F80DF10E0184B06846AC
:1022C000162207F0C3FF0FBC01F077FA0FE1607828
:1022D0008DF80D001D283ED10DF11206A178717107
:1022E000A17801290DD1E178227912EB0121ADF815
:1022F0000E1089B20A460146DFF8C40601F0CEFC92
:10230000F5E002290BD1E078217911EB0021ADF83D
:10231000101089B2DFF8AC0601F0C0FCE7E0032939
:102320000AD1E078217911EB0021F18089B2DFF840
:10233000980601F0B3FCDAE0042940F0D880E07898
:10234000217911EB0021ADF81A1089B2DFF87C0673
:1023500001F0A4FCCBE0032828D1A1780DF15E05A3
:102360006970DFF86C0601F099FC6878012816D1D5
:102370000020142880F2BB8004EB8001CA780B791E
:102380001B0403EB02624B7902EB0322897951189B
:1023900003AA02EB8002C2F80210401CE9E70228FF
:1023A00040F0A580E0788DF85E00A0E01C2827D1E1
:1023B000A0788DF81100A078012808D1E1780DF1FE
:1023C0000D025170DFF80C0601F068FC8FE0022866
:1023D00007D1E1788DF80F10DFF8FC0501F05EFC05
:1023E00085E0032800F08380052840F08080E178B4
:1023F0000DF10F035970DFF8E40501F04FFC76E0B2
:102400002C2830D10DF11200A1788171A07801281B
:1024100003D1E0788DF8120069E0022806D1E07857
:10242000217911EB0020ADF8190060E0032806D1F6
:10243000E078217911EB0020ADF81B0057E004286B
:1024400007D1E078217911EB00200DF11B014880C4
:102450004DE005284BD1E078217911EB00200DF1FA
:102460001B01888043E030281BD1A0788DF80F0035
:10247000A078012804D10DF10D00E178417036E01B
:10248000022834D140F62E22DFF81815DFF8500567
:1024900001F004FCB6F80110E01C08F02CFC01204F
:1024A00024E5342823D10DF11200A1780171A07820
:1024B000012817D10DF10E00E1782279120402EB08
:1024C0000161627901EB0221A279891800EE101AEC
:1024D000B8EEC00ADFED840A80EE200A10EE101A72
:1024E000016004E0022802D1E078CDF81200062055
:1024F0008DF8780020788DF879000DF17B0003A924
:10250000552207F0A3FE0DF179000B214170002048
:10251000ADF8D0001EA801F07BF9C0B2E6E4207847
:1025200001463C2905DBDFF8BC0401F0B7FB0020C5
:10253000DCE4C1EB0112DFF8B01401EB8201897E0B
:10254000012940F09281014603292ED006296BD043
:10255000092931D00C294BD00D2957D0192900F069
:1025600096801A296DD01B2900F0A6801C2900F046
:10257000E4801D2900F0BA801E2900F0EC80262995
:1025800000F0F780272900F002812C2900F0278134
:102590002D2900F03D812F2900F04F81302900F0D6
:1025A0004581342900F055815AE10322611C0DF167
:1025B0000E0001F0ABFA58E10722611C0DF10E008C
:1025C00001F0A4FABDF80E00010A41EA0020ADF8BE
:1025D0000E00BDF81000010A41EA0020ADF810001D
:1025E000BDF81200010A41EA0020ADF812003CE1FA
:1025F0000322611C0DF10E0001F088FABDF80F00F6
:10260000010A41EA0020ADF80F002EE10322611C0F
:102610000DF10E0001F07AFABDF80F00010A41EA4F
:102620000020ADF80F0020E10122611C0DF10E0029
:1026300001F06CFA0DF10D004178EC4801F02EFB31
:1026400013E10B22611C0DF10E0001F05FFADDF8C1
:102650000F00010221F0FF11000A00F0FF100843F3
:10266000CDF80F004FEA3040CDF80F000DF1120603
:102670007088010A41EA00207080002396F9062044
:1026800096F9051096F9040001F060FDEDE00622D0
:10269000611C0DF10E0001F039FABDF80E00010ABF
:1026A00041EA0020ADF80E00BDF81200010A41EA2F
:1026B0000020ADF81200D8E00422611C0DF10E00DC
:1026C00001F024FABDF80E00010A41EA0020ADF83D
:1026D0000E00BDF81000010A41EA0020ADF810001C
:1026E000C34801F0DBFAC0E000401C460922611C2F
:1026F0000DF10E0001F00AFABDF80E00010A41EAE0
:102700000020ADF80E00BDF81000010A41EA0020DB
:10271000ADF81000BDF81200010A41EA0020ADF842
:1027200012000DF11206002396F9042096F9031009
:1027300096F9020001F00AFD97E00DF10D006178B5
:102740004170A0788DF80F00A27861780FF2A82070
:1027500001F0A4FA89E00322611C0DF10E0001F0E2
:10276000D5F9BDF80F00010A41EA0020ADF80F00CD
:102770007BE00522611C0DF10E0001F0C7F9BDF8E8
:102780000F00010A41EA0020ADF80F006DE00A22B7
:10279000611C0DF10E0001F0B9F9BDF90E00C0F396
:1027A000072141EA0020ADF80E00BDF91000C0F38A
:1027B000072141EA0020ADF81000BDF91200C0F376
:1027C000072141EA0020ADF812000DF11206B6F91A
:1027D0000200C0F3072141EA0020708045E0082292
:1027E000611C0DF10E0001F091F9BDF81000010A15
:1027F00041EA0020ADF810000DF11206002396F911
:10280000032096F9021096F9010001F09FFC2CE0DC
:102810000222611C0DF10E0001F078F9BDF80E00E6
:10282000010A41EA0020ADF80E001EE00222611C00
:102830000DF10E0001F06AF917E00DF10D00E178DD
:10284000417020798DF80F000DF10F006179417012
:102850000BE00922611C0DF10E0001F057F904E0B4
:102860008DF80C0060788DF80D0020780146052960
:1028700008D1604801210170687A002810D108460B
:10288000FFF734BB18290BD18DF80C0060788DF858
:102890000D000DF10D00A1784170E0788DF80F006A
:1028A00000208DF8780020788DF879000DF17B00FC
:1028B00003A9552207F0CAFC0DF179000B214170E4
:1028C0000020ADF8D0001EA800F0A2FFC0B2FFF7B4
:1028D0000DBB207801463C2906DB0FF22C1001F0DD
:1028E000DDF90020FFF702BB052905D14148002191
:1028F00001700120FFF7FABA1A291CD10822611CC5
:102900000DF10E0001F002F9DDF80F00010221F0D7
:10291000FF11000A00F0FF100843CDF80F004FEA46
:102920003040CDF80F000DF112067088010A41EA1F
:102930000020708005E02C2903D10DF10D00617895
:10294000417001208DF8780020788DF879000DF124
:102950007B0003A9552207F079FC0DF179000B21CA
:1029600041701EA800F054FFC0B2FFF7BFBA0120AB
:10297000FFF7BCBA2078002803D10FF2AC0008F0B2
:10298000EFFE0120FFF7B2BA04F10802211D204634
:1029900007F0F8F90120FFF7A9BA00002C40002049
:1029A000AC490120FC61030814620308406203087B
:1029B0004C62030858620308686203088C620308CB
:1029C0009C620308AC620308B8620308C46203088F
:1029D000D0620308E4620308F86203080C6303088A
:1029E000206303085C630308ACE2002078630308FB
:1029F00084630308F5560120415044522041444469
:102A000020256420256400004C696272617279207F
:102A100072616E6765206973206F7665722C205233
:102A2000656D6F766500000051505F524551554508
:102A30005354000000487047D046012080B5FFF78E
:102A4000F9FFDFF8441B4860012002BD80B507F0A4
:102A50005BFADFF8381BD1E90023801A02BD01F0D0
:102A6000A5BD2DE9F8430446002005460646DFF8DB
:102A7000201B496804F108073A697B6802EB0308E8
:102A800094F90820002A15D1B8F90000B8F90250CD
:102A9000B8F90460B7F85010411AA8F80010B7F858
:102AA0005210691AA8F80210B7F85410711AA8F851
:102AB000041040E004F16C09012A27D1B8F8001095
:102AC000A4F86C10B8F80210A9F80210B8F80410B5
:102AD000A9F80410B4F86C10BA6D891AA8F800109F
:102AE000B9F80210FA6D891AA8F80210B9F80410A2
:102AF0003A6E891AA8F80410B96DA8F80610F96D95
:102B0000A8F80810396EA8F80A1014E0B4F86C2080
:102B1000A8F80020B9F80220A8F80220B9F804208B
:102B2000A8F804200A6EA8F806204A6EA8F8082023
:102B3000896EA8F80A1094F90810002951D1B8F943
:102B40000010C913B1EBE03F14D0B7F95010C9130E
:102B5000B1EBE03F0ED00FF6502001F09FF8B8F92E
:102B60000000012802DBDFF82C0A01E047F6FF70C5
:102B7000A8F80000B8F90210C913B1EBE53F14D072
:102B8000B7F95210C913B1EBE53F0ED00FF6242070
:102B900001F084F8B8F90200012802DBDFF8F4093B
:102BA00001E047F6FF70A8F80200B8F90410C91355
:102BB000B1EBE63F70D0B7F95410C913B1EBE63F63
:102BC0006AD00FF6FC1001F069F8B8F9040001288A
:102BD00002DBDFF8C00901E047F6FF70A8F8040047
:102BE0005AE0012958D1B4F96C00B8F90010C913A2
:102BF000B1EBE03F14D0B7F95810C913B1EBE03F87
:102C00000ED00FF6A41001F049F8B8F90000012821
:102C100002DBDFF8800901E047F6FF70A8F800004A
:102C200004F16C09B9F90200B8F90210C913B1EB4B
:102C3000E03F14D0B7F95C10C913B1EBE03F0ED000
:102C40000FF6701001F02AF8B8F90200012802DB33
:102C5000DFF8400901E047F6FF70A8F80200B9F973
:102C60000400B8F90410C913B1EBE03F14D0B7F970
:102C70006010C913B1EBE03F0ED00FF6441001F025
:102C80000DF8B8F90400012802DBDFF8080901E0BB
:102C900047F6FF70A8F8040094F90800002804D152
:102CA000002000E0401C0328FCDBBDE8F1830000AD
:102CB000F8B50446A069E1684518002794F9086052
:102CC000052E02D30E2E40F0B480012E01D00E2E20
:102CD00002D12046FFF7C5FE3046012804D9C01EA8
:102CE00002D00B3840F0A080002E01D14FF6FF77C4
:102CF000DFF8940840680E2E03D0301890F88C004E
:102D000001E090F88D00401E062870D8DFE800F042
:102D10000413222F3E4D5E00B5F902002988791A6E
:102D2000B5F90420B5F90830B5F806C0A7EB0C0CCE
:102D3000B5F90A7067E02888381A6988791AB5F9F0
:102D40000420EB88FB1AB5F808C0A7EB0C0CB5F90A
:102D50000A7058E06888381AB5F90010B5F90420EF
:102D60002B89FB1AB5F906C0B5F90A704BE0288823
:102D7000381AB5F90210AA88BA1AEB88FB1AB5F905
:102D800008C0B5F80AE0A7EB0E073CE0B5F9020071
:102D9000B5F90010AA88BA1AB5F90830B5F906C015
:102DA000B5F80AE0A7EB0E072DE0B5F90000698839
:102DB000791AAA88BA1AB5F90630B5F808C0A7EB8F
:102DC0000C0CB5F80AE0A7EB0E071CE06888381A6F
:102DD0002988791AAA88BA1A2B89FB1AB5F806C06D
:102DE000A7EB0C0CB5F80AE0A7EB0E070BE0B5F962
:102DF0000000B5F90210B5F90420B5F90630B5F9AF
:102E000008C0B5F90A70012E07D14FF0000E01E09D
:102E10000EF1010EBEF1030FFADB28806980AA8053
:102E2000EB80A5F808C06F81002E02D12046FFF785
:102E300018FE0120F2BD000070B404680D68166829
:102E40005B1E062B27D8DFE803F004080D11161BC4
:102E500020000560604208601DE062420260684236
:102E6000086018E06A4202600C6014E06142016090
:102E7000704210600FE005600C60704210600AE064
:102E8000684208607042106005E06B420360604277
:102E900008607042106070BC7047000070B52DED86
:102EA000028B82B08169C2688A1890F908100846BE
:102EB0000A2800F2AD80DFE800F0062B89ABAB6595
:102EC000ABABAB96A400B2F90240B2F90450DFF804
:102ED000B80641689FED860AB2F9000000EE900A3C
:102EE000F8EEE00A60EE800AC1ED000A00EE904ABA
:102EF000F8EEE00A60EE800AC1ED010A00EE905A99
:102F0000F8EEE00A20EE800A081D80ED010A83E059
:102F1000B2F90240B2F90450DFF86C0641680E1DA8
:102F20009FED748BB2F9000000EE100AB8EEC00AF3
:102F300010EE100A08F0CAFC53EC182B08F0EEFC57
:102F400008F0BEFDB06000EE104AB8EEC00A10EE08
:102F5000100A08F0BBFC53EC182B08F0DFFC08F05B
:102F6000AFFDF06000EE105AB8EEC00A10EE100A85
:102F700008F0ACFC53EC182B08F0D0FC08F0A0FDD6
:102F8000306149E00020009010680090DFF8F805FB
:102F900041689DED000AB8EEC00ADFEDC00A20EEE0
:102FA000200A81ED0C0A91ED0C0AB5EE400AF1EE13
:102FB00010FA31D090ED020AD1ED0C0A30EE200A61
:102FC00080ED020A0188491C018025E0DFF8B80580
:102FD00041681088A1F85A0001F25A0051884180D6
:102FE0009188818018E0DFF8A005416801F25A005D
:102FF0001188C1805188018191884181D188818166
:103000000AE0DFF884054068118880F8681003E062
:103010000FF2B85000F042FE012002B0BDEC028B6E
:1030200070BD70B50D46DFF8681551F820400026D8
:10303000207F002801D1304670BD607A002804D07E
:10304000D4F820018068804706462846D4F820112D
:10305000C96988470546002E03D0D4F8200140688E
:103060008047284670BD01207047F0B4002A14D470
:1030700000F10804A57EA66892FBF1F76F43B74202
:1030800002DA2264626408E090F908700C2F02D022
:1030900096FBF5F24A4322646264002B03D499073D
:1030A00001D508300376F0BC70470021816441618E
:1030B00081610269C06801F003BB042817D101F1E6
:1030C0000C008A7A012A09D0072242750B228275E8
:1030D000DFF8C424CA600B21416070471522427595
:1030E00019228275DFF8B424CA6019214160704743
:1030F00060F69C3A89AD84FA0A74513F2DE9F24F8B
:1031000098B08046144699460020ADF858008DF8D6
:1031100001000DF101050A2068700020A870E87018
:10312000B8F11C0F7BD24646DFF8640450F82670D5
:103130004FF0020A387F002871D01898C82802D1B1
:10314000B420189003E0422801D13C201890002CB4
:1031500002D1012087F898009DF988B0BBF1000FDB
:1031600009D45FEACB7006D55B464A4618993846C3
:10317000FFF779FF8FE0002C14D1787A00280BD16B
:1031800031460FF2544000F089FD59463846FFF7AA
:103190008CFF012087F899005B464A46189938460B
:1031A000FFF763FF07F58E790F2E01D0102E06D1A1
:1031B0004146C9B218A8D9F80420926990471A2E3E
:1031C00006D14146C9B218A8D9F80420926990479F
:1031D0001B2E06D14146C9B218A8D9F8042092691D
:1031E000904739464046FFF768FF787A00281FD19C
:1031F000214649B23846D9F808201268904700287D
:103200000FD0D9F8040040688047002805D1514606
:10321000A1F1010AC9B20029F3D1002801D100208F
:1032200039E0214649B23846D9F80820526890471B
:10323000787A401C78720C2E0CD0112E0AD00D2EEC
:1032400008D0224652B218993846D9F808301B697E
:1032500098470EE0B86B1421C160002C09D1002002
:1032600087F81901C7F81C01FFF7F0FB0021C7E937
:10327000240100F0F0F8162E0CD1002C0AD1002009
:103280008DF800003B208DF801000A20687000A82E
:1032900000F0BEFA012019B0BDE8F08F0AD7233C38
:1032A0002DE9F04798B007460E461446194600200F
:1032B000ADF858008DF801000DF101050A20687085
:1032C0000020A870E8701C2F08D2B14850F8278061
:1032D0004FF0020998F81C00002801D100205BE0A3
:1032E000C82E01D1B42602E0422E00D13C26002C8B
:1032F00002D14046FFF7D9FE98F8090001281DD1F8
:1033000008F5907A214649B24046DAF804209268DE
:10331000904700280BD0D8F820018068804700280B
:1033200005D14846A0F10109C0B20028F3D12146D9
:1033300049B24046DAF80420D268904798F809006C
:10334000002802D0401E88F809000C2F0DD0112F44
:103350000BD00D2F09D0224652B23146404608F517
:1033600090735B685B69984704E0D8F838004FF0C9
:10337000FF31C16000F06FF8162F0CD1002C0AD17C
:1033800001208DF800003B208DF801000A206870B4
:1033900000A800F03DFA012018B0BDE8F0872DE943
:1033A000F04106460C4615461A461C2E20D2784897
:1033B00050F82670387F00281AD0C82C01D1B424C8
:1033C00002E0422C00D13C249DF91830002B06D499
:1033D000D80704D521463846BDE8F04143E605EB61
:1033E000450007EB8008D8F838008068002801D530
:1033F00000202EE021463846FFF737FE0C2E27D05E
:10340000112E25D00D2E23D0D8F8380080688442A4
:103410001ED0012C1CDB0FF2C81000F03FFC2A4626
:1034200052B2D8F8380081683846D7F824315B6941
:1034300098472A4652B221463846D7F824311B69AC
:10344000984700F008F8002D02D1012087F8980075
:103450000120BDE8F08170B56FF000463446504859
:10346000016804E08A68A24200DA144609688142D1
:10347000F8D14C4D2878401C28706878F02108421B
:1034800002D0992002F072F802F0E6F86878401C49
:103490006870B44200D100243B4E7068C0F884408C
:1034A00000F18402536821468B4211D0002901D0DB
:1034B000002B0AD151600FF2381000F0EFFB70685A
:1034C000D0F8880000F0C6FB02E0012008F04CFBB9
:1034D0006878F021084202D0992002F047F8687815
:1034E000401E6870C0B2002801D102F0AFF802F0AF
:1034F0009DFB012070BD38B505462A4C2078401C44
:1035000020706078F021084202D0992002F02EF855
:1035100002F0A2F86078401C607029460FF2E400C7
:1035200000F0BCFB18484068C0F888501C4801688F
:1035300005E08A68B2FBF5F26A43CA600968814215
:10354000F7D16078F021084202D0992002F00EF8FD
:103550006078401E6070C0B2002801D102F076F899
:10356000BDE8314002F062BB0D490A6808E013690A
:10357000012B01DAD368136113691B1A13611268F6
:103580008A42F4D170470000C4540120C055012084
:10359000AC4901200080FFFF504700202453012048
:1035A0002040002028A8002058206973206F7665ED
:1035B0007200000059206973206F76657200000068
:1035C0005A206973206F766572000000554353548A
:1035D000282564294E5300004164642025640000BE
:1035E0006368616E67652072617465320000000077
:1035F000675F707453682D3E6354696D6572203D3A
:10360000202564006374696D6572203D2025640087
:103610007C487047F8B50C461646012500282BD18A
:10362000C6EB0610774901EB8007386AE040C00717
:1036300008D523463A6A31460FF2883000F02EFB57
:103640000220F2BD4FF0FF30009003462A46796811
:103650002046FFF753FD00280CD023463A6A314636
:103660000FF2703000F01AFB386A2946A140084377
:1036700038622CE00220F2BD012828D1C6EB0610EA
:10368000604901EB8007386AE040C00708D4234650
:103690003A6A31460FF24C3000F000FB032516E089
:1036A0004FF0FF332A4679682046FFF7F9FD0028DE
:1036B00007D023463A6A31460FF2383000F0EEFA6E
:1036C00000E00325386A0121A1408843386228467A
:1036D000F2BD01F0C8BD02B598B00021ADF8581098
:1036E0008DF801100DF101010A224A7000228A7042
:1036F000CA7005218DF800108DF80100042218A968
:103700000DF1030000F002FA0020ADF8580000A807
:1037100000F07EF819B000BD10B40022884201D339
:10372000421A06E00B1A384CA34202D3374A10184B
:10373000421A104610BC704708F080BF38B5447874
:1037400085780078032822D01A2802D02C282AD085
:1037500031BD012C0CD101200AF0E2FB01232246ED
:103760001A210FF2A02001B0BDE8304000F096BA57
:10377000022C21D102200AF0D3FB022322461A2177
:103780000FF2942001B0BDE8304000F087BA012C60
:1037900012D1284608F06FFF29460FF29020BDE8AD
:1037A000344000F07BBA012C06D129460FF2882064
:1037B000BDE8344000F072BA31BD0FB480B50028C6
:1037C00005D10846002802D11046002804D00AF08E
:1037D0007CFE0BF013F901E00AF060FE01BC5DF81D
:1037E00014FB0AF085BE00223C2809D2C0EB00136E
:1037F000044800EB8300006AC840C00700D50122DE
:1038000010467047ACE20020A1780F05005C260549
:1038100030B595B00446012594F90000062800F261
:10382000BC80DFE800F0042648647AB2B600E11CF0
:1038300082B06846552206F009FD0CBC94F90210CE
:1038400094F9010001F049F9022809D1607801F0EA
:103850000EFB002561780FF2E81000F01FFAA2E0DD
:10386000032840F0A08061780FF2DC1000F016FA17
:1038700099E060781A280BD1E01C01F0BDFDA37A15
:10388000D4F8062061790FF2C81000F007FA04E0BE
:103890002C2802D1E01C01F0AFFD94F9021094F93C
:1038A000010001F00FFA03287DD161780FF2B81002
:1038B00000F0F4F977E0B4F8581000A801F0F1FA3C
:1038C0009DF9040002280AD1009800B201F0CFFA55
:1038D000002500990FF2981000F0E0F963E003284A
:1038E00061D100990FF2901000F0D8F95BE00BF075
:1038F00040FE022809D1607801F0B9FA002561780C
:103900000FF27C1000F0CAF94DE003284BD161782A
:103910000FF2741000F0C2F945E0607805280CD170
:1039200028460BF008FF02280DD003283BD1617810
:103930000FF2641000F0B2F935E002280DD10CF05E
:1039400000F80228F1D1607801F091FA0025617841
:103950000FF23C1000F0A2F925E02F2823D10CF043
:103960005FF9022809D1607801F081FA00256178B9
:103970000FF22C1000F092F915E0032813D16178B2
:103980000FF2241000F08AF90DE0204601F0EEFA63
:1039900009E0204601F08DFC05E061780FF210107F
:1039A00000F07CF90025284615B030BD0120704795
:1039B0000FB4022004B07047012070470020704708
:1039C00070470000534D4143202564202564202585
:1039D00064000000534D41202564202564202564A7
:1039E00000000000534D524320256420256420250B
:1039F00064000000534D5220256420256420256476
:103A0000000000004154205249204E6F72202D25A5
:103A100064202564202564004154205249204261DD
:103A200074202D25642025642025640050442055F1
:103A3000542D256400000000534C4D2025640000E7
:103A4000414C4F4620256400414C434620256400EC
:103A50004F4A4820454C203078257820307825780A
:103A60002030782578000000524C43462025640021
:103A7000504C4F4620256400504C4346202564009E
:103A800050414F46202564005041434620256400A4
:103A900050504F4620256400505043462025640076
:103AA00050534F4620256400505343462025640060
:103AB0004558204C4D454C202564000010B50400AD
:103AC00010480078002805D10F480CF06AF90D481D
:103AD000012101700C480CF09EF920000DF06EF8E9
:103AE000040009480CF0CBF9200010BD10B504000B
:103AF00005480CF090F920000DF0BAF902480CF0DE
:103B0000BEF910BDFD5601209054012010B50400EF
:103B1000200006F09BFB200010BD10B450F8041BE1
:103B200081B102681218001D50F8043BDC0744BF45
:103B3000A9F10104E31852F8044B43F8044B091FA0
:103B4000F9D1EBE710BC704738B504000D001748F9
:103B50000078401C1549087015480078002802D0EC
:103B6000A12001F003FD02F020F8A07E662802D01B
:103B7000822001F0FBFC802080F3118800BF00BF91
:103B800008E0382120000DF001FC802080F311882E
:103B900000BF00BFE06821698842F2D02900200000
:103BA0000DF018FC02F042F831BD00BF28A800203B
:103BB000FB56012010B5DFF8D4494FF406720021FE
:103BC000204600F07DFD204610BDDFF8C00970479B
:103BD00010B5FFF7EFFF044600231A4611460846CA
:103BE00000F0B4FAC046C04604F0C4FF0A212046E3
:103BF00000F03DF805F09EFA204600F043FA20461A
:103C000000F018F8DFF88809006805F062F920462E
:103C100000F09BF900F041FB00F0E2F90020607237
:103C2000A072E0722073012060730020E076A07320
:103C3000012010BD10B50446DFF8580905F0ABF8B7
:103C40000120607110BD10B5044605F0C0F90120D7
:103C5000A07110BD80B505F0A7FB012002BD10B515
:103C60000446E07905F098FC0121217010BD70B583
:103C700004460025E679E171FFF7F1FF002807D03F
:103C80002046FFF7D7FF2046FFF7DDFF012503E0C1
:103C9000E6712046FFF7E3FF284670BD0EB470B50D
:103CA000C1B0054600A84FF4807100F047FDFFF752
:103CB0008CFF044645AB2A464FF4807100A80DF0F6
:103CC000F5FB00A80DF010FC451C00A828180021E9
:103CD00000F8011CDFF8C0683078401C3070707844
:103CE000F021084202D0992001F040FC01F0B4FC20
:103CF0007078401C7070207F2818B0F5FA7F10DAB9
:103D0000207F002803D0207F00190A2101772A464E
:103D100000A9207F00191D30FFF7F8FE207F28182A
:103D200020777078F021084202D0992001F01EFC23
:103D30007078401E7070C0B2002801D101F086FC7E
:103D400001F074FF41B070BC5DF810FBDFF80808AB
:103D5000DFF840180160704710B50446FFF735FFE3
:103D6000D0E9042310461946224601F0EBFB00F08F
:103D7000010011F0000101D100280ED0DFF81C482D
:103D80002068401C20601E2807DB0FF62C00FFF780
:103D900085FF05F079FC0020206010BDDFF8FC07EE
:103DA0000021016070472DE9F84305460E4617468D
:103DB0004FF00208DFF8E0476078F021084202D0B7
:103DC000992001F0D3FB01F047FC6078401C607043
:103DD0009DF80000401E8DF8000017F8019B284652
:103DE000FFF7B4FF00AB4A463946304605F092FC77
:103DF000002812D06078F021084202D0992001F00A
:103E0000B5FB6078401E6070C0B2002801D101F09F
:103E10001DFCFFF7C3FF01201FE05FFA88F8424650
:103E200029460FF2A870FFF739FF4046A0F10108BC
:103E30000028D7D16078F021084202D0992001F003
:103E400095FB6078401E6070C0B2002801D101F07F
:103E5000FDFB2846FFF780FF0020BDE8F2832DE937
:103E6000F04704460D4616461F46DFF8F4860898CC
:103E700088F80000DFF8209799F80100F021084247
:103E800002D0992001F072FB01F0E6FB99F80100E5
:103E9000401C89F801002046FFF758FF4FF0020A46
:103EA000434632463946284605F0E2FC002815D044
:103EB00099F80100F021084202D0992001F056FB48
:103EC00099F80100401E89F80100C0B2002801D114
:103ED00001F0BCFBFFF762FF012022E05FFA8AFAE3
:103EE000524621460FF2F060FFF7D8FE5046A0F18F
:103EF000010A0028D4D199F80100F021084202D02B
:103F0000992001F033FB99F80100401E89F8010067
:103F1000C0B2002801D101F099FB2046FFF71CFF39
:103F20000020BDE8F08780B51146029A184604F0DB
:103F3000AFFF012002BD80B510465A1E92B2017833
:103F4000401C04F085FF012002BD1CB50446012081
:103F5000009001AB8F221B210020FFF7E4FF9DF8AA
:103F6000043040F211220FF27C610FF29060FFF7F3
:103F700095FE9DF80410692907D1012084F81202EA
:103F8000CAA0FFF78BFE012016BD0FF28860FFF775
:103F900085FE012084F812020FF29460FFF77EFE86
:103FA000012016BD30B587B0044600A80FF29C6111
:103FB000182206F05BF9FFF708FE90F8120200A93C
:103FC00001EBC000255CFFF700FE2B46224690F86F
:103FD00012120FF29060FFF761FE284607B030BD65
:103FE0000DF062BF2DE9F843054602264FF00008A8
:103FF000DFF8689516E03046461EC0B2002814D19E
:10400000002C0CD1D5E904670120002142460EF0B6
:1040100081F826EA000027EA0101C5E90401022629
:1040200008F10108B8F11C0F18DA59F82800D0F887
:104030002001006880470446012CDCD1D5E90467E3
:104040000120002142460EF065F830433943C5E9AE
:10405000040159F8280001210177D1E7D5E90401CD
:10406000002901D1032807D0002901D1022803D05B
:10407000002905D1012803D140F48050C5E904018D
:10408000BDE8F18305F039BD05F093BD05F049BDEC
:10409000DFF80405026A036A00BF00BF00BF00BF6B
:1040A00000BF9B1A8B42F6DB7047417230B597B068
:1040B000FCF76AF80446FFF788FD054600A85C2176
:1040C00000F03CFB0020ADF858008DF801000DF128
:1040D00001000A21417000218170C170697A0029B4
:1040E0000DD0002C18D000218DF8001005218DF87E
:1040F00001100B21417000A8FFF78AFB0CE0002C97
:104100000AD001218DF8001005218DF801100B2136
:10411000417000A8FFF77CFB17B030BD05F068BD0B
:1041200005F070BD01210846F8E701210846F7E7D0
:1041300002210120F2E702210120F1E705F06CBD28
:1041400010B50446FFF741FD447610BD2DE9F04758
:1041500082B00C4615462F46264680464FF47A71AB
:104160004FF03C0C4FF4616918FB09F216FB0C226E
:10417000BA1801FB0232DFF8ECE39EF900A01AFB4B
:1041800009F99EF901A01AFB0C9C9EF902904CFAC9
:1041900089FCBEF9039001FB0C919EF808C0BCF1AC
:1041A000000F22D144EA00012943194302D0012122
:1041B0008EF808108EF80000B8F1000F04D59EF8B4
:1041C000000018308EF800008EF801408EF8025082
:1041D000AEF8033000933B4632469EF900100FF2D2
:1041E000CC40FFF75BFDBDE8F38791420DD3A1EB17
:1041F000020CACF2D17CDFF8A893CC45DAD30FF2F5
:10420000884002B0BDE8F04748E5D3D2A2EB010CEC
:10421000ACF2D179DFF888A3D145CBD363460FF256
:10422000784002B0BDE8F04738E510B504002FD063
:10423000FCF794F8CB49CA68002A00D0841AB1F878
:104240000320A218A1F8032012B2B2F57A7F06DB90
:10425000A2F57A72A1F803208A78521C8A7091F92B
:1042600002203C2A04DB3C3A8A704A78521C4A708D
:1042700091F901203C2A04DB3C3A4A700A78521C2E
:104280000A7091F90020182A01DB00220A70C86028
:1042900010BDB449052205F0D9BFB3480021017013
:1042A00041701E22B14800F00BBA000053544D007B
:1042B0003FB400210120AC4A1278002A0CD12CE036
:1042C0005C68019DAC4224D11B89BDF80840A34223
:1042D0001FD10020491CC9B291421EDAC1EBC103B3
:1042E000A24C04EB43039DF80340DD78A54213D1B3
:1042F000002CE5D09C88BDF80450AC4209D1DC8884
:10430000BDF80650AC4204D11B89BDF80840A34259
:10431000DFD000F00100DDE7012004B030BC7047C1
:104320007FB40020014626E0C0EBC00254008F4D50
:1043300066193C224FF46163645D757812FB05F5E4
:1043400013FB0454B57864199DF800509DF8016082
:1043500012FB06F213FB05229DF8023052FA83F29B
:10436000A24201D2824B9A18121BB2F5966F00D965
:10437000491C401CC0B27C4A13789842D4DBC9B2B5
:104380008B4202D20020107001E0581A10707FBCDE
:1043900070472DE9FF419DF80340022C5EDA00A82A
:1043A0000FC8FFF785FF012858D100A80FC8FFF7F5
:1043B000B7FF9DF802509DF801606C4FDFF8A881AF
:1043C00098F80000032825D13C214FF461603A7829
:1043D0007B7811FB03F310FB0232BB78D2189DF8F7
:1043E000003011FB06F110FB031050FA85F09042EB
:1043F00001D25F490818811AB1F5966F02D94FF4BE
:10440000966000E0801AA8F80200FFF746FF01203E
:1044100088F8010098F80000C0EBC00149009DF841
:104420000020CA55C9194E708D70CC70BDF8082097
:10443000002C09D1019B4B600A81BDF80A204A81FA
:10444000BDF80C208A8106E0BDF804308B80BDF8F1
:104450000630CB800A81401C88F80000BDE8FF814F
:104460004149487800224A7070473F484088704769
:10447000242200214B4800F023B91CB500A8FFF707
:1044800008FF484C24220021204600F019F99DF82D
:104490000000607604F219009DF8011041709DF84B
:1044A00002108170FF21817213BD00000FB410B59E
:1044B0002DED028B2F4C10460DF03EFE2E4A2F4B59
:1044C00007F02CFA206161619FED2D8B04980DF0AF
:1044D00033FE53EC182B07F021FA20606160059839
:1044E0000DF02AFE53EC182B07F018FAA060E160DB
:1044F0009DF81C00207604F118009DF81D104170F5
:104500009DF81E1081709DF81F10C1709DF820103D
:104510000171BDF8210000EE100AB8EE400A10EE5D
:10452000100A07F0D3F9184A1F4B07F0F7F907F004
:10453000C7FAC4F81D00BDF82300A4F821009DF8B7
:10454000250084F82300BDEC028B10BC5DF814FB41
:104550000849242205F07ABE3CAA0020AC4901207B
:10456000D6560120D4540120485601205C51012028
:1045700080510100FC510120FCA9F1D24D62503F55
:104580008DEDB5A0F7C6B03E3BDF4F8D2832012040
:1045900060AA00200054004028A800204C560120AA
:1045A0005F4C260520520120976EA23F80B50DF08A
:1045B000B9FE002104BD0000233E496E6974696C98
:1045C00061697A652049324300000000495745205F
:1045D00025642025640000004952452025642025DB
:1045E0006400000053485F48415F436865636B3671
:1045F0004178697353656E736F72000025732825C7
:104600006429203A20726567203D205B3078253090
:1046100032785D0057484F414D49206661696C20F2
:104620003A207265675B3078253032785D00000093
:10463000556E6B6E6F776E20366178697320736587
:104640006E736F722121212100000000000102031E
:104650000407060500010203040706050300010222
:104660000504070665364178697353656E736F728A
:104670002825642920446F742825642920417869FD
:10468000732825642900000041542D536574545348
:10469000312025642025640041542D536574545302
:1046A00032202564202564202564000041542D53C8
:1046B0006574542025643A25643A25642E256400E7
:1046C00010B5040010000A00010020000DF090FF5A
:1046D000200010BD50EA010200F00E80094200BF28
:1046E0000BD1B0FA80F18840C1F19D01C9050206E5
:1046F00072F1004241EB10207047B1FA81F2414063
:104700009040C2F1200261FA02F181EA000018BF74
:1047100040F0010002F19D01E8E750F8041B61B18F
:1047200050F8042BD30744BFA9F101039A180023C2
:1047300042F8043B091FFAD1EFE7704700220DF061
:104740008FBF8268521C8260426832B10268531C7B
:10475000036011704168491E4160704770B5DFF811
:10476000104BFEF767F9E0640DF094FFFEF750FF81
:104770002065002517E04FF0FF31C176DFF8841C7B
:104780004162DFF88C1C8162DFF8882CC262DFF89E
:10479000882C0263DFF8842C42638163206D30181B
:1047A000806B80476D1C3C2D80F29581216DC5EB9F
:1047B00005108600002070547018002242700122FB
:1047C000C276002282764FF0FF3242600022827071
:1047D0000262C2702A46921E392ACCD8DFE812F053
:1047E00047003B004F014F00570062007C003A0039
:1047F0003A003A003A003A003A0085008E003A004A
:104800003A003A003A0096003A009F003A005501FB
:10481000B000F80004010E013A00C800D000D90031
:10482000E100F0003A003A003A003A003A003A005B
:104830003A003A001A012F013A003B016A00740065
:1048400046016001BC003A00A8003A007601700100
:10485000680127018FE7DFF8C80BC1F8EC000120E1
:1048600081F8CE0001F17C003C21C16396E701F1A3
:104870007C00DFF8B02B42631420C8678EE701F19B
:10488000EC00DFF8A41B81671421416486E701F581
:10489000B670DFF8982B4263012282753C20C1F884
:1048A0006C017BE701F5B670DFF8841B01673C21E2
:1048B000C16373E701F63C30DFF8781BC163012167
:1048C00081773C21816069E701F63C30DFF8681BA5
:1048D0008167B421416461E7DFF8600BC1F8180219
:1048E00001F5B6701421816758E701F56270DFF8B1
:1048F000502B4263B420C1F888034FE701F5627082
:10490000DFF8401B01673C21C16347E701F59E606A
:10491000DFF8342B42633C20C1F8F0043EE7DFF8B7
:104920002C0BC1F89C0501F59E603C21816735E7A1
:1049300001F66840DFF8181B81673C2141642DE7D0
:1049400001F21460DFF80C1BC1630721C17701215C
:1049500081773C21816021E7DFF8FC0AC1F8680C0F
:10496000012081F84A0C01F6BC30B421816715E7BB
:1049700001F20470DFF8E41A8167142141640DE745
:1049800001F28470DFF8D82A42633C20C1F8840722
:1049900004E701F28470DFF8CC1A01671421C163C7
:1049A000FCE6FFF712F9216D90F81202012803D1FD
:1049B000DFF8B40AC1F830080A20C1F8FC07EDE6B8
:1049C000DFF8A80AC1F86C081420C1F83808E5E639
:1049D000DFF89C0AC1F88C06012081F86E0601F20E
:1049E00014603C214164D9E601F28C60DFF8841A3E
:1049F000C1630121817714218160CFE6DFF8780A55
:104A0000C1F80407012081F8E60601F28C603C2120
:104A10004164C3E601F65420DFF8602A42630322B2
:104A2000C275012282753C20C1F8540AB6E6DFF84F
:104A3000500AC1F80C0E1420C1F8D80DAEE6DFF80C
:104A4000440AC1F8C40A012081F8A60A01F65420DC
:104A50003C21C163A2E6DFF8300AC1F83C0B01201B
:104A600081F81E0B1420C1F8080B97E601F6BC3044
:104A7000DFF8182A42631420C1F8BC0B8EE601F15E
:104A8000EC00DFF80C1AC16388E6DFF8080AC1F809
:104A90001406012081F8F6053C20C1F8E0057DE60A
:104AA00001F6BC30DFF8F01901671421C16375E627
:104AB00001F65850DFF8E4198167142141646DE66E
:104AC00001F65850DFF8D819C16367E6DFF8D4095A
:104AD000C1F8580D62E6012070BD0CB42DE9F04319
:104AE00093B006460F46012534461A2C42D02C2C92
:104AF00040D0C4EB04104FEA8008DFF874970B2F06
:104B000018D1D9F8500040444178002912D090F9CA
:104B10001B20012A0EDB91420CDB304600F068F9C5
:104B20000546D9F850004044002141700FF684102A
:104B3000FFF7B4F8D9F8500018F8001000294FD149
:104B400008EB00014A78002A4AD1002208F8002028
:104B5000104648701AA983B06846582205F086FBB3
:104B60000EBC304600F06AF8022834D0032837D152
:104B7000032535E00B2F15D1C4EB04104FEA800854
:104B8000DFF8EC96D9F85000404490F91B20012A38
:104B900008DB4078904205DB0FF62010FFF77EF827
:104BA000022046E01A2C04D13846C0B208F0F5FACB
:104BB00005E02C2C03D13846C0B20DF00DFE1AA929
:104BC00083B06846582205F051FB0EBC304600F019
:104BD00035F8022801D102202BE0032800D103255B
:104BE0000A2F0DD1DFF88896D9F85000C4EB0411D4
:104BF0004FEA810818F80010491C08F8001017E067
:104C00000B2F15D1DFF86896032C07D1D9F8500087
:104C100090F8B500002801D107F057FCC4EB041050
:104C20004FEA8008D9F8500040444178491C41704F
:104C3000284613B0BDE8F0035DF80CFB0EB42DE977
:104C4000F04193B005460124C0EB00118F00DFF85E
:104C50002066D6F850801A2801D02C2808D117F8E1
:104C60000800002809D107EB08004078002804D18B
:104C700007EB080000218170016219A984B0684621
:104C8000582205F0F3FA0FBC47447F6AB847022860
:104C900001D1022011E0032801D103240CE0D6F851
:104CA0004C80D8E91E67204600212A460DF032FAD2
:104CB00030433943C8E91E01204613B0BDE8F00176
:104CC0005DF810FB2DE9F84304460D460126274602
:104CD000C7EB07104FEA8008DFF89495D9F8500029
:104CE0001A2F4ED02C2F4CD04044417802290BDB98
:104CF00090F91B20012A07DB1346994204DB42701E
:104D00000FF2C470FEF7CAFFD9F8500018F800106F
:104D1000002904D108EB00025278002A65D02A4607
:104D20000A2A09D1002903D0491E08F8001017E00B
:104D3000002108F8001013E00B2A11D108EB000144
:104D40004A78002A02D0521E4A7001E000224A70BE
:104D5000032F05D190F8B500002801D107F0C4FB5E
:104D6000D9F8500018F8001000293ED1404440788E
:104D700000283AD1204600F03BF8032835D103261D
:104D800033E018F80010002904D108EB0002527833
:104D9000002A2AD02A460A2A09D1002903D0491E0E
:104DA00008F800100EE0002108F800100AE00B2AB5
:104DB00008D140444178002902D0491E417001E0E9
:104DC000002141701A2F04D12846C0B208F0E5F93D
:104DD00005E02C2F03D12846C0B20DF0FDFC204683
:104DE00000F006F8032800D103263046BDE8F28320
:104DF0002DE9F04107460126B846C8EB08108500AA
:104E0000DFF86C44206D2818806A8047032800D1A1
:104E10000326B8F12C0F07D1206D295C00290AD197
:104E200028184078002806D1384640B200F07BF9B7
:104E3000032800D10326206D295C002914D12818ED
:104E40004178002910D1002181700162D4F84C8092
:104E5000D8E91E4501203A460DF05CF924EA00002D
:104E600025EA0101C8E91E013046BDE8F08138B5E8
:104E70000446C4EB04108000DFF8F453296D0022CF
:104E800042544018114641702046FFF7B1FFE86CCC
:104E9000D0E91E2321460FF23860FEF7FFFE012005
:104EA00032BD2DE9F041B6B004460E46B6B201203F
:104EB0008DF86400DFF8B8531AA8E96C6C2205F08D
:104EC000D5F917951AA984B068466C2205F0CEF979
:104ED0000FBC00F0CFF900270BE0032803D118978F
:104EE00003208DF86400286D4044002181707F1CF0
:104EF0007FB23C2F2ADAEA6CD2E91E013A4600F072
:104F000021FB00F0010011F0000101D10028EED0DA
:104F1000C7EB07104FEA8008286D4044416800291C
:104F2000E5D48278521C8270D2B2724389B28A422E
:104F3000DDDBC06A80470228CFD1189702208DF8A8
:104F40006400DDE91801C4E9000103E0DDE91801AE
:104F5000C4E9000136B0BDE8F0810021401F42F2F3
:104F60000C72904200D20121084670472DE9F043AF
:104F700083B00446002001900422E11C01A8FEF742
:104F8000C5FD6178BA4E376D3C2515FB0170406850
:104F9000019A904204D10FF24850FEF77FFE68E07C
:104FA0001046FFF7DAFF002809D16178019B15FB55
:104FB000017042680FF23450FEF770FE59E0DFF8DE
:104FC000E8743868D0F8008025E090F9089060789F
:104FD000316D15FB0010006A20FA09F0C00717D5E3
:104FE0004FF0FF3000900346012201994846FEF73A
:104FF00085F840B200280BD1617801980090306D9F
:1050000015FB010043684A460FF2F440FEF746FEE6
:105010004046D0F80080B842D7D13868D0F8008038
:105020001FE090F90890086A20FA09F0C00715D52A
:105030004FF0FF33012249684846FEF731F940B28C
:1050400000280BD1617801980090306D15FB0100AC
:1050500043684A460FF2C040FEF720FE4046D0F8B3
:1050600000806178326D15FB0121B842D9D10198D9
:105070004860BDE8F7832DE9F843814600242546C2
:105080007B4F21E0C5EB05108600386D06EB00086C
:10509000002088F80300FA6CD2E91E012A4600F0CD
:1050A00051FA00F0010011F0000101D100280AD0EE
:1050B0004846D8F830108847002804D0386D30189A
:1050C0000121C1700C466D1C3C2DDBDB2046BDE888
:1050D000F2836748C16CD1E91E23002B01D1002A5D
:1050E0000DD0002107E0C2EB0213026D02EB830238
:1050F0000023D370491C49B20A463C2AF3DB7047AF
:1051000000B502465A48C36CD3E91E0100F01AFAF2
:1051100000F0010011F0000101D1002801D00120B0
:1051200000BD084600BD2DE9F04781460124C9EBCA
:10513000091085004E4E306D2818006A002828D0CE
:10514000D94F3868D0F8008003E003244046D0F8F7
:105150000080B8421DD090F908A0306D2818016A6F
:10516000012202FA0AF2114021FA0AF149B2012998
:10517000ECD14FF0FF33012241685046FEF790F822
:105180000028E2D0524649460FF2A430FEF786FDD1
:10519000DCE72046BDE8F08710B598B004465A22F7
:1051A000002100A8FFF78CFA0020ADF858008DF818
:1051B00001000DF101000A21417000218170C170D0
:1051C0000846ADF85800600737D50520FFF798FF6F
:1051D000002808D004208DF8000005208DF801007B
:1051E00000A8FEF715FB0220FFF78AFF002808D071
:1051F00004208DF8000002208DF8010000A8FEF7C1
:1052000007FB2F20FFF77CFF002808D004208DF833
:1052100000002F208DF8010000A8FEF7F9FA032006
:10522000FFF76EFF002808D004208DF8000003204F
:105230008DF8010000A8FEF7EBFAE00611D5082072
:10524000FFF75EFF00280CD003208DF80000082037
:105250008DF8010000A8FEF7DBFA0FF2E020FEF760
:105260001DFD18B010BD02494C2204F0FFBF000024
:105270002C4E01200FB41B980099016001994160E8
:10528000029981600399C1600499016105994161A6
:10529000BDF85A100183BDF85C104183BDF85E1063
:1052A00081830C990162139941621499816204B05F
:1052B00070474178122904D1401C0179002007F081
:1052C000C6B9132904D1401C4179012007F0BFB9A8
:1052D000142904D1401C8179022007F0B8B915299E
:1052E00003D1401C007907F0D7B9302904D1401C04
:1052F00090F904000AF0F8BC012904D1401C90F98F
:1053000006000AF0DDBC172975D1411CCA78032AB2
:105310000AD01B2A14D01C2A33D01D2A1BD02C2AB9
:105320003FD0342A59D0704790F85610012902D145
:10533000401D07F0D3BD02295DD1401D07F0CEBD51
:10534000087A012802D1888809F0ACB8022852D125
:10535000C88809F0A5B84A7B012A02D1888809F0DB
:1053600033BB022A02D1C88809F022BB042A03D128
:10537000B0F8110009F02ABB032A3CD1C88909F012
:1053800031BBC879012802D108790EF083BB02280D
:1053900002D148790EF08DBB05282CD188790EF00A
:1053A00078BB8A7B012A02D1087A0DF0EEBF022A6F
:1053B00002D1008A0DF0D5BF032A02D1408A0DF038
:1053C000DABF042A03D1123040880DF0F7BF052A56
:1053D00011D1123080880DF0E2BF0A7B012A05D17D
:1053E000D0F8051000EE101A0EF088BB022A02D188
:1053F00088680EF08CBB70472C49086070472B48BA
:1054000000687047B13900082949087070470000EA
:10541000AD390008B9390008BD390008C1390008A4
:105420008FBE000811F90008D1F6000805590308DD
:10543000332F0308A74E030833510308C1F40008B3
:10544000856B0308776F0308E5730308D1720308BF
:10545000C1710308B5DC00086B3D01082DA00108EF
:10546000AB700308615503089B160308B99E010839
:1054700033E40008513A01086BE90008953201084D
:1054800049640308E76C0308EDFB000817380308BC
:1054900001A000083D6E03082DE80208CF6A03084A
:1054A000CD680308456703082C40002050560120B2
:1054B000D7560120414C204558000000414C204562
:1054C000582D415400000000524C20455800000067
:1054D0005445524D20256420256C6C750000000059
:1054E0004558204C4D435231202564004558204CEE
:1054F0004D4352322025642025642025640000009D
:105500004558204C4D4352332025642025642025E6
:1055100064202564000000004558204C4D4352345F
:1055200020256420256420256420256400000000D7
:10553000534D5241202564202564000048572053D4
:105540004D410000D2B2203A22BF21FA02F00021E0
:1055500070472032D141D04048409140D14048402E
:1055600070470268531C03601170704700B585B026
:1055700002460FF2140100A80EF0B4FC00A806F0D9
:10558000EFF805B000BD00004F45256400000000A5
:1055900034488168002904BF08B008E0EFF30982AD
:1055A000A2F12802036882E8F84F83685A6000F08D
:1055B00056F9816859B14A6892E8F84F036002F1E0
:1055C000280282F3098813F47F4F3FD070472648A2
:1055D00026490968401A80F308884FF08071C1613C
:1055E000234981617FF0060E704701BC2046DFF839
:1055F00084E000BDFEE7204800681C490968401AA5
:10560000203820F0070080F308884FF0000115488B
:10561000417081F3118862B600F014F8FEE7036868
:105620000CB44FF0000141704FF0000181F311887C
:105630001249134A0A604FF0800181F311880CBCB3
:10564000036070470D490E4A0A6070474FF0000131
:1056500081F31188704700BF4FF0800181F31188FA
:10566000704700BF28A80020E00F0020A4450208D2
:1056700059410108F55500080000000804ED00E05C
:105680000000001010B4802080F3118800BF00BF1C
:10569000DFF8C0078068DFF8BC1700220A7100211C
:1056A00081F3118800282ED0016800292BD042698F
:1056B00001684969914226D1016800E019000B6830
:1056C000002B02D05C699442F8D0802282F31188CA
:1056D00000BF00BFDFF87C271269824203D1DFF8E8
:1056E000742703681361026A036813601A62016217
:1056F0000B6803600268002A00D01862086091F805
:10570000450081F84400002080F3118810BC7047E8
:10571000802080F3118800BF00BFDFF83C070068DD
:10572000DFF83017096A401A01283ADADFF824074F
:10573000006A05E0DFF81C170862002181F3118878
:10574000DFF818170978C90726D5802181F3118859
:1057500000BF00BFDFF8041709788907EAD5DFF832
:10576000FC16097811F0FD01DFF8F0261170002118
:1057700081F31188DFF8DC16096A8842FAD0DFF875
:10578000D4160862DFF8D0060068401CDFF8C8169F
:105790000860DFF8C0164862802080F3118800BFDF
:1057A00000BF704710B5DFF8AC0600214171DFF88B
:1057B000A406006A10F18040DFF898164862DFF80E
:1057C0009406C069002805D0DFF88806DFF8841643
:1057D000C9698847002080F31188DFF87806C4681B
:1057E0000EE0E068DFF86C16496A401A002803D51D
:1057F000DFF86006E1684162002080F311882468C8
:10580000002C26D0802080F3118800BF00BFDFF875
:1058100044060069002806D06069DFF83816096977
:10582000496988421AD3207C4007E5D5E068DFF853
:105830002416096A401A0128D3DA200000F036FA4B
:10584000802080F3118800BF00BF207C0028C8D1D1
:1058500004E0802080F3118800BF00BF10BD38B580
:10586000DFF8F00500214170DFF8E8050121017043
:10587000DFF8E005C06B002818D0802080F3118885
:1058800000BF00BFDFF8CC05C06B8047002080F36D
:105890001188DFF8C0050021C163DFF8B8050021D9
:1058A0004163DFF8B005002180F838100EF034FBBA
:1058B0000078C0B2CD2802D07D20FFF757FEDFF878
:1058C00094058068002812D0DFF888058068806C15
:1058D00000280CD0DFF87C058068806C0168080027
:1058E000002804D0DFF86C05806840688847DFF83E
:1058F000640590F8310000280FD0DFF85805806863
:10590000DFF8501591F8301080F84410DFF84405A6
:105910000079002801D0FFF7B5FEDFF8380590F8D0
:10592000400000283DD0DFF82C0590F84000C0076B
:1059300018D5DFF82C050068DFF81815096A401A39
:1059400000280FD5DFF80C0590F8400010F0FE009D
:10595000DFF8001581F84000DFF8F80490F8400007
:1059600000281ED0802080F3118800BF00BF0EF0F9
:1059700036FC002181F31188DFF8D81489680029EA
:105980000CD0DFF8D0148968896B4118DFF8D42473
:105990001268891ADFF8BC2492689163DFF8C41496
:1059A0000860DFF8B004806800280ED0DFF8A40497
:1059B0008068007C002808D1DFF898048068406B7C
:1059C000401CDFF8901489684863DFF88804006998
:1059D000002839D006E0DFF87C042168016100204E
:1059E00080F31188802080F3118800BF00BFDFF8AA
:1059F00064040469002C2FD0257CEDB2002D2BD03F
:105A0000680716D5E068DFF84C14096A411A0129C5
:105A100006DA200000F04AF9207C002809D113E0C2
:105A2000DFF83014496A411A002902D5DFF824143E
:105A30004862EDB215F0FB001028CCD1A068806858
:105A40004068007C0028C6D1802080F3118800BF08
:105A500000BF01E0FFF7A6FEDFF8F8034079002859
:105A6000F8D1DFF8F8030078C00701D5FFF750FE42
:105A7000DFF8E00300214171DFF8D8030069002856
:105A800053D0DFF8D0030069007C002809D0DFF88C
:105A9000C403006980688068DFF8B81340688860D4
:105AA00005E0DFF8B003DFF8AC1309698160DFF8C7
:105AB000A403806890F85000642802D08020FFF78B
:105AC00055FDDFF890038068C06A0078CD2802D0C9
:105AD0007820FFF74BFDDFF87C038068806C00289E
:105AE0000CD0DFF870038068806C416808000028E3
:105AF00004D0DFF86003806840688847DFF854030B
:105B0000806890F84400DFF84C1381F83000DFF82B
:105B1000441381F83100DFF83C038068006B401CBF
:105B2000DFF830138968086314E0DFF828030021E8
:105B300080F83110DFF81C03002180F83010DFF806
:105B4000140300218160DFF80C03002101700020A4
:105B500080F31188DFF8FC0232BD80B50EF084FBC3
:105B6000DFF804130978002806D0022810D009D3E2
:105B7000042815D010D314E0002902D0A320FFF789
:105B8000F5FC11E0002902D1A420FFF7EFFC0BE0A7
:105B9000A620FFF7EBFC07E0A720FFF7E7FC03E0F8
:105BA00002E0A820FFF7E2FC01BD10B50EF05CFB9F
:105BB0000400DFF8B4020078002802D0A020FFF72C
:105BC000D5FC002C05D0022C08D003D3032C09D01F
:105BD0000CE00EE0A420FFF7C9FC0AE0A620FFF7C6
:105BE000C5FC06E0A720FFF7C1FC02E0A820FFF7F4
:105BF000BDFC10BD80B50EF037FB002805D0022893
:105C000008D006D3032809D00CE0A320FFF7AEFC90
:105C10000BE00AE0A620FFF7A9FC06E0A720FFF7AB
:105C2000A5FC02E0A820FFF7A1FC01BD80B5DFF8CC
:105C300024020078002802D19720FFF797FCDFF8B4
:105C400014020078401EDFF80C120870C0B2002861
:105C50002BD1DFF800024068002826D0802080F396
:105C6000118800BF00BFDFF8EC01406800280BD0AE
:105C7000DFF8E00101210170DFF8D801FFF7CFFC68
:105C8000DFF8D00100210170DFF8C8014078F02171
:105C9000084202D09920FFF769FCDFF8B80140788C
:105CA000002802D1002080F3118801BD10B5816861
:105CB00000290CD0DFF89C11096AC16081680A686C
:105CC0004968002A00D051600A6000218160017C8F
:105CD00011F003010174C9B2002943D1DFF8741136
:105CE000096900292AD1DFF86C110861DFF8640125
:105CF000007800280CD1DFF85C0101210170DFF889
:105D00005401FFF78CFCDFF84C010021017003E027
:105D1000DFF8400101214171DFF838014078F021BE
:105D2000084202D09920FFF721FCDFF828014078D3
:105D3000002802D1002080F3118813E042694B69EA
:105D40009342D0D38142D1D04B699A420AD1030009
:105D5000FFE71B68002BDFD05C69A242DCD18B42DD
:105D6000F7D1C0E710BD10B504006069002802D16A
:105D7000CB20FFF7FBFB626936480078401C3549B1
:105D800008703A4800E008000168002902D04B6919
:105D90009A42F8D3216020620460002909D00C6285
:105DA0004869904202D194F8450000E0002084F850
:105DB0004400207C002816D1802080F3118800BF89
:105DC00000BF2000FFF772FF22484078F021084210
:105DD00002D09920FFF7CAFB1E484078002802D164
:105DE000002080F31188FFF721FF10BD10B519487E
:105DF000047818480078401C164908701548FFF7C9
:105E00000EFC1448047013484078F021084202D078
:105E10009920FFF7ABFB0F484078002802D1002003
:105E200080F3118810BD10B50EF024FA0948012145
:105E300001700EF071F804006846C046021B203A5B
:105E4000012A03DBCD212000FEF73AFC084801219E
:105E5000017010BD28A80020AC560120FA56012080
:105E6000C4560120B0560120F956012034A8002064
:105E7000FC560120DFF80C09704730B583B00020D4
:105E8000ADF806008DF804000120009001AB00225F
:105E900018210220FDF7E3FF04469DF8040048287E
:105EA0001FD131208DF806000DF106050120687024
:105EB00002230DF1060218211846FDF774FF002891
:105EC0000DD031208DF806000020687002230DF1FE
:105ED000060218211846FDF766FF002802D10020AF
:105EE0003EBD0024DFF8A0581822002105F11C0057
:105EF000FEF7E6FBDFF89408C0F8D45320463EBD19
:105F000070B582B00020ADF800000EF0DCF9044658
:105F1000DFF87C088168497AC268527A51180069B2
:105F2000407A0818012801DB012076BDDFF86458AB
:105F3000687B01281CD032208DF8000000AE0120C3
:105F40007070022300AA18211846FDF72CFF0028C4
:105F50000CD031208DF8000001207070022300AABF
:105F600018211846FDF71FFF002803D1002076BD39
:105F70000120287305F1100061698847012076BD72
:105F800038B50020ADF800000EF09DF90446DFF8AA
:105F900000088168497AC268527A51180069407ACB
:105FA0000818022801DB012032BDDFF8E857287B02
:105FB000012812D031208DF8000000208DF801005A
:105FC000022300AA18211846FDF7EDFE002801D192
:105FD000002032BD0020687301E00020287305F125
:105FE000100021698847012032BD80B50020ADF83E
:105FF000000031208DF8000000208DF80100022300
:1060000000AA18211846FDF7CEFE002801D1002075
:1060100002BD012002BD7CB504460020ADF806009B
:106020008DF804000120009001AB0022182102200D
:10603000FDF715FF05469DF80400482829D13120B9
:106040008DF806000DF106061F20707002230DF179
:10605000060218211846FDF7A6FE002817D00320D7
:1060600000902346602218210220FDF7F8FE002848
:106070000DD031208DF806000020707002230DF144
:10608000060218211846FDF78EFE002802D10020D6
:1060900076BD0025284676BD0021DFF8EC2602E01B
:1060A0000B5C8B54491C1B29FADBDFF8E006C0F8B7
:1060B000D423012070472DE9F04788B004460D46EF
:1060C00016461F464FF000084046ADF8040002A8EF
:1060D00041460A460B460EC04FF0050906C0012096
:1060E000009002AB102218210220FDF7B8FE9DF8A7
:1060F0000810C9070ED501280CD1082000900DF119
:106100000903112218210220FDF7A9FE002807D15A
:1061100040468EE04846A0F1010980B20028DED159
:10612000DFF870969DF8080089F800009DF81000CF
:1061300089F801009DF80F0089F802000AE002A822
:1061400000EB48008178407810EB012024F818001B
:1061500008F10108B8F1030FF1DBB4F900000028E1
:1061600007D1B4F90200002803D1B4F904000028D3
:1061700024D0DFF81C06D0F80C8008F10C0A9AF83D
:1061800015202146DAF80C00D8F80C30C018FDF7BD
:10619000BDFC4046FCF78CFD9AF81520DAF80C009F
:1061A000D8F80C1041182046FDF7B0FC9AF81520DD
:1061B000214609F10300FDF7A9FC03E00FF200609E
:1061C000FDF76CFDDFF8C485109B05AA214640460B
:1061D0000EF0A2FA98F9F4023860B8F8EE002880C0
:1061E00008F2EE00418869808188A9808189218038
:1061F000C1896180008AA08020882988401A308067
:1062000060886988401A7080A088A988401AB08088
:1062100031208DF8040001208DF80500022301AA29
:1062200018211846FDF7BFFD002801D1002000E02D
:10623000012008B0BDE8F08770B586B004460020A4
:10624000ADF8040002A800210A460B460EC0052541
:10625000DFF83805B0F9F612091881F8F522114671
:10626000A0F8EE1000F2EE00418081800EF02BF8D5
:106270000146DFF8206506F11000496988470120D2
:10628000009002AB102218210220FDF7E8FD9DF8D6
:106290000810C9070ED501280CD1082000900DF177
:1062A0000903112218210220FDF7D9FD002806D18B
:1062B000002028E02846451E80B20028DFD19DF846
:1062C0000800307002A8017A7170417821708178DD
:1062D0006170C178A1700179E170407920719DF8F9
:1062E0000E00607131208DF8040001208DF805004A
:1062F000022301AA18211846FDF755FD002801D1F7
:10630000002000E0012006B070BD2DE9F04182B010
:1063100004460025FCF78EFB8046FFF7ABFD0646E2
:10632000DFF86C040769D8E91C0100F0040011F0E3
:1063300000010ED100280CD1009406F1140306F1DF
:106340000C02B11D3046FFF7B6FE002801D12846E9
:1063500014E0B87A01280CD10FE006EB4500C188A3
:1063600004F8151004EB4501B0F90600001248705E
:106370006D1C032DF1DB7069A0710120BDE8F68171
:10638000F8B504460025FCF755FB0746FFF772FDFC
:106390000646D7E91C0100F0080011F0000101D108
:1063A000002805D02046FFF747FF002827D10AE044
:1063B000009406F1140306F10C02B11D3046FFF7FC
:1063C0007AFE002814D12846F2BD36F8150004F8EC
:1063D000150004EB450036F915100912417006EB63
:1063E00045018A898271B1F90C100912C1716D1CC5
:1063F000032DEADB18223146E248FDF787FB012036
:10640000F2BD7CB504460020ADF806008DF804000E
:10641000FDF7DBFB05460120009001AB00221821AF
:106420000220FDF71CFD9DF80410482932D13120CF
:106430008DF806000DF106061F20707002230DF185
:10644000060218211846FDF7AEFC00281BD03120AB
:106450008DF806000020707002230DF1060218214D
:106460001846FDF7A0FC00280DD001212846FDF7B5
:106470000FFE0120009001AB312218210220FDF710
:10648000EEFC002801D1002076BD9DF804002070AC
:10649000012076BDFF21217076BD2DE9F04387B044
:1064A000044604A800210A460B460EC00846ADF873
:1064B0000C000525FDF789FB064632208DF80C00FF
:1064C00003AF01207870022303AA18211846FDF7B4
:1064D0006AFC002800F0F58001213046FDF7D8FD68
:1064E0000220009004AB00221821FDF7B8FC804682
:1064F0009DF81000482840F026819DF8100020707B
:106500000DF1100999F80100607031208DF80C0030
:106510001F207870022303AA18211846FDF743FCB8
:10652000002800F012810320009004AB60221821A3
:106530000220FDF794FC002800F007819DF8100070
:10654000A07099F80100E07099F8020020713120E4
:106550008DF80C0000207870022303AA1821184639
:10656000FDF721FC002800F0F08001213046FDF706
:106570008FFD0120009004AB312218210220FDF78D
:106580006EFC002800F0E1809DF81000607531205D
:106590008DF80C0001207870022303AA18211846F8
:1065A000FDF701FC002800F0D0801E213046FDF7E9
:1065B0006FFD0120009004AB102218210220FDF78E
:1065C0004EFC80469DF81000C0070ED5B8F1010FB3
:1065D0000BD1082000900DF1110311221821022087
:1065E000FDF73DFC002805D16BE02846451E80B232
:1065F0000028DED199F80600029099F80500019074
:1066000099F80400009099F8033099F8022099F85D
:1066100001100FF2C010FDF741FB99F8020099F844
:10662000011011EB002099F8041099F8032012EBE7
:10663000012199F8062099F8053013EB0222034650
:106640001BB21B126371A071084600B20012E07108
:106650002172104600B200126072A2729DF8100002
:10666000E07299F80800207331208DF80C0010209A
:106670007870022303AA18211846FDF794FB00281E
:1066800063D01E213046FDF703FD05250120009053
:1066900004AB102218210220FDF7E1FB80469DF893
:1066A0001000C0070FD5B8F1010F0CD108200090E1
:1066B0000DF11103112218210220FDF7D0FB002853
:1066C00006D1002042E02846451E80B20028DDD1D8
:1066D00099F80600029099F80500019099F80400D5
:1066E000009099F8033099F8022099F801100FF200
:1066F0000010FDF7D3FA99F8020099F8011011EB98
:10670000002099F8041099F8032012EB012199F860
:10671000062099F8053013EB022203461BB21B1228
:106720006373A073084600B20012E0732174104630
:1067300000B200126074A2749DF81000E07499F821
:106740000800207501E04FF00008404607B0BDE8A2
:10675000F08318B404460B4611460020032C04D0E5
:10676000042C05D0072C06D008E0184614BC52E4CF
:10677000184612BC45E6184612BC8DE412BC7047A0
:1067800005487047C4A80020A8A80020681301206D
:10679000AC490120A45201207853012010B50FF21A
:1067A0006C04214602200BF0D5F90FF28801042079
:1067B0000BF0D0F921460320BDE810400BF0CAB918
:1067C00047656F20416C6C2064617461206973209F
:1067D00030000000474D53312D25642C2025642CBA
:1067E0002025642C2025642C2025642C2025640081
:1067F000474D53322D25642C2025642C2025642CF4
:106800002025642C2025642C202564007B5E000854
:10681000015F0008815F0008EB5F000800000000D6
:1068200081630008000000009B64000853670008B3
:10683000000000007B5E0008015F0008815F000827
:10684000EB5F0008000000000B6300080000000080
:106850009B6400085367000800000000BFF34F8FDF
:10686000DFF8600A016801F4E061DFF85C2A114397
:106870000160BFF34F8FFEE77CB506460C46154618
:106880000020ADF806008DF804000120009001AB57
:10689000324672210720FDF7E2FA002801D10020DC
:1068A00076BD8DF806609DF80400A04328438DF85E
:1068B00004009DF804008DF8070002230DF1060284
:1068C00072210720FDF76FFA002801D1002076BD64
:1068D000012076BD38B50020ADF800000246402109
:1068E000AB20FFF7C9FFC0208DF8000000AC0F20DF
:1068F0006070022300AA72210920FDF754FA0028D3
:1069000001D1002032BDC1208DF800000020607050
:10691000022300AA72210920FDF745FA002801D1BF
:10692000002032BDC2208DF800000F2060700223CD
:1069300000AA72210920FDF736FA002801D10020B3
:1069400032BDC3208DF8000000206070022300AA31
:1069500072210920FDF727FA002801D1002032BD5D
:10696000C4208DF800000F206070022300AA72215D
:106970000920FDF718FA002801D1002032BDC520FA
:106980008DF8000000206070022300AA7221092007
:10699000FDF709FA002801D1002032BDC6208DF88C
:1069A00000000F206070022300AA72210920FDF769
:1069B000FAF9002801D1002032BDC7208DF800006F
:1069C00000206070022300AA72210920FDF7EBF974
:1069D000002801D1002032BD81208DF80000F52073
:1069E0006070022300AA72210920FDF7DCF900285B
:1069F00001D1002032BDDFF8D4586078687382205E
:106A00008DF8000006206070022300AA7221092080
:106A1000FDF7C9F9002801D1002032BD287C0028EB
:106A20001DD08E208DF8000045206070022300AA42
:106A300072210920FDF7B7F9002801D1002032BDED
:106A40008F208DF8000058206070022300AA722168
:106A50000920FDF7A8F900281FD1002032BD8E20A3
:106A60008DF8000082206070022300AA72210920A4
:106A7000FDF799F9002801D1002032BD8F208DF853
:106A800000008C206070022300AA72210920FDF70B
:106A90008AF9002801D1002032BD80208DF8000045
:106AA00007206070022300AA72210920FDF77BF9FC
:106AB000002801D1002032BDDD208DF8000020200B
:106AC0006070022300AA72210920FDF76CF90028EA
:106AD00001D1002032BD012032BD10B582B00020AE
:106AE000ADF800000446FDF770F80A21FDF7D0FA72
:106AF00000E0641C032C12D2DFF8D407215C8DF86F
:106B00000010201800798DF80100022300AA7221DC
:106B10000720FDF748F90028EBD1002016BD012021
:106B200016BD10B5DFF8A447A37D627D617C0FF22E
:106B30002800FDF7B3F8607C617D0843A17D084320
:106B40004FF4004103D00020FDF7E8FA02E00020F6
:106B5000FDF7E6FA012010BD233E50777220502544
:106B600064204D25642049256400000070B582B082
:106B700004460E46FBF75EFF0020ADF80000DFF88C
:106B80004C57688C0146002E02D02043688401E0F7
:106B9000A0436884688C00281DD001283AD00228C0
:106BA0006ED003286CD0042800F02E81052800F058
:106BB0007B81062800F05681072800F0D981102833
:106BC00067D0112800F0AE80202800F08D802128A9
:106BD00000F0E8801CE0DD208DF8000000AC002013
:106BE0006070022300AA72210920FDF7DCF800285A
:106BF00000F0F28180208DF80000002060700223F8
:106C000000AA72210920FDF7CEF8002800F0E481E7
:106C1000012076BD880701D5012028760022402179
:106C2000AB20FFF729FE81208DF8000000ACF52095
:106C30006070022300AA72210920FDF7B4F8002831
:106C400000F0CA8160786873DD208DF800000020B4
:106C50006070022300AA72210920FDF7A4F8002821
:106C600000F0BA8180208DF80000032060700223BC
:106C700000AA72210920FDF796F80028C8D1ABE1DF
:106C8000012901D101202876FFF724FE0028BFD179
:106C9000A2E18F208DF8000000AC08206070022374
:106CA00000AA72210720FDF77EF8002800F09481E9
:106CB00080208DF8000081206070022300AA7221DC
:106CC0000720FDF770F8002800F08681DD208DF8A0
:106CD000000008206070022300AA72210720FDF73F
:106CE00062F8002894D177E180208DF8000000AC94
:106CF00081206070022300AA72210720FDF753F85B
:106D0000002800F06981DD208DF800000820607007
:106D1000022300AA72210720FDF745F800287FF41E
:106D200077AF59E1880701D50120287681208DF8B9
:106D3000000000ACF5206070022300AA7221092037
:106D4000FDF731F8002800F04781607868738F20E4
:106D50008DF8000008206070022300AA722107202D
:106D6000FDF721F8002800F0378180208DF8000021
:106D700083206070022300AA72210720FDF713F818
:106D8000002800F02981DD208DF8000008206070C7
:106D9000022300AA72210720FDF705F800287FF4DE
:106DA00037AF19E1880701D50120287681208DF8B9
:106DB000000000ACF5206070022300AA72210920B7
:106DC000FCF7F1FF002800F00781607868738020ED
:106DD0008DF8000083206070022300AA7221072032
:106DE000FCF7E1FF002800F0F780DD208DF80000BF
:106DF00008206070022300AA72210720FCF7D3FF4D
:106E000000287FF405AFE7E081208DF8000000AC9A
:106E1000EE206070022300AA72210920FCF7C3FF54
:106E2000002800F0D98060786873DD208DF80000BC
:106E300000206070022300AA72210920FCF7B3FF32
:106E4000002800F0C98080208DF8000003206070C9
:106E5000022300AA72210920FCF7A5FF00287FF475
:106E6000D7AEB9E00846800715D581208DF800001F
:106E700000ACEE206070022300AA72210920FCF70A
:106E800092FF002800F0A880607868730FF24C1021
:106E9000FCF704FFBCE648077FF5BAAEFFF71AFD22
:106EA00000287FF4B5AE97E00846C0072CD58120B6
:106EB0008DF8000000ACEE206070022300AA722161
:106EC0000920FCF770FF002800F086806078687366
:106ED000DD208DF8000000206070022300AA7221DE
:106EE0000920FCF760FF002876D080208DF8000094
:106EF00003206070022300AA72210920FCF753FFCF
:106F000000287FF485AE67E048077FF581AE002258
:106F10004021AB20FFF7B0FC81208DF8000000ACD1
:106F2000F5206070022300AA72210920FCF73BFFC4
:106F3000002851D060786873DD208DF800000020B3
:106F40006070022300AA72210920FCF72CFF0028A0
:106F500042D080208DF8000003206070022300AA38
:106F600072210920FCF71FFF00287FF451AE33E0A7
:106F700011F0050F05D0FFF7ADFC00287FF448AEF7
:106F80002AE081208DF8000000ACEE206070022322
:106F900000AA72210920FCF706FF00281CD06078A7
:106FA0006873DD208DF8000000206070022300AAC5
:106FB00072210920FCF7F7FE00280DD080208DF803
:106FC000000003206070022300AA72210920FCF750
:106FD000EAFE00287FF41CAE002076BD233E21216E
:106FE00050522D3E4952000080B50FF24000FCF790
:106FF00055FE0020ADF8000080208DF80000032031
:107000008DF80100022300AA72210620FCF7CBFEB6
:10701000002801D1002002BD01210020FFF7A6FDBC
:10702000002801D1002002BD012002BD233E484CB2
:10703000530000001CB5044600208DF80400ADF894
:1070400006000120009001ABDE2272210720FCF730
:1070500006FF002801D1002016BDDE208DF80600B5
:107060009DF8040020438DF8070002230DF106026D
:1070700072210720FCF797FE002801D1002016BDE1
:10708000012016BD30B583B00FF29C00FCF706FE60
:107090000020ADF804000446FFF71FFDDFF8A41D33
:1070A00008700028DFF8A05D06D10FF28400FCF71D
:1070B000F5FD20463EBD641C0D2C11D260190079EF
:1070C0008DF804006019007D8DF80500022301AAE7
:1070D00072210720FCF767FE0028ECD100203EBD9E
:1070E0007A4C0120009004F11A03912272210720AA
:1070F000FCF7B5FE002801D100203EBD0120009024
:107100002B46922272210720FCF7A9FE002801D10C
:1071100000203EBD2A78A17E0FF22000FCF7BEFDC4
:1071200002F07EF801203EBD233E50525000000088
:10713000233E50505F4641494C000000233E5052D0
:107140002052455620307825782044455620307806
:107150002578000038B55D4DA97E0FF2D400FCF70C
:107160009DFD0020ADF8000028848C208DF80000E3
:1071700000AC2020607000202873022300AA722136
:107180000720FCF710FE002801D1002032BD0120AD
:107190006874FFF7C6FC01210220FFF7E7FC002816
:1071A00001D1002032BD88208DF80000F0206070F1
:1071B000022300AA72210720FCF7F5FD002801D167
:1071C000002032BD89208DF800003F20607002232E
:1071D00000AA72210720FCF7E6FD002801D100205B
:1071E00032BD8A208DF8000000206070022300AAC2
:1071F00072210720FCF7D7FD002801D1002032BD05
:107200008B208DF8000000206070022300AA7221FC
:107210000720FCF7C8FD002801D1002032BD202046
:10722000FFF708FF002801D1002032BD012032BD48
:10723000233E50524F2030782578000000B583B0AF
:107240000FF29000FCF72AFD00208DF80400DFF813
:10725000FC0B816A497A01291ED1C069407A012854
:107260001AD101210020FFF781FC002801D1002064
:107270000EBD0120009001AB802272210720FCF797
:10728000EEFD002801D100200EBD9DF804100FF284
:107290004C00FCF703FD0BE00C4800214174022078
:1072A000FFF764FC002801D100200EBDFFF739FC78
:1072B0002020FFF7BFFE002801D100200EBD0120D5
:1072C0000EBD00000CED00E00400FA0538A7002018
:1072D00044AA0020233E505243000000233E2626AD
:1072E000656E61626C6520307825780001207047FA
:1072F0001CB50446FBF79EFB0020ADF806008DF898
:1073000004000120009001AB9E2272210720FCF7AF
:10731000A6FD00280ED09DF80400000612D502201C
:1073200000900DF106039C2272210720FCF797FDC7
:10733000002801D1002016BD9DF8060020709DF8A0
:1073400007006070012016BD2DE9F04784B00446A7
:10735000FBF770FB0546FCF738FC06460020019061
:10736000ADF80800012000900DF107039E22722164
:107370000720FCF774FD002801D10020F8E201206D
:1073800000900DF10603932272210720FCF767FDA0
:10739000002801D10020EBE20220009002AB9422F1
:1073A00072210720FCF75BFD002801D10020DFE2FD
:1073B0000DF1080999F801009DF8081041EA002034
:1073C000DFF8787D797BC1F58071BA7BDFF8703D9D
:1073D000D25C12FB01F140F242325143FA7E012AA3
:1073E00003D140F2E362504302E040F621325043C1
:1073F0006422504390FBF1F0F97C002901D1B8647C
:1074000008E0B86CB97F4A1CBA77062902DB002174
:10741000F974B977397C00290BD141F6593188428A
:1074200028DB01213974F8640020F877FFF7DCFDD0
:1074300094E2F96C411A44F62162914212DA40F664
:10744000B831884214DA9DF80620920610D5FA7FEA
:10745000531CFB77C92A01DA88420BDA884201DA29
:1074600000213974F8640020F877FFF7BDFD75E25C
:107470000020F8779DF80600800640F17882012010
:1074800038770220009002AB9C2272210720FCF783
:10749000E6FC002801D100206AE299F801009DF87D
:1074A000081041EA00280FFA88F841460FF2C84058
:1074B000FCF7F4FB9DF80800607099F80100A070DB
:1074C000A7F82080787C002872D0387B00286FD104
:1074D000002030768C208DF804000DF10409202066
:1074E00089F801003873022301AA72210720FCF7F2
:1074F0005AFC002801D100203AE205F2920AB5F8C0
:107500009200002803D0BAF8020000280BD10FF235
:107510003470FCF7C3FB4FF4FA60A5F8920040F218
:10752000DC50AAF8020088208DF80400002089F8B9
:107530000100022301AA72210720FCF734FC002875
:1075400001D1002014E289208DF80400002089F880
:107550000100022301AA72210720FCF724FC002865
:1075600001D1002004E28A208DF80400B5F89200D1
:1075700089F80100022301AA72210720FCF713FCFD
:10758000002801D10020F3E18B208DF80400B5F82C
:107590009200000A89F80100022301AA7221072043
:1075A000FCF701FC002801D10020E1E10120387541
:1075B00005F2920ABAF80220B5F892100FF2C43020
:1075C000FCF76CFB787C002800F0C881B5F89200CD
:1075D000804551DB307E00284ED10120F8732070A9
:1075E0002078307688208DF804000DF10409BAF86F
:1075F000020089F80100022301AA72210720FCF78A
:10760000D2FB002801D10020B2E189208DF80400CE
:10761000BAF80200000A89F80100022301AA7221C7
:107620000720FCF7C0FB002801D10020A0E18A2040
:107630008DF80400FF2489F80140022301AA722179
:107640000720FCF7B0FB002801D1002090E18B203F
:107650008DF8040089F80140022301AA7221072055
:10766000FCF7A1FB002801D1002081E141460FF287
:107670002430FCF713FB71E1BAF80200404553DBFC
:10768000307E012850D10120F8730020207020782E
:10769000307688208DF804000DF10409002089F867
:1076A0000100022301AA72210720FCF77CFB0028BD
:1076B00001D100205CE189208DF80400002089F8C8
:1076C0000100022301AA72210720FCF76CFB0028AD
:1076D00001D100204CE18A208DF80400B5F8920019
:1076E00089F80100022301AA72210720FCF75BFB45
:1076F000002801D100203BE18B208DF80400B5F873
:107700009200000A89F80100022301AA72210720D1
:10771000FCF749FB002801D1002029E141460FF286
:107720007C20FCF7BBFA19E1B5F89200404557DB25
:10773000307E002854D1387D012851D10120F873C2
:1077400000202070207830760020387588208DF851
:1077500004000DF10409002089F80100022301AAA8
:1077600072210720FCF71FFB002801D10020FFE059
:1077700089208DF80400002089F80100022301AA65
:1077800072210720FCF70FFB002801D10020EFE059
:107790008A208DF80400B5F8920089F801000223D0
:1077A00001AA72210720FCF7FEFA002801D100206F
:1077B000DEE08B208DF80400B5F89200000A89F80D
:1077C0000100022301AA72210720FCF7ECFA00282D
:1077D00001D10020CCE00FF2CC10FCF75FFABDE045
:1077E000B5F89200804555DB307E012852D1387DB6
:1077F00001284FD10120F8732070207830760020C6
:10780000387588208DF804000DF10409BAF80200DB
:1078100089F80100022301AA72210720FCF7C3FAAC
:10782000002801D10020A3E089208DF80400BAF8D7
:107830000200000A89F80100022301AA7221072030
:10784000FCF7B1FA002801D1002091E08A208DF8E0
:107850000400FF2489F80140022301AA72210720B5
:10786000FCF7A1FA002801D1002081E08B208DF8DF
:10787000040089F80140022301AA72210720FCF7C5
:1078800092FA002801D1002072E00FF22010FCF7DC
:1078900005FA63E0B5F8920080455BDABAF80200B9
:1078A000404557DA307E012854D1387D012851D126
:1078B0000120F87300202070207830760020387581
:1078C00088208DF804000DF10409002089F80100DA
:1078D000022301AA72210720FCF765FA002801D1D2
:1078E000002045E089208DF80400002089F801007F
:1078F000022301AA72210720FCF755FA002801D1C2
:10790000002035E08A208DF80400B5F8920089F84F
:107910000100022301AA72210720FCF744FA002883
:1079200001D1002024E08B208DF80400B5F89200EE
:10793000000A89F80100022301AA72210720FCF73E
:1079400032FA002801D1002012E00FF26800FCF7A3
:10795000A5F903E00FF26400FCF7A0F92020FFF77F
:1079600069FB002801D1002002E0012000E0002096
:1079700004B0BDE8F0870000233E507261772025F7
:1079800064000000233E55703D25642C4C6F3D255E
:1079900064000000233E503120256400233E503215
:1079A00020256400233E526554483100233E526531
:1079B00054483200233E526554483300233E456C00
:1079C000736500002DE9FC4104460D46002001903E
:1079D0000746DFF8686730770120009001AB9322FB
:1079E00072210720FCF73BFA002801D1384695E0C8
:1079F000012000900DF105039E2272210720FCF763
:107A00002EFA002801D1384688E09DF804000007CE
:107A100009D5707D002806D00120307700F00AFDDE
:107A20003846F0757AE0FBF705F88046207807289D
:107A300025D16078FF2822D12946601CFFF758FC29
:107A4000A078617841EA002212B2B8F8920082422E
:107A500007DB0120207021780FF2C400FCF71EF92B
:107A60000AE0B8F89400904206DB3846207021788E
:107A70000FF2AC00FCF712F901204FE07F1C002050
:107A8000F07529462046FFF75FFC00280DD0707C7A
:107A900000280AD0F07B002807D00FF29800FCF7EE
:107AA000FDF80020F0730120F075052F03DA02F0D5
:107AB00007F90028E2D09DF80400C021084201D057
:107AC00001203077307F002809D1706C411C71642F
:107AD0009DF804200FF26400FCF7E0F801E00020BC
:107AE0007064706C1E2807DB0FF26800FCF7D6F894
:107AF000FEF7B4FE00207064DE208DF80600FA2048
:107B00008DF8070002230DF1060272210720FCF711
:107B10004AF9002801D1002000E0F07DBDE8F6819F
:107B2000233E536C65657020414443202564202525
:107B300064000000233E505550000000233E696E53
:107B40007620696E742025642073746174757320C7
:107B500025780000233E5265736574525100000081
:107B600070B582B005460020ADF80000FAF762FF5C
:107B70000446DFF8C805012101752878697841EAD3
:107B80000020A4F8920004F29206A878E97841EA6D
:107B900000207080B4F89200002802D0708800287D
:107BA00009D10FF2A000FCF779F84FF4FA60A4F8BD
:107BB00092000020708088208DF8000000ADF02039
:107BC0006870022300AA72210720FCF7ECF8002855
:107BD00001D1002076BD89208DF800003F2068701B
:107BE000022300AA72210720FCF7DDF8002801D14A
:107BF000002076BD8A208DF80000002068700223E6
:107C000000AA72210720FCF7CEF8002801D100203D
:107C100076BD8B208DF8000000206870022300AA3A
:107C200072210720FCF7BFF8002801D1002076BDA3
:107C30007288B4F892100FF63450FCF72FF8012038
:107C400076BD0000233E5054483D300010B584B04E
:107C5000044601A800210A4606C00820009001AB96
:107C6000C02272210920FCF7FAF8002801D1002077
:107C700019E09DF80400207001A8417861708178B6
:107C8000A170C178E17001792171417961718179C7
:107C9000A171C179E17142789DF804100FF6DC40C2
:107CA000FBF7FCFF012004B010BD80B50FF21401FA
:107CB000072009F04FFF0FF234010A20BDE804400D
:107CC00009F048BF85700008557100083D72000832
:107CD000ED72000800000000C5790008617B000813
:107CE0000000000000000000000000008570000897
:107CF000557100083D720008ED7200080000000098
:107D0000F1720008617B0008000000000000000024
:107D100000000000002070470020704700207047DE
:107D200000207047002070470020704700207047F7
:107D30000FF20801062009F00DBF0000157D0008B4
:107D4000197D00081D7D0008217D0008000000004D
:107D5000257D0008000000002D7D0008297D000819
:107D60000000000038B50FF62C40FBF797FF354CAC
:107D70002078002817D00020ADF80000054600E06C
:107D80006D1C052D11D2281900798DF800002819D5
:107D9000007B8DF80100022300AA72210920FCF764
:107DA00002F80028ECD1002032BD012032BD10B510
:107DB00082B0E24CA17E0FF6E430FBF76FFF0020AB
:107DC000ADF8000090208DF8000003208DF8010030
:107DD000022300AA72210920FBF7E5FF002801D148
:107DE000002016BD0320A07301206076A07403203C
:107DF000206301210846FEF7B9FE002801D10020CA
:107E000016BD1020FFF716F9002801D1002016BD7D
:107E1000012016BD80B50FF69030FBF73FFFC74835
:107E2000002181740120FEF7A1FE002801D100206D
:107E300002BD1020FFF7FEF8002801D1002002BD8E
:107E4000012002BD98A9002040A90020AC490120D2
:107E5000012070472DE9F04F8DB006460AA8002199
:107E60000A4606C088460846CDE90801DFF8D00A70
:107E7000D0F824A008468AF872000120009006ABD2
:107E8000AB2272210720FBF7EAFF002864D09DF89F
:107E90001800400660D4A94F787F00284BD038786E
:107EA000307078787070B878B070F878F070387991
:107EB000307178797071B879B071F879F071387A79
:107EC0003072787A70727078317841EA0029F078EF
:107ED000B17841EA00247079317941EA0025F079DE
:107EE000B17941EA002808A8009043462A46214675
:107EF000484600F090F9DDE90801C7E90A01494662
:107F000079632246BA632B46FB63386B0128C0F2C3
:107F10001181DDE90845CDE90445B87B0290787B05
:107F20000190CDF800800FF68820FBF7B7FE386B84
:107F3000401E3863FEE0787E012803D0387E00289A
:107F400040F09180082000900AAB94227221092011
:107F5000FBF785FF002801D14046ECE09DF82800A2
:107F6000B0710AA84178F17181783170C17871706F
:107F70000179B1704179F17081793171C079707195
:107F8000787B3072B87B70727078317841EA002962
:107F9000F078B17841EA00247079317941EA00251E
:107FA000F079B17941EA002808A8009043462A46B2
:107FB0002146484600F02FF900281BD1787E012881
:107FC00052D100207876DFF87C095B210170002116
:107FD0004170852181700021C170AE2101710021A5
:107FE0004171702181710121C171EE210172002165
:107FF000417239E000207876DFF848093178017065
:1080000071784170B1788170F178C1703179017106
:1080100071794171B1798171F179C171317A0172EE
:10802000717A4172DDE90801C7E90A01CC46C7F857
:1080300034C02246BA632B46FB63386B012862DBEF
:10804000DDE90801CDE90401B87B0290787B01905D
:10805000CDF8008061460FF68C10FBF71FFE386BE1
:10806000401E38634FE04ED0DFF8D80801783170F9
:10807000417871708178B170C178F1700179317196
:10808000417971718179B171C179F171017A31727E
:10809000407A7072002038767078317841EA002991
:1080A000F078B17841EA00247079317941EA00250D
:1080B000F079B17941EA0028787B8DF81900307A9F
:1080C000787397F80EB0707AB87308A8009043469A
:1080D0002A462146484600F09EF8DDE90801CDE930
:1080E0000401B87B0290787B0190CDF800802B468C
:1080F000224649460FF62010FBF7D0FD9DF81900E7
:10810000787387F80EB01FFA89F9B9F15B0F11D1B6
:10811000A4B2852C0ED1ADB2AE2D0BD1B8F5B87F7F
:1081200008D1307AEE2805D1707A002802D10120DA
:108130008AF8720001200DB0BDE8F08F38A700204A
:10814000D88A00081CB504460020ADF806008DF85A
:1081500004000120009001AB902272210920FBF75E
:108160007EFE002801D1002016BD9DF8040000F01D
:10817000FC008DF80400012C0AD0042C04D0102C33
:108180001FD0402C22D026E040F001008DF80400E2
:1081900090208DF806009DF804008DF80700DFF8A8
:1081A000A8479DF8040000F00300A07302230DF11E
:1081B000060272210920FBF7F6FD00280DD10020F0
:1081C00016BD40F002008DF80400E1E740F0030026
:1081D0008DF80400DCE7002016BD0120E07416BD18
:1081E000DFF86417C8767047DFF85C27D2E90A0128
:1081F000704730B4DFF85047656B0560A06B0860CE
:10820000E06B1060206C1860D4E90A01029AC2E9A0
:10821000000130BC70472DE9F44F86B0DFF8289795
:1082200099F81B20012A0CD140F2E36203924FF42B
:10823000FA784FF4D77540F66B6440F2C36202924D
:108240000BE040F6213203924FF4AF786FF009054E
:1082500040F6573440F2976202921A468B468246A5
:108260000BEB0A00BDF8181010FA81F0801A00EB31
:10827000D070461036B299F80E000FF65C01405CE3
:1082800099F80D10C1F5807110FB01F740F6DC2C58
:108290000CFB07F704978902B1F5803F01D34FF635
:1082A000FF71C9000A27B1FBF7F1102865D18B4295
:1082B00063D30120FFF746FF002876D1AAEB060022
:1082C0000190ABEB060CBDF81800811B0091109FCC
:1082D00056450BDAD7E9000102460B46019800FB30
:1082E00008F0C11710185941C7E900015E450CDAC2
:1082F000D7E9000102460B464FF47A7000FB0CF000
:10830000C11710185941C7E90001BDF8180086428D
:1083100008DAD7E90001009A6A43801851EBE2714C
:10832000C7E90001D7E90001002905DC00DB03D221
:1083300000200146C7E90001D7E90023DDF80CA0C1
:108340004FEAEA7BAAFB02010AFB03110BFB0211B5
:10835000C7E90001049A00230CF0B6FCC7E900014C
:1083600000986043019990FBF1F002990818C9F850
:108370004000012007B0BDE8F08F102807D1642A23
:1083800005DA4020FFF7DEFE00280ED196E74028F0
:1083900002D164398B4203D201288FD1642A8DDA4D
:1083A0001020FFF7CFFE002888D00020E2E70FF270
:1083B0002C71092009F0CEBBDFF88C15487501201F
:1083C000704710B5DFF884452020207000206070D1
:1083D0000A20A0700020E0700A2020710020607147
:1083E0003220A0710020E07207222146DFF86005EC
:1083F000FBF78CFB00206072012010BD00B583B03C
:1084000000A800210A4606C00722DFF840150DF13A
:108410000100FBF77BFBA0208DF80000082300AAD9
:1084200072210720FBF7BFFC002801D100200EBD00
:1084300001200EBD80B5DFF81405417B012903D171
:1084400000F0F9F8012002BD018AFF290CD00029B3
:108450000DD0C27A521CC272491E0182417AD2B238
:10846000914201D20021C17200F010F805E0418A6A
:1084700001820021C17200F009F80820FEF7DAFD40
:10848000002801D1002002BD012002BD38B5002026
:10849000ADF80000DFF8B444208A002801D1A07AAA
:1084A00060720722E07AC0EBC000DFF8A414411824
:1084B0002046FBF72BFBFFF7A1FFA7208DF800005C
:1084C00000ADE0896870022300AA72210720FBF743
:1084D0006AFC002801D1002032BD01211020FEF7E6
:1084E00045FBA9208DF8000001206870022300AA36
:1084F00072210720FBF757FC002801D1002032BD74
:10850000012032BD3EB50446607902902079019089
:10851000E0780090A378627821780FF23450FBF76E
:10852000BDFBDFF830548122FF212846FCF7C8F854
:1085300080222146681CFBF7E9FA0020287081237D
:108540002A4672210720FBF72EFC002805D10FF2E6
:108550001850FBF7A3FB00203EBD01203EBD10B527
:1085600001780F2905DADFF8E423527A521C8A4297
:1085700005DA0FF20050FBF791FB002010BD4278A6
:10858000202A01DB202242700022C2704271C1EB1E
:10859000C102DFF8BC332021D154D11800244C7023
:1085A0004478002C01D1002401E06400641E8C7129
:1085B0008C79002C01D0012C02D13024D45401E05C
:1085C0002024D45482788A70C278CA7002790A71E1
:1085D00040794871012010BDDC48417A491C417244
:1085E00081720120704738B50446D84D2C82FFF7C0
:1085F000E8FE002C00D06C8221460FF28840FBF789
:108600004DFB012032BDD149487301207047D2494A
:10861000087001207047D0480078704780B5CB497A
:1086200008730A7B5200CA8101460FF26840FBF7CB
:1086300035FB012002BD10B5C44C217A0FF2644015
:10864000FBF72CFB0020FFF7B7FE00206073607281
:1086500001461020FEF78AFAFEF763FA0820FEF7BB
:10866000E9FC002801D1002010BD012010BD38B563
:108670000FF23C40FBF712FB0020ADF80000B74CB6
:108680002078002814D0002500E06D1C052D11D2A3
:10869000281900798DF800002819007B8DF8010059
:1086A000022300AA72210920FBF77DFB0028ECD1F0
:1086B000002032BD012032BD10B582B0A24CA17E97
:1086C0000FF2F830FBF7EAFA0020ADF80000902036
:1086D0008DF8000003208DF80100022300AA72210A
:1086E0000920FBF760FB002801D1002016BD002007
:1086F000A0840320A0730120607701460420FEF7C8
:1087000035FA002801D1002016BDFA20FEF792FCB0
:10871000002801D1002016BD012016BD80B50FF242
:10872000AC30FBF7BBFA8848002141770420FEF704
:108730001DFA002801D1002002BDFA20FEF77AFCC4
:10874000002801D1002002BD012002BD0120704798
:10875000F0B587B002A800210A4606C00846CDE958
:1087600004018DF80400012000900DF105039E2204
:1087700072210920FBF773FB002801D1002057E08C
:108780000120009001ABAB2272210720FBF767FBB1
:10879000002801D100204BE09DF80500400603D5DC
:1087A0009DF80400400601D5002041E0082000901B
:1087B00002AB942272210920FBF751FB002801D162
:1087C000002035E0002202218020FEF755F85E4AA5
:1087D0009DF80800907102AB5E78D67198781070A1
:1087E000DC785470197991705D79D5709F79177123
:1087F00093F807C082F805C0537B1372937B5372C2
:1088000004AB0093927942EA062347EA0C2241EA3C
:10881000052140EA0420FFF7FEFC40221146AB2070
:10882000FEF72AF8022211468020FEF725F80120E3
:1088300007B0F0BD7FB5044602A800210A4606C075
:108840003F48056E08468DF80400012000900DF1A8
:1088500005039E2272210920FBF701FB002801D1AC
:10886000002069E00120009001ABAB2272210720BB
:10887000FBF7F5FA002801D100205DE09DF8050026
:10888000400603D59DF80400400601D4002053E0C3
:108890000820009002AB942272210920FBF7DFFA36
:1088A000002801D1002047E0002202218020FDF7AE
:1088B000E3FF02A841789DF8082042EA0121C2782E
:1088C000837843EA022212FA81F14279037943EA7A
:1088D000022211FA82F1C279807940EA022011FA6B
:1088E00080F0194E411000EB91708010B08400228E
:1088F0004021AB20FDF7C0FF022211468020FDF78A
:10890000BBFFB6F924002070001260703078A070B0
:108910007078E070B0782071F07860713079A07173
:108920007079E071B0792072F0796072307AA0725B
:10893000707AE0720120A87704B070BD00000000DA
:10894000AC4901203855012038A7002018540120D7
:10895000B8310120A8480120D556012098A900204F
:108960000FF2A011182009F0F5B80000233E54487A
:10897000534554202564202564000000233E5052B6
:1089800020474554205452494D20307825782030D6
:1089900078257800233E4C4947500000233E4C493F
:1089A000474F203078257800233E4C49474300004C
:1089B000233E6920723D256420673D256420623D89
:1089C000256420633D2564206174696D653D2564DF
:1089D00020616761696E3D2564206C75783D256C6A
:1089E0006C642000233E723D256420673D25642091
:1089F000623D256420633D2564206174696D653D99
:108A0000256420616761696E3D2564206C75783D41
:108A1000256C6C6420000000233E4040723D2564BC
:108A200020673D256420623D256420633D25642048
:108A30006174696D653D25642C20616761696E3DD7
:108A40002564206C75783D256C6C64200000000066
:108A50004D4244202564202564202564202564207F
:108A600025642025640000004D6F6265616D20570C
:108A7000460000004D6F6265616D20486F702046B2
:108A800061696C004D4220486F70436F756E7420B1
:108A9000256400004D6F6265616D204C656E3D255B
:108AA000640000004D4220436C6F73652025640014
:108AB000233E4C494749525000000000233E4C4998
:108AC0004749524F2030782578000000233E4C491A
:108AD000474952430000000001041040657D000832
:108AE000AF7D0008157E0008517E000800000000E0
:108AF000557E00080000000000000000000000009B
:108B0000000000006F860008B98600081D87000875
:108B10004D870008518700083588000800000000D4
:108B20000000000000000000000000000901002813
:108B300007D500F00F00DFF8BC2B801800F8041CEC
:108B40007047DFF8B42B8154704710B5401EB0F168
:108B5000807F01D3012010BDDFF8A04B60600F21A2
:108B60004FF0FF30FFF7E2FF0020A06007202060F9
:108B7000002010BDF0B583B0DFF8844B20460CF028
:108B80003DF9DFF8805B28460CF038F9DFF8786BA8
:108B900030460CF033F9012108460CF052FA01215D
:108BA00002200CF04EFA012104200CF04AFA0121B7
:108BB00008200CF046FA012110200CF042FA0121A5
:108BC00080200CF03EFA03208DF8040001208DF87F
:108BD000060000208DF807008DF805004FF6FF779E
:108BE000009700A920460CF065F9009700A92846D7
:108BF0000CF060F9009700A9DFF8100B0CF05AF99F
:108C000000A9DFF80C0B0CF055F900A9DFF8580C9F
:108C10000CF050F900A930460CF04CF9002101206D
:108C20000CF00FFA002102200CF00BFA00210420B6
:108C30000CF007FA002108200CF003FA00211020A4
:108C40000CF0FFF9002180200CF0FBF901218320BA
:108C50000CF0F7F901208DF8040000208DF80500D4
:108C600001208DF8060000208DF8070003200090F9
:108C700000A928460CF01EF9032128460183C046AE
:108C800001208DF8040000208DF80500ADF80600E5
:108C90004FF40040009000A920460CF00BF94FF46F
:108CA000004120464183C0460420009001208DF8F9
:108CB00006008DF8040000208DF8050002208DF8D4
:108CC000070000A920460CF0F5F80820009000A944
:108CD00020460CF0EFF80422062128460CF038F963
:108CE0000422072128460CF033F902208DF80400F5
:108CF00001208DF805008DF8060000208DF8070092
:108D00004020009000A928460CF0D4F88020009064
:108D100000A928460CF0CEF8012180200CF091F932
:108D2000012000908DF806008DF8040000208DF8D9
:108D300005008DF80700012130460183C04600A9D7
:108D400030460CF0B7F8012180200CF07AF90220AF
:108D5000009000208DF8060001208DF8040000200E
:108D60008DF805008DF8070000A930460CF0A2F838
:108D7000022130460183C04601208DF80400002006
:108D80008DF80500ADF806000C20009000A92046E3
:108D90000CF090F8F7BD1FB5DFF8D04AA0422FD1F4
:108DA00001214FF400100CF057F9012102200CF0C2
:108DB00048F901214FF400100CF06FF900214FF435
:108DC00000100CF06AF90020ADF804004BF6FF70BB
:108DD000ADF806004FF48060ADF80A004FF4804013
:108DE000ADF80C000A20ADF80800DFF8640C009024
:108DF00000A920460CF0EDF9012120460CF04CFAB8
:108E00001FBDF8B5044640F6FF752E46DFF8447CDA
:108E1000022138460CF00AFB002805D12846451EE1
:108E20000028F5D10020F2BD214638468181C04698
:108E3000012138460CF0FAFA002804D13046461ECB
:108E40000028F5D1EEE738468089C046C0B2F2BDB1
:108E5000F8B504460D461646DFF8A8784FF4805161
:108E600038464183C04605F07F00FFF7CAFF03E0A4
:108E700014F8010BFFF7C5FF3046461E80B20028EC
:108E8000F6D14FF480513846BDE8F4400CF05CB8A0
:108E9000F8B504460D461646DFF868784FF4805161
:108EA00038464183C04645F08000FFF7AAFF04E042
:108EB0000020FFF7A6FF04F8010B3046461E80B2E3
:108EC0000028F5D14FF480513846BDE8F4400CF04D
:108ED0003BB830B587B0044601214FF480400CF018
:108EE000BBF8012102200CF0ACF801208DF8040041
:108EF00000208DF8060001208DF8070000208DF875
:108F000005004FF480500090DFF8F85700A928467C
:108F10000BF0D0FF4FF4805128464183C04600201B
:108F200040F6FF7100E0401C8842FCD34FF48051B2
:108F300028460183C04605220D2128460CF008F87A
:108F400005220E2128460CF003F805220F212846A1
:108F50000BF0FEFF02208DF804000020ADF80600A3
:108F60008DF805004FF46040009000A928460BF0F2
:108F7000A1FF20460CF0F2F90020ADF80800ADF892
:108F80000C000220ADF80E000120ADF810004FF4E7
:108F90000070ADF812001820ADF814000020ADF8F4
:108FA00016000720ADF818004FF48270ADF80A00E3
:108FB00002A920460CF001FA0321DFF8980AC94300
:108FC0000181012120460CF01BFA07B030BD2DE9CC
:108FD000F04192B001214FF480500CF048F801218B
:108FE00008460CF02EF801214FF480000CF029F80F
:108FF000DFF80C470522114620460BF0A9FF052299
:10900000072120460BF0A4FF0522062120460BF085
:109010009FFF0522042120460BF09AFF02208DF8C5
:10902000040001208DF805000020ADF80600202086
:10903000009000A920460BF03DFF8020009000A981
:1090400020460BF037FF4020009000A920460BF08F
:1090500031FF1020009000A920460BF02BFFDFF815
:10906000F84920460CF07AF9DFF8F0590020288002
:1090700068600120288100206881E860072028823C
:1090800000206880DFF8D86930460CF0D7F9DFF8A7
:10909000D47938460CF0D2F94FF480600690002164
:1090A0000D9103210E9100210F910A910890DFF894
:1090B0008C0A039008461090099007904FF40030F6
:1090C0000C9008460B904FF0C068CDF80880402007
:1090D00005900846049002A930460CF033FA0020AF
:1090E0000B90CDF80880059005F11400049002A9BA
:1090F00038460CF027FA00206880294620460CF0FC
:109100005CF90122022120460CF086F90122114669
:1091100020460CF081F9012120460CF071F9002164
:1091200030460CF036FA002138460CF032FA12B014
:10913000BDE8F08100B585B0012103200BF081FF6F
:1091400001214FF480400BF092FF00208DF81000B9
:1091500001208DF81300039003A9DFF8A4050BF09C
:10916000A9FE002108460CF07DFA00208DF80800C9
:1091700001208DF80A0001900C208DF8090001A84B
:109180000CF084FA17208DF800000F208DF80100F4
:1091900000208DF8020001208DF8030000A80CF0DB
:1091A000C4FA05B000BD10B586B0012103200BF054
:1091B00048FF01214FF480400BF059FF00208DF84B
:1091C00010008DF813004FF40074039403A9DFF826
:1091D00034050BF06FFE092101200CF043FA00204A
:1091E0008DF8080001208DF80A00019408208DF800
:1091F000090001A80CF04AFA20460CF089FA172061
:109200008DF800000F208DF8010000208DF802007D
:1092100001208DF8030000A80CF087FA06B010BDFD
:1092200000B585B0012103200BF00BFF01214FF4A5
:1092300080400BF01CFF00208DF810008DF813000B
:109240000820039003A9DFF8BC040BF033FE0321D0
:1092500001200CF007FA00208DF8080001208DF89D
:109260000A00082001900C208DF8090001A80CF0DC
:109270000DFA08200CF04CFA09208DF800000F20A0
:109280008DF8010000208DF8020001208DF8030008
:1092900000A80CF04AFA05B000BD30B58DB0044608
:1092A00001214FF480700BF0E2FE00A80BF03CFEB1
:1092B0000A20009003208DF8040000208DF807009C
:1092C00000A9DFF83C040BF0F5FD0CF067FA02A8EA
:1092D0000CF0A9FA4FF48030039002A80CF095FA34
:1092E00006A80CF088FADFF8785B06A928460CF08F
:1092F00062FA07230122214628460CF0A5FA012133
:1093000028460CF0E4FA012128460CF092FA0DB040
:1093100030BD38B5DFF8484B20460CF0D3FA4FF497
:109320007A75022120460CF0E9FA002803D128467C
:10933000451E0128F5DA2046BDE832400CF0D2BACD
:1093400080B50021DFF8180B0CF073FA00214FF400
:109350008070BDE804400BF08ABE80B502F0FAFBD5
:1093600000280FD0002002F0FFFBF9F763FBD0F8D4
:109370008400FAF76FFCDFF84C1B0620BDE80440C0
:1093800000F032BFDFF8780A0068002801D10CF045
:10939000DFFADFF8700A0CF0F8FCDFF8281B022077
:1093A000BDE8044000F020BF38B5040011D0DFF85C
:1093B000500A0068002801D10CF0CAFADFF8445ABC
:1093C000214628460CF06CFD2846BDE832400CF0E2
:1093D000DCBCDFF8300A0CF02AFDBDE831400CF0AF
:1093E000C9BA000070B501240023DFF8781A1A46C4
:1093F0008A608A6812F00C0FFBD1DFF86C2A0546F0
:109400000B2D45D8DFE805F01C44444406171C2BFF
:1094100030353A3F8D6845F080058D60DFF8A85AF9
:109420004FF4C0662E600D6825F080750D60DFF882
:109430009C5A15602DE02346DFF8945A156028E009
:109440008D688D60DFF8805A4FF4C0662E600D681D
:1094500025F080750D60DFF87C5A156019E0022355
:10946000DFF8745A156014E00323DFF8705A1560B2
:109470000FE00423DFF8685A15600AE00523DFF8DF
:10948000F45A156005E00623DFF8EC5A156000E099
:109490001C46002B4AD003EBC3030FF2BC055B193B
:1094A0008D688D600D6825F080750D600D6825F064
:1094B00080650D609D781E8845EA8615DE78760801
:1094C000761E45EA06451E7945EA06654D60DD884B
:1094D0001E7A360746EA8515DFF8A46A35600D68FE
:1094E00045F080750D600D68AD01FCD55B7943F4E6
:1094F000C063DFF8D4592B608B688B608B688B60FE
:10950000052804D1886840F09000886005E00A28AA
:1095100003D1886840F480508860886840F0020079
:109520008860886800F00C000828FAD11068DFF81D
:109530006C1A884207D2DFF8680A016821F44041BA
:1095400041F48041016010684FF47A71B0FBF1F092
:10955000FFF7FBFA204670BD200110040F03020143
:1095600003F00010060F01020103C00010080F01F4
:10957000020103C00010060F01020103F0001006F3
:109580000F01020103C80010040F02020103A8002A
:1095900010020F030201030024E7002800E0401E30
:1095A000FDD1704730B583B00725B04988426AD1F4
:1095B00001208DF804008DF805008DF806000020CC
:1095C0008DF8070040200090DFF8D84900A9204618
:1095D0000BF070FC8020009000A920460BF06AFC84
:1095E000402120464183C0460F20FFF7D6FF40218F
:1095F00020460183C0460F20FFF7CFFF2846451EB7
:1096000080B20028ECD18020009000A920460BF009
:1096100051FC402120464183C0460520FFF7BDFF95
:10962000802120460183C0460520FFF7B6FF402178
:1096300020460183C0460A20FFF7AFFF40212046A5
:109640004183C0460520FFF7A8FF802120464183C3
:10965000C0460520FFF7A1FF02208DF8040001207D
:109660008DF805008DF8060000208DF807004020D9
:10967000009000A920460BF01DFC8020009000A95E
:1096800020460BF017FC37BD38B50024DFF8185919
:10969000012128680BF039FE28680BF06BFD286863
:1096A000FFF779FB05E02868FFF77CFF2868FFF7E4
:1096B00072FB4FF4003128680BF032FE002802D014
:1096C000641C332CEFDB31BD30B40022838A008B65
:1096D000DFF8D448656843EA00400840000255EAD4
:1096E000102060600840884200D10122104630BC42
:1096F0007047000018ED00E000E400E010E000E03A
:109700000000024000040240001C02400008024029
:10971000000C02402DE9F84F04460D4616464FF462
:1097200020691F78DFF880884FF40031D8F80000F6
:109730000BF0F6FD002808D04846A0F101090028EA
:10974000F2D1FFF7A1FF00208CE0D8F800000188DB
:109750004FF6FF52114001800121D8F800000BF0B4
:10976000A7FD4FF4007AD1460020C8F80400D8F8CD
:1097700000B0DFF838185846FFF7A6FF002805D1DB
:109780004846A0F101090028F1D163E0D14600224A
:10979000214658460BF0A4FD0020C8F80400D8F874
:1097A0000040DFF80C182046FFF78EFF002805D197
:1097B0004846A0F101090028F1D14BE03146C9B279
:1097C00020460182C046D1460020C8F80400D8F8DF
:1097D0000040DFF8E0172046FFF776FF002805D1AC
:1097E0004846A0F101090028F1D133E0012F15D13D
:1097F000297820460182C046D1460020C8F80400DE
:10980000DFF8B417D8F80000FFF75EFF002823D177
:109810004846A0F101090028F2D11BE03846471E56
:10982000C0B2002818D015F8011BD8F8000001823A
:10983000C046D1460020C8F80400DFF87C17D8F8ED
:109840000000FFF741FF0028E8D14846A0F10109D8
:109850000028F2D1002005E00121D8F800000BF02B
:1098600033FD0120BDE8F28F00100240005400409B
:109870002DE9F54F81B00D461E464FF4206837782C
:10988000DFF824474FF4003120680BF049FD002831
:1098900008D04046A0F101080028F3D1FFF7F4FEFC
:1098A0000020D3E0206801884FF6FF52114001806C
:1098B000012120680BF0FCFC4FF40079C846002021
:1098C0006060DFF8E8A6D4F800B051465846FFF7CC
:1098D000FBFE002805D14046A0F101080028F2D186
:1098E00091E000229DF8041058460BF0F9FCC846A0
:1098F00000206060D4F800B0DFF8B4165846FFF7D7
:10990000E3FE002805D14046A0F101080028F1D16E
:1099100079E0BDF80810C9B258460182C046C84671
:10992000DFF8981620680BF0FBFC002805D14046B4
:10993000A0F101080028F3D165E0012120680BF0B7
:10994000B7FCC84600206060D4F800B051465846C5
:10995000FFF7BAFE002805D14046A0F10108002813
:10996000F2D150E001229DF8041058460BF0B8FCEB
:10997000022FC84639DADFF8481620680BF0D0FC11
:10998000002805D14046A0F101080028F3D13AE0B3
:10999000002120680BF0ADFC2068018B01210BF049
:1099A00093FCC846DFF81C1620680BF0B9FC0028B1
:1099B00005D14046A0F101080028F3D123E020683A
:1099C000008AC0B228703078401E3070C8462068C7
:1099D0000188890505D54046A0F101080028F6D187
:1099E00011E001210BF085FC2BE000206060DFF826
:1099F000D8152068FFF768FE002806D14046A0F180
:109A000001080028F3D1002020E0012616E0012FF4
:109A10000CD1012E0AD10026314620680BF069FCDA
:109A20002068818A018B01210BF04EFC2068818A1D
:109A3000490603D5008A05F8010B7F1EFFB2002FEF
:109A4000E5D1012120680BF054FC0120BDE8FE8F18
:109A5000801A06000038004000300140D851012033
:109A60008864024010640240DFF86005016808293C
:109A700033D1DFF8F0130A6842F080720A6042685E
:109A8000B2F1806F03D10A6842F080620A600A680E
:109A90009201FCD58A6842F002028A608A6802F06C
:109AA0000C02082AFAD14268B2F1806F02D10A682A
:109AB0001201FCD5DFF8B0130968DFF8E024914209
:109AC00007D2DFF8DC140A6822F4404242F48042F4
:109AD0000A6000210160416070474168B1F1806F08
:109AE0000AD1DFF880130A6842F080620A600A68CF
:109AF0001201FCD5002141607047DFF8D4040168F1
:109B000041F080510160DFF89804016889088900FC
:109B100041F001010160DFF8BC040FF22501016092
:109B20007047DFF8B404016821F00401016030BF20
:109B3000016841F004010160704700000C300140F1
:109B400010B5FAF742F8807A012803D101200CF011
:109B5000CEF902E000200CF0CAF9DFF87C44802145
:109B6000DFF878040BF062FC002818D172B6BD480B
:109B7000DFF85814826802F00C020A60006800F0F6
:109B800080604860206840F00400206030BF62B60A
:109B9000206820F004002060BDE8104064E72068E1
:109BA00020F00400206030BF206840F004002060F6
:109BB00010BDDFF82004006800470000DFF8201423
:109BC000401E052812D8DFE800F00306090C110F2B
:109BD000DFF8D0130AE0DFF80C1407E0DFF8081410
:109BE00004E0DFF8081401E0DFF8041408467047C9
:109BF00010B50C46FFF7E2FF214689B2BDE81040E0
:109C00000BF0A2B910B50C46FFF7D8FF214689B278
:109C1000BDE810400BF09AB9E0B500238DF808308C
:109C200001238DF80A30002A03D10C228DF8092077
:109C300002E008228DF80920042840D8DFE800F06F
:109C40000316222B2B000820019009208DF800001C
:109C50000F208DF8010000208DF80200012924D189
:109C600018468DF803008DF80A0022E0184601908E
:109C700010208DF8090006208DF800000E208DF8C8
:109C80000100E8E70220019007208DF800000F2076
:109C90008DF80100DFE74FF40070019017208DF878
:109CA00000000F208DF80100D5E78DF803008DF836
:109CB0000A0001A80BF0EAFC00A80BF036FD07BD76
:109CC0000821B8480BF039B910B5044601214FF40A
:109CD00080200BF0B6F92146102008F0DEFB0021B1
:109CE0004FF48020BDE810400BF0ABB910B5012156
:109CF0004FF480200BF0A5F9102008F0DBFB0446A0
:109D000000214FF480200BF09CF97B200BF0E6F94A
:109D1000002802D099A0F9F7C1FF7A200BF0DEF9F4
:109D2000002802D097A0F9F7B9FF79200BF0D6F9F7
:109D3000002802D094A0F9F7B1FF7C200BF0CEF9F7
:109D4000002802D091A0F9F7A9FF7D200BF0C6F9F9
:109D5000002802D08EA0F9F7A1FF7E200BF0BEF9FB
:109D6000002802D08BA0F9F799FF7F200BF0B6F9FD
:109D7000002802D088A0F9F791FF0BF0C1F9204626
:109D8000C0B210BD3EB50C4615460422014602A8DD
:109D9000F9F7BCFE0422214601A8F9F7B7FE042218
:109DA000294600A8F9F7B2FE02A9002008F046FAF9
:109DB00001A9002008F0BBFA08F0B4FA04468D4A65
:109DC000002300981946101A63EB0101490341EA88
:109DD000D04140030AF09AFF0090844205D2011B53
:109DE0004FF0004008F073FB37BDA04207D2C4F526
:109DF0000050009909184FF0004008F068FB37BD8B
:109E00008851012098E200202DE9704384B0044677
:109E10000D46164602A9002008F05FFA01A90020AD
:109E200008F0D5FA08F07EFA0090724AA2FB008989
:109E30004FEA583848EAC948A2EB080000900422CB
:109E400002A92046F9F762FE042201A92846F9F783
:109E50005DFE042200A93046F9F758FEBDE87F8375
:109E60000020014000380240D0A9002070B48C1EB0
:109E7000012C01DA0C34401E3C216425B0FBF5F5C1
:109E8000C5EB90054FF4C876B0FBF6F6751940F2B5
:109E90006F1674430C26B4FBF6F46419121940F2E1
:109EA0006D1404FB0020544A101800EB400203EB31
:109EB000C200039A01FB0020049A01FB002070BC41
:109EC00070470000F0E10020003C024000127A00E0
:109ED000809698000024F40000366E010048E801E6
:109EE000005A62021CB50C4601680191416800915C
:109EF0008368C2680169491C406900F26C70FFF711
:109F0000B5FF2060002016BD10B58EB03B4800683C
:109F10008404A40C01A9002008F0DFF900A90020A6
:109F200008F055FA9DF8040006909DF8050005908C
:109F30009DF8060004909DF80100401E08909DF8D1
:109F4000020007909DF803006430099002A904A85C
:109F5000FFF7C8FF4FF47A7010FB04F0800BC0F5D8
:109F60007A700390029A4FF47A73C117E3FB0201EF
:109F70000EB010BD80F0FA0200BD0105504F520036
:109F80008438024050494E00424F5200534654001C
:109F900049574400575744004C50570001879303DA
:109FA00000700040000402403CAA002001000300B1
:109FB00082000700800007008400070004000010F2
:109FC000020000104000001002000300A85501200C
:109FD00040380240A055012010ED00E00030014063
:109FE0000000024000080240000C02400010024045
:109FF000001C024000CA9A3B7505F5FF2828004066
:10A0000038B5F9F705FB0446104DF8F713FD286045
:10A010000AF054F90AF057F968600AF091FA0C480E
:10A02000C4F8140104F58A700A4941600A49816044
:10A030000A49C1600A490161012032BD03494968EA
:10A04000896808470148406800680047C8550120F2
:10A05000B1390008AD390008B9390008BD39000828
:10A06000C13900082DE9F04786B0044601A8142143
:10A07000FAF764FBF9F7A9FD05464FF00208002640
:10A0800001E0761C76B20A2E80F29F80022EF8D074
:10A09000032EF6D0062EF4D0524850F82670787A67
:10A0A000002805D1D7F82001406880470028E8D073
:10A0B00008F8046008F101084FFA88F830460928CA
:10A0C00051D8DFE800F0050A505014245019504BC5
:10A0D000C8212846F9F7DCFF45E095F8120201286F
:10A0E00041D04FF448712846F9F7D2FF3BE03221C6
:10A0F0002846F9F7CDFF36E007208DF80400FF2051
:10A100008DF8050032212846F9F7C2FF2BE03C21EB
:10A110002846F9F7BDFF4FF00009B9F1030F22DA25
:10A120000020D7F820110969884714212846F9F73B
:10A13000AFFF0120D7F8201109698847142128466C
:10A14000F9F7A6FFB9F1020F05DA062101A8D7F841
:10A1500020215269904709F10109DEE74FF4167199
:10A160002846F9F795FF07F10C0999F8151001A891
:10A17000D7F8202152699047002819D0D9F80C004F
:10A18000F96800EB010A99F8152001A95046F9F782
:10A19000BDFC3846F8F78CFD99F81520514608EBC0
:10A1A0000400F9F7B3FC99F9150080444FFA88F8D8
:10A1B000787A00287FF465AFD7F82001806880475F
:10A1C00000287FF45EAF002009E0A8F10200ADF89E
:10A1D0000000022200A92046F9F798FC002006B0F2
:10A1E000BDE8F087AC49012038B505000C0094F8B3
:10A1F0005000642802D08020FBF7B8F9FBF7ADFCD3
:10A20000802080F3118800BF00BFA0692843A061AF
:10A21000207C10F0F800082806D1E069A169084206
:10A2200002D02000FBF742FD07484078F0210842A9
:10A2300002D09920FBF79AF903484078002802D110
:10A24000002080F3118831BD28A8002062B38B075D
:10A2500008D0521E11F8013B00F8013B00F02480A9
:10A260008B07F6D1830740F0208000BF103A07D358
:10A2700030B4B1E83810103AA0E83810F9D230BC48
:10A28000530724BFB1E80810A0E8081044BF51F8F4
:10A29000043B40F8043BD20724BF31F8022B20F8DE
:10A2A000022B44BF0B7803707047083A07D3B1E81C
:10A2B0000810083A40F8043B40F804CBF7D25307A3
:10A2C000E4E7000038B50C46154600F0FBF92046DF
:10A2D00000F04CFA00F0CEFAC046C046002D03D084
:10A2E000DFF84C0BC06A32BDDFF8481B0878002845
:10A2F00003D0DFF83C0BC06A01E04FF0FF300022D2
:10A300000A7032BD0000000070B52DED068BB0EE76
:10A31000408A0120DFF8F42A00E0401CDFF8F01A40
:10A32000896888420ADA52F8303000EE103AB8EE06
:10A33000C00AB4EE480AF1EE10FAEEDB884208DB00
:10A3400002EBC10050F8040C00EE100AF8EEC08ACF
:10A350004AE002EBC004A4F10806DFF8B81A01EBEA
:10A36000C00555E90201002213460BF0C7FD37D2A4
:10A370009FEDD29B18EE100A01F0A8FA53EC192BAE
:10A380000BF0D4FD41EC100B0BF044FEB0EE40AAF4
:10A39000F0EE60AA54F8080C07F0CEFE53EC192B2F
:10A3A0000BF0C4FD41EC100B0BF034FE51EC1A0B1A
:10A3B00053EC102B0BF038FE55E9022301F0AEFAF6
:10A3C00004460D46706807F0B7FE22462B460BF098
:10A3D000ADFD0BF0E9FE00EE100AF8EEC08A03E0D6
:10A3E00096ED010AF8EEC08ABDEEC80A10EE100A1A
:10A3F00000F0DAFC38EE800ABDEC068B70BD000080
:10A4000038B52DED048BB0EE408A0120DFF8082A24
:10A4100000E0401CDFF8F819496888420ADA02EBCC
:10A42000C00393ED010AB8EEC00AB4EE480AF1EE9B
:10A4300010FAEEDB884208DB02EBC10050F8080C92
:10A4400000EE100AB8EEC00A47E002EBC00454F870
:10A45000081C08EE901ADFF8C41901EBC00555E995
:10A460000201002213460BF049FD34D218EE900A87
:10A4700007F062FEDFF8A829DFF8A8390BF056FDD7
:10A4800041EC100B0BF0C6FDB0EE409AF0EE609A76
:10A4900054F8040C00EE100AB8EEC00A38EE400A78
:10A4A00010EE100A01F012FA55E9022301F036FA13
:10A4B00053EC192B0BF03AFD41EC110B9FEDA90B5E
:10A4C0000CF0DEF851EC100B0BF06EFE00EE100AF3
:10A4D000B8EEC00A01E0B8EEE80ABDEC048B31BD6D
:10A4E00038B52DED048BB0EE408A0120DFF8382915
:10A4F00000E0401CDFF81819C96888420ADA02EB4C
:10A50000C00393ED010AB8EEC00AB4EE408AF1EE42
:10A5100010FAEED5884208DB02EBC10050F8080CB7
:10A5200000EE100AB8EEC00A47E002EBC00454F88F
:10A53000081C08EE901ADFF8F41801EBC00555E985
:10A540000201002213460BF0D9FC34D218EE900A17
:10A5500007F0F2FDDFF8C828DFF8C8380BF0E6FC9A
:10A5600041EC100B0BF056FDB0EE409AF0EE609A05
:10A5700054F8040C00EE100AB8EEC00A38EE400A97
:10A5800010EE100A01F0A2F955E9022301F0C6F914
:10A5900053EC192B0BF0CAFC41EC110B9FED710B26
:10A5A0000CF06EF851EC100B0BF0FEFD00EE100AF3
:10A5B000B8EEC00A01E0B8EEE80ABDEC048B31BD8C
:10A5C00070B52DED028B94B0DFF86448207B002835
:10A5D00008D140F229120FF680010FF69400F9F726
:10A5E0005DFB67E012A8009010AB0DAA0EA90FA8A2
:10A5F000FDF7FFFD94ED010AFFF786FEB0EE408AFD
:10A60000FFF7FEFE84ED090AB0EE480AFFF768FF87
:10A6100084ED0A0A18EE100A01F058F941EC100B0B
:10A620000CF04EFA51EC100B0BF0BEFD0546DFF8B6
:10A630000468E06AA84229D00C95A06A01F046F9A6
:10A64000CDE90A01606801F041F9CDE90801606ACD
:10A6500001F03CF9CDE90601A06801F037F9CDE938
:10A660000401206802900D9801900E9800900F9BB5
:10A6700040F237120FF2E0710FF62C00F9F70EFBE3
:10A68000E06A2063E5620120307001E00020307054
:10A6900094ED010ADFEDAC0AB4EE600AF1EE10FAB7
:10A6A00001DB012000E0002094F84410814201D039
:10A6B00084F8440014B0BDEC028B70BD7B14AE472F
:10A6C000E17A843F80B52DED028B90ED000AD0ED4C
:10A6D000010A90ED028A20EE000A00EEA00A08EEC0
:10A6E000080A10EE100A01F0F1F841EC100B0CF022
:10A6F0000DFA51EC100B01F0E3F900EE100ADFED5A
:10A70000930AB4EE600AF1EE10FA28D4DFED900A55
:10A71000B4EE600AF1EE10FA21DA88EE000A10EECB
:10A72000100A01F0D3F841EC100B0CF0FFFA51ECD9
:10A73000100B01F0C5F900EE100ADFED860A20EEDD
:10A74000200ADFF8EC06DFED840A20EE200AD0EDC7
:10A750000D0A9FEDD41A00EE810A80ED0D0ABDECC2
:10A76000028B01BD000000000000244010B52DED5B
:10A77000028B00EE100AB8EEC08AF0EE488ADFF8CD
:10A78000B04684ED000A207D002804D0C4ED028A82
:10A790000020207568E094ED0D0ADFEDCE0AB4EEDE
:10A7A000600AF1EE10FA0AD5D4ED010A9FEDCA1A3B
:10A7B000F4EE410AF1EE10FA01D5012000E000208C
:10A7C000401E8041C043C00F84F8380094F8380020
:10A7D00000280DD094F83910814209D010EE100AEB
:10A7E00001F074F802460B460FF2F060F9F756FAE2
:10A7F00094F8380094F8391081F00101084308D129
:10A80000606B01F063F802460B460FF2FC60F9F74B
:10A8100045FA94F8380094F8441008420BD094EDAF
:10A82000090AB4EE408AF1EE10FA04D5002084F84B
:10A830003800F0EE408A94F83800002808D094EDF3
:10A84000010AF4EE408AF1EE10FA01D5F0EE408AEA
:10A8500084F8390094ED040A30EE280AF6EE000A76
:10A8600020EE200A84ED020AC4ED048ABDEC028BBE
:10A8700010BD000000B583B000A8F9F70AFD9DF9EE
:10A8800000004FF461619DF90120C2EB02139A00B0
:10A8900011FB00209DF9021040FA81F04FF47A710B
:10A8A000BDF9032001FB0020DFF8841591ED020AB9
:10A8B0000A7B002A09D181ED010A01220A730022D4
:10A8C0008A61C861BDE807407AE6D1ED0A0AB4EEB4
:10A8D000600AF1EE10FA0FDB8A69012A02DA01221E
:10A8E0008A61C861CA6902F57A7290422BDB81EDF8
:10A8F000010ABDE8074063E6D1ED090AF4EE400A1B
:10A90000F1EE10FA19DBD1ED010A9FEDBB1AF4EE5E
:10A91000410AF1EE10FA10DB8A69002A03D44FF0E5
:10A92000FF328A61C861CA6902F6B83290420ADB16
:10A9300081ED010ABDE8074042E68A69002A02D09B
:10A9400000228A61C86107BD00803B45DD0CFB40E9
:10A95000A7493C41E42E65428C2EBA3DF0B589B042
:10A960000446DFF8AC54A1F1F000F1280BD30B46FC
:10A9700040F2CB120FF2C0510FF2E050F9F78EF90E
:10A98000002028708BE02378062B0AD040F2D712E3
:10A990000FF2A4510FF2F850F9F780F90020287057
:10A9A0007DE003A81821F9F7C9FE6078686003907C
:10A9B00003AEA0787060E078A860B0602079F060A5
:10A9C0006079E8603061A07908900727002100E0F5
:10A9D000491C06290ADA56F821201F2AF8DB0FF253
:10A9E000E850F9F75BF90020287058E0F0220021C8
:10A9F000DFF82404F9F764FEF0220021DFF80C04EC
:10AA0000F9F75EFEF0220021DFF81C04F9F758FE8A
:10AA100000A80FF2DC51B1E80C10A0E80C100021E6
:10AA20001CE03B5D7F1C17F804C043EA0C237F1C2D
:10AA300017F804C043EA0C437F1C17F804C043EA2C
:10AA40000C637F1C0DF1000C5CF821C00CEBC20CF8
:10AA5000CCF80430521C8242E3DB491C03291BDA88
:10AA6000002213E0385D7B1C1F5D40EA07205B1C61
:10AA70001F5D40EA07405B1C1F5D40EA07605F1CEA
:10AA800000AB53F8213043F83200521C56F8310025
:10AA90008242E7DB0022DEE702202870012009B0B5
:10AAA000F0BD00002EBA683FE14800210160FF219F
:10AAB000C1630021016401210175E3494163002163
:10AAC000816001734FF0FF31C1620021018780F87E
:10AAD0004410704700008C4201007A4410B5ADF577
:10AAE000347D78A80FF21451F022FFF7BFFB3CA889
:10AAF0000FF2F851F022FFF7B9FB00A80FF2DC616A
:10AB0000F022FFF7B3FBC24C0C2060601C20A06059
:10AB10001020E060F02278A9BF48F8F7F7FFF02294
:10AB20003CA9BA48F8F7F2FFF02200A9BE48F8F7AE
:10AB3000EDFF012020700DF5347D10BD38B52DEDF1
:10AB4000068B044615469FEDBC0BAC4250D0994293
:10AB50004ED0581A07F0F0FA41EC180B9FEDBB9B52
:10AB6000204607F0E9FA53EC192B0BF0DFF941EC22
:10AB70001A0B284607F0E0FA53EC192B0BF0D6F924
:10AB800041EC100B0A98002818D00BF043FAB0EEF5
:10AB9000409AF0EE609AB0EE4A0AF0EE6A0A0BF0C4
:10ABA00039FA53EC102B51EC190B0BF03DFA53EC26
:10ABB000182B0CF0C3F841EC100B19E00BF02AFA3B
:10ABC000B0EE409AF0EE609AB0EE4A0AF0EE6A0AF1
:10ABD0000BF020FA53EC102B51EC190B0BF024FA6C
:10ABE00002460B4651EC180B0CF0A8F841EC100B88
:10ABF000BDEC068B31BD0000010080402DE9F84F0F
:10AC0000DFF81892F02200214846F9F759FD814CEF
:10AC1000F02200212046F9F753FD844DF022002157
:10AC20002846F9F74DFD7A4E7068A0F1010AB06828
:10AC3000471EF068A0F101084FF0000B11E07648C4
:10AC400000EBCB0101220092CB688A68496850F87A
:10AC50003B00FFF773FF09EBCB0080ED000B0BF11E
:10AC6000010BD345EBDB4FF0000911E0674800EB27
:10AC7000C90100220092CB688A68496850F83900FF
:10AC8000FFF75CFF04EBC90080ED000B09F101093F
:10AC9000B945EBDB002410E0634800EBC40101225E
:10ACA0000092CB688A68496850F83400FFF746FF85
:10ACB00005EBC40080ED000B641C4445ECDB3078F0
:10ACC000022801D103203070BDE8F18F80B50FF26A
:10ACD000FC50F8F7E3FF4E480078002808D14822DE
:10ACE00000215348F9F7ECFCFFF7F8FEFFF786FF69
:10ACF000BDE80140D8E638B504460D462078FF2867
:10AD000005D1691E89B2601CBDE8344015E00FF220
:10AD1000C450F8F7C3FF3E48007802280CD0FFF774
:10AD2000C3FE29462046FFF719FE002801D1FFF790
:10AD3000D5FEBDE8314061E731BDF8B504460025D8
:10AD40003F4E207840083060012729E0385D791CAB
:10AD50000A5D40EA0220491C0A5D40EA0240491CA3
:10AD60000A5D40EA0262491C364840F835200A5D17
:10AD7000491C0B5D42EA0322491C0B5D42EA034277
:10AD8000491C0B5D42EA03634F1C00EBC5014B609D
:10AD900050F8352029460FF25850F8F77FFF6D1C08
:10ADA00030688542D2DBF1BD70B40021244A1268BC
:10ADB000002A244B03D19FED270A24E0491C53F8B5
:10ADC0003140914201DA8442F8DA03EBC102A2F188
:10ADD0000805686852F8086CB44204D100EE100A05
:10ADE000B8EEC00A0FE0344656680546751B53F8A6
:10ADF00031102246891A95FBF1F101FB040000EEA7
:10AE0000100AB8EEC00A70BC7047000074A200209F
:10AE1000E8A900207841012084A100208840012079
:10AE20007B14AE47E17A843F64A30020684201208E
:10AE3000804E0120B59500200000000000000000B9
:10AE400030560120983F0120000080BF7B14AE47A0
:10AE5000E17A843F0000000075706461746541759B
:10AE6000746F4272696768746E65737300000000E6
:10AE70005B5353505D5B44415649445D202573202C
:10AE800028256429206E6F206C75782076616C759A
:10AE9000652066726F6D2073656E736F72206D61D1
:10AEA0006E616765722000002573202825642920C3
:10AEB0002825642025642025642925642C20252E3E
:10AEC000316C662C20252E316C663C252E316C664B
:10AED0003C252E316C662028256429005B53535095
:10AEE0005D204175746F4272696768746E65737333
:10AEF000202D204C4F434B20696E202874416E67F3
:10AF00003A20252E316629005B5353505D20417550
:10AF1000746F4272696768746E657373202D204C7C
:10AF20004F434B206F7574202874416E673A20257B
:10AF30002E316629000000007061727365427269EB
:10AF40006768746E65737341727261797346726F6C
:10AF50006D506C6174666F726D0000005B535350EE
:10AF60005D5B44415649445D20496E76616C69647D
:10AF7000204272696768746E657373205461626CF5
:10AF800065204C656E6774682028256429000000E0
:10AF90005B5353505D5B44415649445D202573200B
:10AFA00028256429205461626C6520436F756E7496
:10AFB000206973206E6F742076616C696420282587
:10AFC00064292121000000005B5353505D20627210
:10AFD000696768746E657373436E744172726179E8
:10AFE0005B25645D203A202564203E20313000003E
:10AFF00084A1002074A2002064A3002000000000AF
:10B0000009000000000000004000000005000000F2
:10B01000540000001900000080000000C80000007B
:10B02000FF0000002C010000010100009001000061
:10B0300003010000F401000005010000E803000026
:10B0400007010000D007000009010000B80B000054
:10B050000B010000881300000D010000000000003B
:10B0600000000000000000000000000000000000E0
:10B0700000000000000000000000000000000000D0
:10B0800000000000000000000000000000000000C0
:10B0900000000000000000000000000000000000B0
:10B0A00000000000000000000000000000000000A0
:10B0B0000000000000000000000000000000000090
:10B0C0000000000000000000000000000000000080
:10B0D0000000000000000000000000000000000070
:10B0E0000000000000000000000000000000000060
:10B0F00009000000010000000B0000000200000039
:10B100000E00000003000000130000000400000017
:10B110001500000005000000170000000A000000F4
:10B120002B0000001E000000540000003200000050
:10B13000540000006400000056000000C800000039
:10B1400063000000F401000080000000E80300003C
:10B15000A5000000D0070000FF000000B70B0000B2
:10B16000FF000000B80B0000010100009F0F00006D
:10B1700001010000A00F0000030100008713000080
:10B180000301000088130000050100000F270000E4
:10B190000501000010270000070100001F4E0000FD
:10B1A00007010000204E0000090100002F7500007B
:10B1B00009010000307500000B0100003F9C0000F9
:10B1C0000B010000409C00000D0100000000000089
:10B1D000000000000000000000000000000000006F
:10B1E0000900000004000000090000000700000042
:10B1F0000B0000000A0000000E0000000F0000001D
:10B20000130000002C01000054000000E8030000BF
:10B210006F000000DC05000080000000B80B00009B
:10B22000A500000088130000D9000000701700007E
:10B23000FF0000001027000001010000102700009F
:10B2400003010000409C000005010000409C00003C
:10B250000901000040420F000B0100000000000047
:10B2600000000000000000000000000000000000DE
:10B2700000000000000000000000000000000000CE
:10B2800000000000000000000000000000000000BE
:10B2900000000000000000000000000000000000AE
:10B2A000000000000000000000000000000000009E
:10B2B000000000000000000000000000000000008E
:10B2C00000000000000000000000000041425F4953
:10B2D0006E6974005B5353505D20557064617465F2
:10B2E0004272696768746E6573735461626C65005D
:10B2F0005B5353505D206272696768746E65737347
:10B300004F66667365745461626C655B25645D208D
:10B310003A2025642C20256400000000EFF3038010
:10B32000704770B582B006460C46204606F0DCF841
:10B330000546202D05D10422314600A8F8F7E6FB8A
:10B3400006E0102D16D10222314600A8F8F7DEFBE8
:10B35000002000E0401CA8420EDA015D7829F9D0F7
:10B36000009A2B465B1E1B1ADA4002F001023039AC
:10B370008A42EFD0002076BD012076BDDFF80814A8
:10B38000016006207047A0F10060B0F5483F01D889
:10B390000120704700207047F8B504460D46002094
:10B3A00000902068FFF7EFFF00281AD000A8FFF7F1
:10B3B000E5FF0646002700E07F1CB74211D2009847
:10B3C00050F8371000EBC70040684042226852082E
:10B3D00010EB4200FFF7A5FF0028EDD02F60012001
:10B3E000F2BD0020F2BDF8B507460C461546002612
:10B3F00030460090002F1ED0002C09D1F2BD06EB84
:10B400008600800057F8041B490849004151761C0A
:10B410000C2E0FD200A93846FFF7BEFF002807D137
:10B420003868FFF7B0FF002802D13F1DBC42F1D2BF
:10B43000BC42E4D23046F2BD38B5D44904220A6099
:10B44000D34A1268121F1623B2FBF3F24A6010F1BE
:10B45000030F02D010F1130F0BD1CE4CA0680BF0EC
:10B4600091FD0546A0680BF099FD4119CA48806A14
:10B4700007E008F051FD044608F050FD0119C648E8
:10B48000406AC64AC44B9B6913601432FFF7ABFF96
:10B49000012032BD2DE9FC4104460025B9A60FF27A
:10B4A0002432314608F01EFD0746BD4802680FF2FF
:10B4B0004431381908F016FD00EB0708B64FB86C98
:10B4C0000190B86B00907B6B3A6B0FF2403108EB48
:10B4D000040008F007FD8044FA6C0FF2683108EBB5
:10B4E000040008F0FFFC80447B69BA690FF2683100
:10B4F00008EB040008F0F6FC804407F194020FF218
:10B50000703108EB040008F0EDFC00EB08070FF2C7
:10B5100070323146381908F0E5FCC71907E05918B0
:10B520000B1D0FF2703108F0DDFCC7196D1C05EB27
:10B530008500830099495A583819002AEFD10FF233
:10B540006032314602B0BDE8F04108F0CBBC95480E
:10B5500095490A6802604A6842608A688260CA68DF
:10B56000C2600A6902614A6942610A7E8261097F9A
:10B5700081618E490A7882614A6842628A68826281
:10B58000CA68C2620A6902634A6942638A6982635D
:10B59000CA69C2638A6EC0F88820854A9369C0F878
:10B5A0009830D368C0F88C301369C0F89030536974
:10B5B000C0F894300B6FC0F89C304B6FC0F8A030CF
:10B5C0008B6FC0F8A430C96FC0F8A810794909681A
:10B5D000C0F8AC1078490B68C0F8CC304B68C0F8A4
:10B5E000D0308B68C0F8D430CB68C0F8D830096947
:10B5F000C0F8DC105168C0F8E8101168C0F8E41019
:10B600007047F8B507460C460025634E6FF01E01E3
:10B61000401A29D0083827D0001F10D0001F1AD098
:10B62000083818D0001F28D104F120003062EFF351
:10B63000148040F00200F062306AB0621DE004F154
:10B6400064003062EFF3148040F00200F062306A70
:10B65000B062012511E004F120003062EFF31480A4
:10B66000F062306A706208E004F164003062EFF367
:10B670001480F062306A70620125EFF30580306358
:10B68000EFF300807063FFF749FEB063EFF31080C3
:10B69000F063EFF311803064EFF313807064F1EE28
:10B6A000100AB064F764002004E054F8201046F853
:10B6B0002010401C0828F8D3012D0AD1002006E0F4
:10B6C00006EB800104EB8002126A0A65401C112817
:10B6D000F6D3F1BD0BF0DCBC89B20BF079BC70B5D0
:10B6E00082B00024754601462846FFF78AFFFFF71F
:10B6F0002EFF2846FFF7A0FE0220ADF8020040F61C
:10B700000200ADF800002D4D02220DF10201284685
:10B71000F8F7FCF9022200A9A81CF8F7F7F9DD20D8
:10B72000287140F606060DE06C714FF40062E002ED
:10B7300000F10051A81DF8F7E9F931462846FFF756
:10B74000CBFF641C402CEFD3DD206871A81DFFF7F0
:10B75000A1FE31462846FFF7BFFFFFF7BBFF73BDD1
:10B7600010B5044605F0C0FEC0B2142800DB13205B
:10B77000024621461248F8F7C9F94FF0AC3000787C
:10B7800010BD00002573000010A9002010560120F4
:10B79000FCFF030828A80020784701205843012017
:10B7A00068AA00204844012000ED00E020ED00E000
:10B7B00004E000E0A0ED00E034EF00E088F90020B4
:10B7C0000C4801200A0A0A0A3D3D3D3D3D3D3D3DF4
:10B7D0003D3D3D2043726173682044756D70204982
:10B7E0006E666F203D3D3D3D3D3D3D3D3D3D3D0A4D
:10B7F00000000000204669726D7761726520566511
:10B800007273696F6E203A2025640A0020495053F4
:10B8100052203D20307825782C2041505352203D35
:10B8200020307825780A2078505352203D203078F7
:10B8300025782C205046534352203D2030782578DF
:10B840000A000000204372617368204D6F64652018
:10B850003D20307825780A00205043203D20307864
:10B8600025782C204C52203D20307825780A000085
:10B87000204361757365203A2025730A000000009B
:10B880000A203C3C2043616C6C20537461636B2044
:10B890003E3E0A002030782578202025730A0000DB
:10B8A0003D3D3D3D3D3D3D3D3D3D3D3D3D3D3D3DC8
:10B8B0003D3D3D3D3D3D3D3D3D3D3D3D3D3D3D3DB8
:10B8C0003D3D3D3D3D3D3D0A0A0000005FF0FF0C5F
:10B8D0001CEAD05114BF614506E0C110400721F0B9
:10B8E000E04101F16051704779B900F00041000278
:10B8F0000AD0B0FA80FC00FA0CF001F16051A1EB23
:10B900000C5101EBD0214005704741020CBF40F4BF
:10B91000E0016FF00001002070470000B0B581EA3F
:10B92000030C0CF0004C40F2FF7515EA11541DBFDA
:10B9300015EA1357AC42AF4239E0E41923EA455304
:10B9400043F48013C90241F0004141EA505EC7024E
:10B950001100A7FB020200284FF00000EEFB0120BF
:10B960004FF00001E3FB072118BF42F0010240182D
:10B9700000214941E3FB0E01A4F580640F0302D2CC
:10B9800052004041494154F101046CDD470872F115
:10B99000004250F1000051EB0451A1F580115CBF51
:10B9A00041EA0C01B0BD4CEA05510020B0BD05EAEA
:10B9B0001357AC4214BFAF4241E050EA410E1CBFE6
:10B9C00052EA430E02E061460020B0BD24423C44EE
:10B9D0001BD15FEA070EF6D0090302BF0146002023
:10B9E000AEF1140EB1FA81F7AEEB070401FA07FECF
:10B9F0000C37C7F1200100FA07F7C8404EEA000EE5
:10BA000023EA455343F48013A2E733F00043B3FA2B
:10BA100083F704BFB2FA82FE77440B3FE41BB7F111
:10BA2000200E2FBF02FA0EF3BB40C7F1200E22FA00
:10BA30000EFE38BF43EA0E03BA40641C82E750EAA8
:10BA4000410E14BF52EA430E6FF000014FF400178D
:10BA500017EB430F8ABF194617EB410FB5E74CEAC6
:10BA600005510020B0BDD4F10104B4F120070FDA74
:10BA7000C4F12007520828BF42F0010210FA07F56E
:10BA800001FA07F7E1BF2A43E0403843E1400FE005
:10BA9000352C98DCC7F1200452EA400220FA07F264
:10BAA00018BF42F0010231FA07F0A1400A43002119
:10BAB00072F1004250F1000051EB0C01B0BD0000EA
:10BAC0004FEAF17CBCF1E04C2CBFBCF5001F11E04B
:10BAD0005FEA4C0C34BFBCF17F5F2EE05FEA9C0C48
:10BAE0004FEA0C1C4FEA3C0CC10071F100414CEBD9
:10BAF00050707047C90241EA5051C00218BF41F06E
:10BB0000010141F000414FEA6C50C0F109002128C9
:10BB100010D240EACC7CCCF1200C11FA0CF070F180
:10BB20000040CCF1200C21FA0CF00CF0004C40EB62
:10BB30000C0070474FEACC707047490011F5001FA8
:10BB400004D84FEACC10FF30C0057047C8177047C3
:10BB50000BF09FBA80B5F6F76DFFD0F88800F7F7C5
:10BB600003FD0348007802BD0149087070470000DA
:10BB7000F65601200FB410B5032200210846F7F74E
:10BB800049FD022801D1022020E00FF24800F8F719
:10BB900085F8DFF8944C0020E073E082E0629DF8C5
:10BBA0000C209DF80B109DF80A000BF048FD582260
:10BBB0000021DFF8080DF8F783FD00202064A07451
:10BBC00020746083E06160642075012010BC5DF822
:10BBD00014FB000050443A20537461727450656441
:10BBE0006F2D30383232000080B503220021012051
:10BBF000F7F710FD032801D1032002BD012002BD8B
:10BC000070B52DED028B96B002A8F7F762FDDFF854
:10BC1000185C286A697A427A914205D0407A0EF01F
:10BC200073F8286A407A6872286A297A027B9142FE
:10BC300005D0007B0EF065F8286A007B287205218C
:10BC40000320F7F7D0FD002814D1DFF8740C0A9018
:10BC500000206883A883E88B401CE88380B240F210
:10BC6000EF2188424ADB0FF2E800F8F717F80020CE
:10BC7000E88343E09DED0A8A95F90A00022836D14F
:10BC800095ED110AB4EE408AF1EE10FA03D1688BFB
:10BC9000401C688301E0002068839FEDA60AB4EE93
:10BCA000408AF1EE10FA06D49FEDA30AB4EE408A62
:10BCB000F1EE10FA03DBA88B401CA88301E0002002
:10BCC000A883AE8B6C8B972C01DA972E12DB18EEC3
:10BCD000100AFFF7FBFDCDE90001324621460FF2C5
:10BCE0008400F7F7DBFF00206883A88302E00020D0
:10BCF0006883A8830020E88385ED118A686AD0F8FC
:10BD0000B8400BF01BFCA87295F90A00022806D176
:10BD10003C2C04D114210320F7F7DDFC07E00128B7
:10BD200005D1142C03D13C210320F7F7D4FC204685
:10BD300080B2DDED0A1A02A991EC030A0BF04BFA6E
:10BD4000A86A2018A862012016B0BDEC028B70BD55
:10BD500050443A204261726F44697361626C656459
:10BD60000000000050443A204241524F20256420F8
:10BD7000256420256600000010B5DFF8AC4A94F970
:10BD8000000000283AD494F90C0094F90110814283
:10BD900028D1A17B0818207340B23D2801DB3C3834
:10BDA000207394F90C100FF27000F7F777FF002062
:10BDB000A062DFF8A00B90F9010010F1010F01D192
:10BDC000012010BD94F90110081A06F0B5F921F010
:10BDD00000410AF0E9F940B2012801DB012010BD61
:10BDE000002010BDDFF8700B90F90120914203D0C4
:10BDF000D4E90023C0E90023002010BDA06ADFF8C9
:10BE0000601B884205DB0FF21C00F7F747FF01209B
:10BE100010BD002010BD000050443A204E54202593
:10BE20006400000050443A204E6F54696D65000074
:10BE30002DE9F8430026DFF8F04901E07819207376
:10BE400094F90C50002E1BD46078461B76B294F9FE
:10BE50000E70002EF2D5304606F06EF921F000414A
:10BE600002460B4690469946384606F065F942462A
:10BE70004B460DF0A9FFE3D2E81B20730026DFE755
:10BE80003C2D02DBA5F13C002073BDE8F18310B529
:10BE9000DFF89449002020740120A0720020E07295
:10BEA0004FF0FF3020700F2060731420A07300202B
:10BEB000E073E082E062E074A063E0632822014660
:10BEC000DFF8A00AF8F7FCFBF7F7A2FB6062F7F7D0
:10BED0007CFE2062606ADFF8901AC0F8D810D83073
:10BEE000DFF8881A4160DFF8881A81600FF27D213F
:10BEF000C1600FF685210161012010BD10B582B02F
:10BF00004FF46163C1EB0114A40013FB0043D31889
:10BF10004FF47A746343DFF84C4A2360DFF8083942
:10BF20009B7C009313460A460146DFF8480AF7F760
:10BF3000B5FE13BD0000FA430180BB442DE9F0417A
:10BF40002DED028BAAB0DFF87469314684B06846E3
:10BF50005822FEF78BF90FBC00F0B4FC10EE100A6B
:10BF6000FFF7B4FC41EC100B9FED7E8BDFF8F4493A
:10BF7000656853EC102B51EC180BFFF7CFFC0AF05F
:10BF800013F915FA80F060604FF6FF75A84200D3F0
:10BF90006560314684B068465822FEF767F90FBCE9
:10BFA00000F044FC10EE100AFFF790FC41EC100B7F
:10BFB000A76853EC102B51EC180BFFF7AFFC0AF0FD
:10BFC000F3F817FA80F0A060A84200D3A560002023
:10BFD000139002201290314684B068465822FEF732
:10BFE00045F90FBC00F0A2FAA1894018A08180B2E7
:10BFF000FF2801DBFF20A081002013900320129076
:10C00000314684B068465822FEF730F90FBC00F084
:10C010008DFA216940182061A84200D325610020D3
:10C02000139006201290314684B068465822FEF7DD
:10C030001DF90FBC00F07AFAA18A4018A08280B2E4
:10C04000FF2801DBFF20A082002013900720129020
:10C05000314684B068465822FEF708F90FBC00F05C
:10C0600065FAE18A4018E08280B2FF2801DBFF20F8
:10C07000E0820020139008201290314684B0684678
:10C080005822FEF7F3F80FBC00F050FAA1694018EF
:10C09000A061A84200D3A56100201390092012904E
:10C0A000314684B068465822FEF7E0F80FBC00F035
:10C0B0003DFAE1694018E061A84200D3E56114A8A7
:10C0C0000BF041FADFF86077D7F838802398FFF754
:10C0D000FDFB0022DFF8943DFFF720FC0AF064F836
:10C0E00058FA80F0B863F96B491CF963B0FBF1F0C2
:10C0F00084F820000020139001201290314684B073
:10C1000068465822FEF7B2F80FBC00F00FFA616AD9
:10C1100040186062A84200D36562787C00F005FB9D
:10C120002AB0BDEC028BBDE8F081DFF838088189C8
:10C13000002914D10169002911D1818A00290ED169
:10C14000C18A00290BD18169002908D1C169002960
:10C1500005D1406A401E8041C043C00F7047012096
:10C160007047000000000000000059402DE9F04F2A
:10C17000ABB0814600254E46DFF8AC46207C4946F0
:10C1800088420ED0012E40F09E8028460BF09AFE89
:10C19000606A90F9B42090F9B510DFF8D40CF7F785
:10C1A0007DFD14A80BF0CFF9DFF810A728461390F7
:10C1B00001201290514684B068465822FEF756F886
:10C1C0000FBC00F0B3F907469DED230ADAED0F0A24
:10C1D00030EE600A10EE100AFFF778FB2A46DFF80F
:10C1E0008C3CFFF79BFB09F0DFFF80461FFA88F8C5
:10C1F000BDF89A00BAF84A10A0EB010B5FFA8BFB6E
:10C20000606A90F84517002903D190F84417002977
:10C2100005D0616B149A5118226C891A616300F67B
:10C2200034014978002903D190F83428002A05D038
:10C23000226B149B9A18236CD21A2263B9F1000F57
:10C2400052D1226B002A08D0002903D190F834087B
:10C25000002802D001200DF04EFE606B00280BD0AC
:10C26000606A90F84517002903D190F84407002828
:10C2700002D001200DF0F9FE002F02D15BEA080088
:10C2800000D001250020A0624FF0FF302070DFF8C1
:10C29000C826D4E90001C2E90001DFF83C2CC2E95C
:10C2A0000001DFF8B026C2E90001607B2073207C2A
:10C2B000002851D000202074A07C00284CD0012000
:10C2C000E074054648E0B9F1000F07D10FF6A4303D
:10C2D000F7F7E4FC01200BF0F5FD62E70FF6A03064
:10C2E000F7F7DCFC2846EDE000F0ADF900281BD0A4
:10C2F00000A8F7F7CEFF204600A90522FDF7A6FF0C
:10C300002846E072DFF85026D4E90001C2E90001B6
:10C3100094F9023094F9012094F900100FF67C3062
:10C32000F7F7BCFCFFF784FD00A8F7F7B2FF204643
:10C3300000A90522FDF78AFFFFF71EFD00280BD09C
:10C34000DFF81026D4E90001C2E90001A07C002832
:10C3500001D00120E0740125012E07D1207C49463F
:10C36000884203D000F04FFA84F81090012E58D183
:10C37000002F56D0DFF8609B607CA17C08430CD175
:10C380000120A0740522214609F10800F7F7BEFB41
:10C39000A27861782078FFF7B1FD94F9010099F94E
:10C3A0000910401A411E222901D2012005E010F196
:10C3B000230F01DA012000E0002001282AD100200B
:10C3C000A063E063FFF7B1FE002823D028220021FC
:10C3D000DFF89005F8F774F9607C401C6074C0B217
:10C3E000152809D10FF6CC20F7F758FC0120E0748E
:10C3F0000020607401250DE0A07C401CA074A27890
:10C4000061782078FFF77AFD0522214609F10800BE
:10C41000F7F77CFBFFF792FD582214A95046F7F777
:10C4200075FBE07B012833D1E08A002805D10FF6A7
:10C430009420F7F733FC012523E0E16A814218D20A
:10C44000002F02D15BEA080000D00125DFF8889AAE
:10C4500099F9020094F90220904212D0491CE1623D
:10C460000FF6C430F7F71AFCD4E90001C9E900015E
:10C4700007E00020E073E082E0620FF6BC30F7F7DF
:10C480000DFC012E04D1A07C002801D00120E07415
:10C490002846012801D10021A162616A91F8B510F6
:10C4A000002906D10021A162012801D100F0ABF9D9
:10C4B0000025002D03D1207D012800D101251498ED
:10C4C000206428462BB0BDE8F08F10B5DFF81C0BB8
:10C4D00000218162032205210020F7F79BF8044622
:10C4E00000F007F8204610BD032205210120F7F7D0
:10C4F00091B800B597B000A80BF025F8582200A914
:10C50000DFF8F00AF7F702FB012017B000BDDFF8F3
:10C51000DC0A006B7047DFF8D40A00210163704722
:10C52000DFF8C80A00214163704700000FB410B55E
:10C5300096B000249DF9BC0001280BD10BF070F9D6
:10C540001899884202D3441AE4B272E08038441A3F
:10C55000E4B26EE000A80AF0F6FF9DF9B800401EB4
:10C56000082866D8DFE800F02905111D2936424E5B
:10C570005A0001981999884201D3441A59E0DFF80A
:10C580008C2A1018401A441C53E002981A998842C9
:10C5900001D3441A4DE0DFF8742A1018401A441CE5
:10C5A00047E003981B99884201D3441A41E0DFF821
:10C5B0005C2A1018401A441C3BE0009818998842E5
:10C5C00001D3441A35E0DFF8441A08181899401AC4
:10C5D000441C2EE004981C99884201D3441A28E098
:10C5E000DFF8282A1018401A441C22E005981D99EB
:10C5F000884201D3441A1CE0DFF8102A1018401AB0
:10C60000441C16E006981E99884201D3441A10E093
:10C61000DFF8F8291018401A441C0AE007981F99FF
:10C62000884201D3441A04E0DFF8E0291018401AC8
:10C63000441C204616B010BC5DF814FBDFF8AC09B2
:10C640000121C1727047DFF8A409C07A704710B5A4
:10C6500004460AF08BFF022C0CD1DFF89009406AE7
:10C6600090F9B42090F9B5100FF6E010BDE8104035
:10C67000F7F714BB10BD0146DFF87029792902DBFA
:10C680007820D08200E0D0820120D0730FF6D41041
:10C69000F7F704BB0000000010B5040001D101242D
:10C6A00002E0072C00DB062421460FF6CC10F7F73A
:10C6B000F5FA641E052C2DD8DFE804F0030A1118E2
:10C6C0001F26DFF82809372141733C21817321E0BF
:10C6D000DFF81809192141731E2181731AE0DFF870
:10C6E0000C090F2141731421817313E0DFF8FC085A
:10C6F0000A2141730F2181730CE0DFF8F008072154
:10C7000041730C21817305E0DFF8E00805214173D6
:10C710000A218173DFF8D408417B0173BDE8104022
:10C72000FFF786BBDFF8AC08704700EB800188009C
:10C73000421CDFF8A0088B4992B20B681B0E135401
:10C74000521C92B20B681B0C1354521C92B20B6811
:10C750001B0A1354521C92B20B681354521C92B20F
:10C760004B681B0A1354521C92B24B681354521C50
:10C7700092B28B681B0A1354521C92B28B681354EA
:10C78000521C92B28B891354521C92B20B691B0A31
:10C790001354521C92B20B691354521C92B28B8ADE
:10C7A0001354521C92B2CB8A1354521C92B28B690E
:10C7B0001B0A1354521C92B28B691354521C92B22E
:10C7C000CB691B0A1354521C92B2CB691354521CEE
:10C7D00092B291F820301354521C92B24B6A1B0A49
:10C7E0001354521C92B2496A11540F48511C0183D0
:10C7F000704710B5DFF8F447218B0FF68800F7F784
:10C800004DFA208B10BD80B5282200215548F7F73E
:10C8100057FFDFF8D807002141740121018300216F
:10C8200081748163C16301BDC84E01200FB400B59E
:10C8300097B000A80AF087FE9DED090ADDED210AF8
:10C84000B4EE600AF1EE10FA02DB30EE600A05E0A9
:10C850009FED421A71EE600A30EE800A10EE100A67
:10C86000FFF734F8DFF87027DFF8703709F05EFB68
:10C87000FFF726F9FFF72AF80022DFF86437FFF701
:10C880004DF809F091FC00EE100AB8EEC00A10EE67
:10C89000100AFFF71BF8DFF84027DFF84837FFF7EB
:10C8A0003DF8DFF84427DFF8683709F03FFBFFF772
:10C8B00007F900EE100A17B05DF814FB7C4D01205B
:10C8C00000007A440FB400B597B000A80AF03BFE10
:10C8D0009DED0E0ADDED260AB4EE600AF1EE10FAC7
:10C8E00002DB30EE600A05E09FED1C1A71EE600A73
:10C8F00030EE800A10EE100AFEF7E8FFDFF8D826C7
:10C90000DFF8D83609F012FBFFF7DAF8FEF7DEFFA2
:10C910000022DFF8CC36FFF701F809F045FC00EE05
:10C92000100AB8EEC00A10EE100AFEF7CFFFDFF8CB
:10C93000A826DFF8B036FEF7F1FFDFF8AC26DFF807
:10C94000D03609F0F3FAFFF7BBF800EE100A17B083
:10C950005DF814FBD8550120D055012000247449FE
:10C9600040771B00B051012075BB0008E9BB0008EF
:10C9700001BC0008647703082DE9F0472DED068B14
:10C98000AAB006460D4614A80AF0DDFD40F249148F
:10C99000287814FB006001210170DFF85076F87BE5
:10C9A000012804D1F88A002801D10020F8732878E2
:10C9B00014FB00604170287814FB00600321817033
:10C9C000387D012813D1287814FB0060E021017123
:10C9D0005022DFF81C16287814FB0060401DF7F782
:10C9E00095F82878401C28700020387539E2F87CCA
:10C9F000012820D1B87C00281DD0297814FB0161C2
:10CA0000C0220A71DFF8CC150870287814FB006882
:10CA1000FFF7EFFEA8F85500287814FB0064FFF735
:10CA200081FEC4F857002878401C2870FFF7EBFE01
:10CA30000020F87415E20DF18C099FED868B9FEDB7
:10CA4000879BDFF8B07500201390012012903946C3
:10CA500084B068465822FDF709FC0FBCFFF766FD5D
:10CA60000A28287814FB006080F0FC800021017106
:10CA7000287814FB006898F804A008461390022058
:10CA80001290394684B068465822FDF7EFFB0FBC80
:10CA9000FFF74CFD40EA0A0088F80400287814FBF0
:10CAA00000680020139003201290394684B0684635
:10CAB0005822FDF7DBFB0FBCFFF738FD88F80500B7
:10CAC000287814FB00680020139004201290394647
:10CAD00084B068465822FDF7C9FB0FBCFFF726FD5E
:10CAE00088F80600287814FB0068002013900520C1
:10CAF0001290394684B068465822FDF7B7FB0FBC48
:10CB0000FFF714FD88F80700394684B068465822BC
:10CB1000FDF7ACFB0FBCFFF7D5FE10EE100AFEF7D9
:10CB2000D5FE41EC100B287814FB006853EC102B59
:10CB300051EC190BFEF7F2FE09F036FBA8F80E00D7
:10CB4000287814FB00682398FEF7C0FE53EC182BDE
:10CB5000FEF7E4FE09F028FB88F81000287814FBA3
:10CB60000060B9F80E104174394684B06846582206
:10CB7000FDF77CFB0FBCFFF759FE10EE100AFEF725
:10CB8000A5FE41EC1A0B287814FB006853EC1A2B15
:10CB900051EC190BFEF7C2FE09F006FB88F81200F3
:10CBA000287814FB0068D9F80800FEF78FFE53ECD4
:10CBB000182BFEF7B3FE09F0F7FA88F8130028786F
:10CBC00014FB00680020139006201290394684B0B0
:10CBD00068465822FDF74AFB0FBCFFF7A7FC88F810
:10CBE0000800287814FB006800201390072012909A
:10CBF000394684B068465822FDF738FB0FBCFFF772
:10CC000095FC88F80900287814FB00680020139030
:10CC100008201290394684B068465822FDF726FB5A
:10CC20000FBCFFF783FC88F80A00287814FB006427
:10CC30000020139009201290394684B0684658228B
:10CC4000FDF714FB0FBCFFF771FCE0722878401C65
:10CC5000287004E1000000000000244000000000F3
:10CC60000000594080210171287814FB00680020E1
:10CC7000139002201290394684B068465822FDF77E
:10CC8000F5FA0FBCFFF752FCC8F80500287814FB32
:10CC900000680020139003201290394684B0684643
:10CCA0005822FDF7E3FA0FBCFFF740FCC8F8090073
:10CCB000287814FB00680020139004201290394655
:10CCC00084B068465822FDF7D1FA0FBCFFF72EFC5E
:10CCD000C8F80D00287814FB006800201390052088
:10CCE0001290394684B068465822FDF7BFFA0FBC4F
:10CCF000FFF71CFCC8F81100394684B0684658227A
:10CD0000FDF7B4FA0FBCFFF7DDFD10EE100AFEF7D9
:10CD1000DDFD41EC100B287814FB006853EC102B60
:10CD200051EC190BFEF7FAFD09F054FAC8F8270088
:10CD3000287814FB00682398FEF7C8FD53EC182BE5
:10CD4000FEF7ECFD09F030FA88F82B00287814FB88
:10CD50000060B9F80E1080F82C10394684B068468F
:10CD60005822FDF783FA0FBCFFF760FD10EE100AA2
:10CD7000FEF7ACFD41EC1A0B9F4AA04B09F0BEF840
:10CD800006D89F4A9F4B0DF01FF801D29FEDA1AB33
:10CD9000287814FB006853EC1A2B51EC180BFEF7A3
:10CDA000BDFD09F001FAA8F82D00287814FB0068F1
:10CDB000D9F80800FEF78AFD53EC182BFEF7AEFDFC
:10CDC00009F0F2F988F82F00287814FB0068002099
:10CDD000139006201290394684B068465822FDF719
:10CDE00045FA0FBCFFF7A2FBC8F81500287814FB22
:10CDF00000680020139007201290394684B06846DE
:10CE00005822FDF733FA0FBCFFF790FBC8F8190062
:10CE1000287814FB006800201390082012903946EF
:10CE200084B068465822FDF721FA0FBCFFF77EFB5D
:10CE3000C8F81D00287814FB006400201390092016
:10CE40001290394684B068465822FDF70FFA0FBC9D
:10CE5000FFF76CFBC4F821002878401C2870FFF70E
:10CE600048FB2AB0BDEC068BBDE8F08700002440EB
:10CE70007877030850443A206C63646F6E000000BA
:10CE800050443A206249734150536C656570696E35
:10CE9000672077726F6E67202564000050443A2047
:10CEA00054696D654E6F74692025642025642025C2
:10CEB0006400000050443A20425420424620465527
:10CEC0004C4C000050443A20526571205065646F0C
:10CED000496E666F31000000F454012010B582B035
:10CEE00004460020002C05D10FF2AC10F6F7D6FE58
:10CEF000002016BD04F15001497801295AD10FF2E2
:10CF0000AC10F6F7CBFE0020ADF8000020E0BDF835
:10CF1000000054F82000BDF80010354A42F8210006
:10CF2000BDF8000054F8200000EE100AB8EE400AE8
:10CF3000DFED270A20EE200ABDF80000324901EBA0
:10CF4000800080ED000ABDF80000401CADF8000034
:10CF5000BDF80000142827DABDF8000054F82000BE
:10CF6000B0F52F7F07D3BDF8000054F8200040F241
:10CF700015518842CBD3BDF8000054F82020BDF8ED
:10CF800000100FF23410F6F789FEBDF800001E49BC
:10CF90004FF07E5241F82020BDF8000014494FF4B4
:10CFA0007A7241F82020CEE71748012101650AF086
:10CFB0008BFF0BE0022909D194F850100FF20C10EE
:10CFC000F6F76CFE94F850000120C046C0B216BDC2
:10CFD0006F12833A0C3801207B14AE47E17A743F1C
:10CFE00000005940E17A843F2D431CEBC84E0120DC
:10CFF000D8A700207C4D0120B81E85EB51B89E3F7C
:10D000009A9999999999B93FE4A600208096980039
:10D01000E2361A3F9A9999999999B93F80B50AF0E1
:10D0200055FF012002BD000050443A207574696D1F
:10D03000657220256400000050443A20526571203A
:10D040005065646F496E666F3200000050443A20AC
:10D05000526566322045282564292C4928256429F3
:10D060000000000050443A205374617274204461FF
:10D07000746120256400000050443A205554202556
:10D080006400000050443A204241544C454E4754FD
:10D09000482025640000000050443A2053462050A8
:10D0A000545233206E756C6C0000000050443A20DE
:10D0B000534620534554310050443A2053462045AE
:10D0C00052525B25645D20256400000050443A20E4
:10D0D00053462053455432202564000010B5DFF834
:10D0E000704D4FF4397200212046F7F7E9FAFF201E
:10D0F0002070E07284F863020020C4F8B8020120B6
:10D10000C4F8BC0210BD30B4034601200B2B25D15E
:10D1100001290ED1DFF8381D511891F954321C46FF
:10D12000DFF8305D555DAC4210DA5A1C81F85422AC
:10D1300031E002292FD1DFF8181D511891F954322E
:10D14000012B03DB5A1E81F8542224E0DFF8000D86
:10D150001018002180F8541208461CE00A2B1AD13E
:10D16000012908D1DFF8E81C511801F515714A7939
:10D17000521C4A710FE002290DD1DFF8D41C51185E
:10D1800001F5157191F90520012A02DB521E4A7141
:10D1900001E00020487130BC7047DFF8B41C81F812
:10D1A0005E0270470FB42DE9F043AFB00124DFF801
:10D1B000A85CA868DFF8986C90F8181600294BD185
:10D1C00090F81906002847D1B4208DF80A004620AF
:10D1D0008DF80B0020468DF80C0000208DF86000C3
:10D1E00003208DF861000DF1630002A95522FDF7BF
:10D1F0002DF80A208DF8620018A8F6F709FB002820
:10D2000001D10220C8E000A8F7F743F89DF800001C
:10D21000B0779DF90100F0779DF9021086F8201093
:10D22000BDF90320A6F821209DF900304FF4616775
:10D23000C0EB001C4FEA8C0017FB030040FA81F0A2
:10D240004FF47A7101FB0020C6F80200C6F80D0009
:10D250000020287000F017FF9DF8DA70B846A1464C
:10D26000B8F1010F1DD1DDF8DB00402805D0D6F85C
:10D2700017100843C6F817000BE0204607E0D6F861
:10D28000171009FA00F21143C6F81710401C0628BF
:10D29000F5DBF07E9DF9DF1009FA01F10843F07625
:10D2A00057E008EB060090F95412002951D190F98B
:10D2B000590200284DD1B8F1020F33D100A8F6F77A
:10D2C000E8FF9DF900004FF461619DF90120C2EB78
:10D2D00002139A0011FB00209DF9021040FA81F020
:10D2E0004FF47A71BDF9032001FB0020C6F8AB02B0
:10D2F000C6F8A70206F12B0006F11E010522FCF775
:10D30000A5FF4FF49660B083DFF8F00CC6F89F02DB
:10D310000020C6F8B8022046C6F8BC0200202861EA
:10D32000E86016E0B8F1030F13D1DDF8DB00C6F8B2
:10D330002300BDF8E0004FF47A714843C6F8270097
:10D340000020C6F8B30286F86D0286F86E0286F8F1
:10D35000B70209FA07F0B17D0143B17531780029B0
:10D3600010D0B8F1010F08D109FA01F1DDF8DB2086
:10D37000914202D1002186F8621296F86A1208439F
:10D3800086F86A023A46214696F85E02FFF7BBFE2F
:10D39000002800D1022420462FB0BDE8F0035DF83C
:10D3A00014FBF0B597B0F8F72AF805460124002DD4
:10D3B00000F08680DFF8986AAA78022196F85E026B
:10D3C000FFF7A1FE002800D10324A87801282BD163
:10D3D000D5F8031006F21700402911D0D6F817200F
:10D3E00022EA0101C6F817100279012395F90770A6
:10D3F000BB409A4302710FF2FC00F6F74FFC03E0CA
:10D400000021C6F817100171D6F8170000282CD19A
:10D41000B07D012195F9022091408843B0750FF24B
:10D42000E000F6F73BFC20E0801990F95402002858
:10D430001BD1A878801990F95902002815D1A87835
:10D4400003280BD106F217000021C16001610846D4
:10D45000C6F8B30206F25E20C1730174B07D0121EB
:10D4600095F9022091408843B075B07D002814D111
:10D470000FF29800F6F712FCFFF730FE01208DF84E
:10D48000000003208DF801000A208DF8020000A89A
:10D49000F6F7BEF900282AD126E0DFF8E00C806814
:10D4A00090F8B410002922D1002180F8181680F8D5
:10D4B0001916FFF713FE0FF62450F6F7EFFB16E0F0
:10D4C0000FF62C50F6F7EAFBFFF708FE20468DF822
:10D4D000000003208DF801000A208DF8020000A84A
:10D4E000F6F796F9002801D1032001E00324204635
:10D4F00017B0F0BD41542D524D20256400000000AE
:10D5000041542D524D2D494E5400000041542D419F
:10D510004C4C52454D4F5645440000002DE9F04F0C
:10D520008DB000208DF8180009A8F6F7B2FE0BA800
:10D530000AF013F84FF00009484602900890DFF80F
:10D5400010499DF82400A0719DF82500E0719DF818
:10D5500026002072BDF82700A4F80900A0794FF436
:10D560006161E279C2EB02139A0011FB0020217A7B
:10D5700040184FF47A71B4F8092001FB0020C4F878
:10D580000200BDF82C0001900090BDF82E70D4F878
:10D590000D10D4F8020000F048FC0600DFF8B8587F
:10D5A00001D0C92E0AD3A868D0F81C2631460FF640
:10D5B0004C40F6F773FBA868D0F81C660198012868
:10D5C00009D1304600F000FD002807D1FFB2022F3C
:10D5D00004D1012702E04846C4F8D802A07D10F02B
:10D5E000040012D0E9687118E96047F230529142A4
:10D5F0000BD32A6989182961D4F89F228A424946A7
:10D6000001D3E96001E02961E96094F80B80019998
:10D61000884500F09F806770019921704946C4F8E1
:10D62000A312002800F07F80D4F8A712D4F80200DB
:10D6300000F0FBFB8346D4F8AF0244F6206AD345E2
:10D6400040D25844C4F8AF0204EB8800D0F88712E7
:10D650005944C0F88712E07A04EB8000D0F86F12CA
:10D6600000EE101AE17AD0F8C022D4F8BC0204EB24
:10D67000810101F26F21D4EDAE0A002A03D110EE30
:10D68000902A0A6015E001EE102AB8EEC11A21EEC8
:10D69000000A01EE100AB8EEC11A01EE200A821843
:10D6A00000EE902AF8EEE00A80EE200A10EE102A32
:10D6B0000A60E17A04EB8101D1F8C0228018C1F838
:10D6C000C00215E083444846C4F8AF021822014660
:10D6D00004F28720F6F7F4FF1822494604F26F207F
:10D6E000F6F7EEFF1822494604F53070F6F7E8FF2A
:10D6F000D4F8AF02504501D300F082FC94F85F02E9
:10D70000002810D0E07A8DF80C0094EDAE0A00F0FD
:10D7100041FC8DF80D005A4603A903A800F01CFC3B
:10D72000484684F85F02D4F80200C4F8A7024846CD
:10D7300084F8620284F867724FF00109484602904B
:10D74000FFB200EE107AB8EE400A84EDAE0AC4F8DB
:10D75000BC024DE0D4F8A3127118C4F8A312D4F897
:10D76000BC22521CC4F8BC22FFB200EE107AB8EE04
:10D77000400A022A02DA84EDAE0A16E0531E00EED9
:10D78000903AF8EEE00A01EE102AB8EEC11AC0EEA7
:10D79000810A94EDAE1A20EE811AF7EE001A71EEAE
:10D7A000E00A00EE801A84EDAE1A94F86722BA42BD
:10D7B00006D0677084F867724FF001094A460292FA
:10D7C000227B63789A4213D12278904510D144F697
:10D7D000206A51450AD3002806D094F85F02002839
:10D7E00002D1012084F85F02C4F8A3A24FF000091F
:10D7F00094F86A02002808D0B9F1000F05D14FF063
:10D800000109C00701D548460290A07D400713D505
:10D81000D4F80270D4F8AB12384600F006FBD4F806
:10D820009F12884202D22878002805D04FF00109C3
:10D8300048460890C4F8AB72B9F1000F00F00581BA
:10D84000002744F6206A28E0401D80B20246424587
:10D85000FAD3A86890F81906002811D094F9560256
:10D8600001280DDB00290BD0B8F1000F08D042468B
:10D8700004F130010120F4F758F80020E860286135
:10D8800004F12B00A11D0522FCF7E0FC002084F828
:10D890006602A4F86B0228707F1C032F80F2D580EB
:10D8A000A07D3841C007F7D594F86A0240FA07F125
:10D8B000C90701D40028EFD1002F03D0022F21D0B7
:10D8C0000CD3E9E76868407A0028E5D1029800287F
:10D8D000E2D00021012000F029FADDE7D4F817009A
:10D8E0000199C840C007D7D560780028D4D094F8F3
:10D8F00062020028D0D1012084F86202014600F0C3
:10D9000015FAC9E70898002802D128780028C3D062
:10D91000D4F80280D4F8A712404600F086FA814677
:10D92000D4F8AF0200EB090BD1450FD3D9462078CC
:10D930008DF80C0094EDAE0A00F02CFB8DF80D0074
:10D940004A4603A903A800F007FB5FE0D34506D3CE
:10D950005A4604F10B01204600F0FEFA56E0297801
:10D96000012947D194F86612002943D14844C4F8EC
:10D97000AF02E07A04EB8000D0F887124944C0F887
:10D980008712E07A04EB8000D0F86F1200EE101AD4
:10D99000E17AD0F8C022D4F8BC0204EB810101F294
:10D9A0006F21D4EDAE0A002A03D110EE902A0A604E
:10D9B00015E001EE102AB8EEC11A21EE000A01EEC0
:10D9C000100AB8EEC11A01EE200A821800EE902A61
:10D9D000F8EEE00A80EE200A10EE102A0A60E17AE2
:10D9E00004EB8101D1F8C0228018C1F8C00200F018
:10D9F00007FB0BE0A8EB0B010DF1190000F02EFA6C
:10DA0000A01D0DF119010522FCF720FCB4F86B8272
:10DA1000A8F1090004F090FBDFF87827DFF87837E9
:10DA2000FDF77CFF08F0C0FB80B2014694F8662247
:10DA3000914201D084F8660294F8661284F8381096
:10DA4000012084F86102092000E7A07D00075ED56F
:10DA5000D4F82300410000990DD5012905D1800794
:10DA60000FD501208DF818000BE001208DF818006B
:10DA70001E20009005E0C840C00702D501208DF8A7
:10DA800018009DF8180001283AD194F86D0200287A
:10DA900094F86E02009929D1884223D0084694F860
:10DAA000B712884205D0C4F8B362009884F8B70270
:10DAB00004E0D4F8B3023018C4F8B302D4F8B302C7
:10DAC000D4F82710884222D30321012000F02EF938
:10DAD0000020C4F8B302012084F86D02009884F895
:10DAE0006E0214E00020C4F8B30210E088420ED0A9
:10DAF000002084F8B70284F86D02C4F8B30206E08F
:10DB0000002084F86E0284F8B702C4F8B3023046ED
:10DB100000F0C0FA04F10B0021460B22FCF796FB43
:10DB2000002084F86A0201200DB0BDE8F08F2DE9D5
:10DB3000F04383B00546002700A83B461C4618C0AA
:10DB4000DFF8584604F2612694F86102002803D0F9
:10DB5000184684F8610270817089002836D104F279
:10DB60002B0094F82B304FF4616C90F801E0CEEB71
:10DB70000E184FEA880E1CFB03E3807818184FF448
:10DB80007A73B4F82EC003FB00C004F22E034FF0EA
:10DB9000010C83F802C083F803C04FF01A0C83F81D
:10DBA00004C04FF0040C83F805C04FEA106C83F8F2
:10DBB00006C04FEA104C83F807C04FEA102C83F8D8
:10DBC00008C058727079987209207081002A02D0BA
:10DBD000022A1FD057D228788DF8000000A86A7852
:10DBE00042700A0C82700A0A8DF803200171052226
:10DBF00000A9708900193030F5F788FF7089401D41
:10DC000070812878B0706878F0707079401C7071FD
:10DC1000012738E0708900EB040808F12C025378E2
:10DC200092F802C04FEA0C2C0CEB0343D2789A18FE
:10DC300001EB020998F82C306D789D4213D06943AE
:10DC400003FB021100EE101AB8EE400A00EE909AA3
:10DC5000F8EE600A80EE200A001990F82B0000F020
:10DC600099F988F82C00708900194FEA194180F859
:10DC70002D10708900194FEA192180F82E10708933
:10DC8000001980F82F90D4F80200C4F8A7020020F1
:10DC9000C4F8AF023846BDE8FE83DFF8000590F80F
:10DCA0006112002904D0002180F861120120704720
:10DCB0000020704710B5684CF5F7AAFCA060F5F796
:10DCC00084FF6060A068DFF8D814C0F83C1600F24A
:10DCD0003C60DFF8D0144160DFF8CC1481600FF2B3
:10DCE0001101C1600FF281010161012010BD00002E
:10DCF00000205949896891F81916002915D0014664
:10DD0000DFF8983400E0491CC9B20A46052A05DA52
:10DD1000D21892F95422012AF5DB0120002801D102
:10DD200000207047184690F968027047DFF86C24AD
:10DD300002F515731875002813D00846042805DA73
:10DD4000801890F9540201280DDB03E092F9540287
:10DD5000012808DB587C012202FA01F108435874BB
:10DD600070470020587470477CB5002340F2491278
:10DD70000C7812FB0404012525700C7812FB0404B6
:10DD80001A25A570DFF8144494F865520B26354225
:10DD900014D00B7812FB030301255D7094F86532F3
:10DDA000DD0603D503F0EF0384F865320B7812FB30
:10DDB000030394F86552DD70012313E0ED0611D5DD
:10DDC0000B7812FB030303255D700B7812FB030332
:10DDD00001259D720B7812FB0303DD70002384F88C
:10DDE00069322B46002B12D00B7812FB0303D4F8B8
:10DDF00002505D600B7812FB030325781D720B78CF
:10DE000012FB0300627842720878401C08700021FF
:10DE10000846FFF78BFF94F86902012804D104211A
:10DE20000120BDE87C4081E773BD10B40022884228
:10DE300001D3421A08E00B1ADFF87043A34203D360
:10DE4000DFF86C231018421A104610BC704700000F
:10DE5000AC2901204CAA00202C5401202DE9F041CE
:10DE60002DED028B82B007460E46304604F06EF967
:10DE700041EC180B53EC182BCE48CF49FDF74EFD63
:10DE800008F092F98DF800004FF4616853EC182BFC
:10DE9000CA48CB49FDF742FD04460D469DF80000F7
:10DEA00018FB00F004F048F902460B4620462946CC
:10DEB00008F0BAF841EC180B53EC182B4FF0113066
:10DEC000C049FDF72BFD08F06FF904468DF80140BD
:10DED0003C25E4B215FB04F004F02EF902460B4693
:10DEE00051EC180B08F0A0F808F05EF98DF802006C
:10DEF0009DF8001011FB08F114FB051151FA80F098
:10DF00004FF47A7101FB1060ADF80300384600A9A8
:10DF10000522FCF79BF902B0BDEC028BBDE8F08155
:10DF20009E4981F86902887D052210420FD091F840
:10DF30006902012802D104210120F7E6022803D159
:10DF40008E48012101707047002081F869027047F6
:10DF500092490B22FCF77AB93CB40B4611468F4A22
:10DF600002F26324E478002C04D092F863221D7836
:10DF7000AA4203D0002202B030BCD8E5002C06D063
:10DF8000AA4204D10222184602B030BCCFE533BC0D
:10DF9000704700000021F6EE000AB7EE081A0428C8
:10DFA00003D1DFED770A9FED771AB4EE600AF1EE48
:10DFB00010FA07D4B4EE401AF1EE10FA01D502219E
:10DFC00000E001210846704738B50446002500A846
:10DFD0000AF00AF871489DF80010012909D1D0F81B
:10DFE000D8126118C0F8D8127748814204D30125AD
:10DFF00002E02946C0F8D812284632BD804F1200F0
:10E000003EB50020654C04F287256968D4F8872264
:10E01000914200D30120022109E0D2F8872204EBCB
:10E020008303D3F887329A4200D20846491C04EB96
:10E030008002C9B20B46062BEFDB8DF80000D2F848
:10E040006F0200EE100A9DF80000FFF7A3FF8DF8A5
:10E050000100AA6A00A900A8FFF77EFF182200218C
:10E0600004F28720F6F72CFB1822002104F26F201F
:10E07000F6F726FB1822002104F53070F6F720FB96
:10E080000020A86237BD5148002213460260436059
:10E090007047000038B52DED028B98B008EE100ADD
:10E0A00000A809F05AFABDF80000484C022801D037
:10E0B00003281CD102A809F046FA20686168444D83
:10E0C000F6F708FB00EE100ADDED100A95ED001AD8
:10E0D00070EEC10A9FED2C1A00EE810A10EE100AB4
:10E0E0000CF000F8206061601098286030E004288F
:10E0F00016D120686168F6F7EDFA00EE100AF8EE26
:10E10000480A9FED221A60EE810A9FED1F1A00EE69
:10E11000810A10EE100A0BF0E5FF2060616017E045
:10E12000052815D120686168F6F7D4FA00EE100AC8
:10E13000F8EE480A9FED161A60EE810A9FED121A5A
:10E1400000EE810A10EE100A0BF0CCFF2060616037
:10E15000226863681F485D218B420BD301D882423D
:10E1600008D3206861681C4A6FF05D03801859412C
:10E170002060616018B0BDEC028B31BD2C540120D1
:10E180009A99993E3333333F0000C8421CEBE23C7E
:10E19000C6DC353C9A9999999999C93FAC290120D7
:10E1A000A5D10008A3D300081DD50008A1780F054C
:10E1B000005C2605B9791F962FA4923EFCA9F1D2E6
:10E1C0004D62503F1111913F20BF0200882C012069
:10E1D0005C56012000A0DB21006024DE41542D4666
:10E1E0004F5243454452454D4F56454400000000B0
:10E1F00041542D524C204E756C6C0000534C4D20F8
:10E2000041542D43757253543A256420256400000F
:10E2100080B5B048C16891F85516002901D1002099
:10E2200002BD012101710CF0C7F800280AD00DF0E1
:10E23000BCF801460FF2FC20F5F730FD0CF0C0F8F9
:10E24000012002BD002002BD0FB400B597B00BF055
:10E250006DFFA04800218170C17001714170BDF84F
:10E26000620000F01FF9BDF8640000F019F9012008
:10E270008DF86400AA208DF862003C208DF86300C0
:10E2800000208DF8000003208DF801000DF103003F
:10E2900018A95522FBF7DAFF0A208DF8020000A822
:10E2A000F5F7B6FA002805D10FF29C20F5F7F6FC39
:10E2B000022000E0012017B05DF814FB00B597B014
:10E2C0000BF0D2FF01208DF8000003208DF8010033
:10E2D0000A208DF8020000A8F5F79AFA002801D16B
:10E2E000032000E0012017B000BD70B504460D46C4
:10E2F00040F24916287816FB0040012101700DF00C
:10E3000054F801281AD1287816FB004005214170E5
:10E31000287816FB00401B2181700FF24020F5F792
:10E32000BDFC287816FB00400221C170287816FB3E
:10E3300000401E2141710CF053F818E00DF039F83F
:10E34000012814D1287816FB00400121417028785B
:10E3500016FB00401B2181700FF21020F5F79EFC88
:10E36000287816FB00400121C1700CF049F828788C
:10E37000401C2870BDE870400CF022B870B5A0B009
:10E38000554E304609F0DFF814A8FFF7E1FD30687C
:10E39000504C2169411A89B2002904D12278B6F87B
:10E3A0004A309A4203D02061B6F84A002070E068F3
:10E3B000D0F858563160A068807AC046C0469DF8B3
:10E3C00050001390314683B068465822FBF74EFF49
:10E3D0000EBCADB228460DF0E1FC6070A0780128BB
:10E3E0001DD117A8F6F7B4F81BA80268436843ECE0
:10E3F000122B19A80268436843EC112B17A8026876
:10E40000436843EC102B0DF17500837A82784178D4
:10E410009DF8750000F02DF80020A07006E0E0786F
:10E42000012803D100F03AF80020E070012020B06C
:10E4300070BD10B5274CF5F7C8FBA060F5F7E8F8FC
:10E44000E060F5F7C2FBA0600020206120700BF0B7
:10E45000EAFEE0682149C0F8781600F278602049A9
:10E460004160204981602049C1602049016101204B
:10E4700010BD80B5DBB2D2B2C9B2C0B20BF0ECFFB6
:10E48000002803D0BDE801400BF0CABF0FF2EC003A
:10E49000F5F704FCBDE801400BF0CDBF0BF0CBBF9E
:10E4A0000BF004BF0BF0F1BE0BF012BF0BF028BF56
:10E4B00080B50CF07AFF002805D0064800790028C6
:10E4C00001D1012002BD002002BD0248012181705E
:10E4D000704700007C540120D44D012049E200081F
:10E4E000BDE200087DE3000811E20008EBE200084D
:10E4F00080B50DF028FC0FF29400BDE80240F5F75E
:10E50000CDBB0CF091BF0CF095BFC9B20CF0A6BF0B
:10E510000BF066BF0BF0B8BE80B50DF08DF8C0B241
:10E5200002BD80B50DF062F8C0B202BD0DF0E0BBD7
:10E530000DF0DFBB4C5420436D6452656164795F1C
:10E5400053532025640000004C54205065646F4FE5
:10E5500070656E4661696C20535300004C54205224
:10E5600045515545535420504F5300004C542052B0
:10E570004551554553542041434B00004C542050C5
:10E580004F4E4F5420444953540000005353203AF7
:10E590002043656C6C4368616E676564204E6F74E0
:10E5A0006900000070B50024FFF777FB0646DFF82E
:10E5B000B458FFF77DFF012805D1287940F001000C
:10E5C00028710A202872F6B2002E0CD0FFF7A4FFA3
:10E5D000002823D00FF6C000F5F760FB287940F043
:10E5E000020028711AE0FFF7A3FF064628780028EA
:10E5F00000D12E702878864210D03046012806D1EE
:10E60000FFF78AFF287940F00200287105E0022810
:10E6100003D1287940F0020028712E702879002853
:10E6200000D00124E86890F8CD06002800D100242D
:10E63000204670BD0FB400B597B0DFF82808002160
:10E64000017001214171C06890F8CC16002946D1B3
:10E6500090F8CD06002842D100208DF800001B2044
:10E660008DF801000DF1030018A95522FBF7EEFD0E
:10E670000A208DF8020000A8F5F7CAF8002805D195
:10E680000FF62000F5F70AFB022029E002208DF8A2
:10E6900062004FF49660ADF868000020CDF863008A
:10E6A0008DF867008DF800001A208DF801000DF13B
:10E6B000030018A95522FBF7C9FD0A208DF80200B6
:10E6C00000A8F5F7A5F8002805D10FF2E870F5F7D6
:10E6D000E5FA022004E04FF49660FFF71BFF0120EB
:10E6E00017B05DF814FB00B597B00FF2D870F5F7CE
:10E6F000D5FA01208DF800001B208DF801000A20BA
:10E700008DF8020000A8F5F783F8002801D1032056
:10E710001AE001208DF800001A208DF801000A206F
:10E720008DF8020002208DF805000020ADF80B00E6
:10E73000CDF806008DF80A0000A8F5F769F8002862
:10E7400001D1032000E0012017B000BD2DE9F84FF2
:10E750002DED028B92B004460D4640F24916287802
:10E7600016FB004001210170DFF8F8A69AF80400BA
:10E77000810740F1B580287816FB004001214170E7
:10E78000287816FB00401D218170287816FB004078
:10E7900000214171FFF7C5FE002805D0FFF7B1FE4B
:10E7A00083465FFA8BFB01E04FF0000B287816FBE5
:10E7B000004080F807B04FF0000879E0414601A81A
:10E7C000FFF7A3FEFFF7B4FE814649460FF2FC6057
:10E7D000F5F764FAC8EB48170DF12D00297816FB00
:10E7E000014179189DF82D204FF4616390F801C024
:10E7F000CCEB0C1E4FEA8E0C13FB02C28078101873
:10E800004FF47A72BDF9303002FB0030C1F81B00C2
:10E810009FED998B287816FB00403818009001A8CE
:10E820000268436851EC180BFDF778F807F0BCFC60
:10E830000099C1F80B00287816FB004038180090AA
:10E8400003A80268436851EC180BFDF767F807F05E
:10E85000ABFC0099C1F80F00287816FB004038186F
:10E86000009005A8026843680020DFF8FC15FDF75A
:10E8700055F807F099FC0099C1F81300287816FBA9
:10E8800000403818DDF83E10C0F81F10287816FB3D
:10E8900000403818BDF84410A0F81910287816FB6D
:10E8A00000403818C0F8239008F101085FFA88F892
:10E8B000D84583DBFFF727FE287816FB00400521AB
:10E8C000A0F84311287816FB00400AF13801C0F87F
:10E8D00045119AF8040080F002008AF8040027E04D
:10E8E000C00725D5287816FB0040052141702878FF
:10E8F00016FB00401D218170287816FB0040012185
:10E900004171287816FB00409AF808108171FFF7D2
:10E91000FFFD9AF8040080F001008AF8040000204E
:10E92000CAF81000FF2000F08AFA0020CAF82C0074
:10E930002878401C287012B0BDEC028BBDE8F18F26
:10E9400010B584B000A8FFF703FBDFF82045204690
:10E9500000A90B22FBF77AFC61782078FFF7E6FD2F
:10E9600000F08EF8012004B010BD38B5F4F750FE69
:10E970000446DFF8F054EC6000F054F8DFF8F004DF
:10E98000C4F8F00604F2F060DFF8E8144160DFF844
:10E99000E8148160DFF8E414C160DFF8E414016179
:10E9A0000522002105F13800F5F78AFE012032BD6D
:10E9B00010B5044621460FF22C50F5F76FF92046AA
:10E9C000BDE81040FFF76CBDFFF76CBD10B5044605
:10E9D00021460FF21C50F5F761F92046BDE81040C2
:10E9E000FFF764BD10B5044621460FF21450F5F749
:10E9F00055F92046BDE81040FFF756BD10B58AB066
:10EA0000DFF8604400206063E079012808D100A8A5
:10EA1000F5F79EFD9DF82300012801D10020E0714B
:10EA20000AB010BD10B5DFF83C4400202071206111
:10EA3000A061E06160616070A070E0704FF4FA70F6
:10EA40002062DFF840046062DFF83C04A0625822D4
:10EA50000021DFF83804F5F733FE58220021DFF8F3
:10EA60003004F5F72DFE0020607160632063E071D3
:10EA7000A0710A20207210BD0000000080842E4189
:10EA80002DE9FE4F0024DFF8DC53E868D0F8D0967B
:10EA9000DFF8F863DFF8F873386800280BD13068C6
:10EAA000002808D1384608F04EFD30463946582235
:10EAB000FBF7DCFB02E0384608F045FDDFF8D483C5
:10EAC00008F10C00B8E80E000EC0A8F10C0800A870
:10EAD000FFF73EFA404600A90B22FBF7B7FB98F878
:10EAE0000100E87098F80000012806D0022804D040
:10EAF000032802D0042088F8000098F8001098F845
:10EB00000C00814204D0A9700FF20040F5F7C6F85E
:10EB1000E86A39683268891A10FA81FBC5F82CB0A6
:10EB200028696FF00F01884201D248442861686B60
:10EB3000884201D24844686395F807A0BAF1010FF2
:10EB400005D1286B884204D24844286301E020465E
:10EB500028636878002800F0CA80022801D05BD3BF
:10EB600013E195F80280B8F1040F16D1052000F0EA
:10EB700066F9686948446861696A8842C0F005813D
:10EB8000FF2000F05CF90120E871A8712A69414674
:10EB90000FF29030F5F782F8F7E0B8F1020F02D0EB
:10EBA000B8F1030F19D1042000F049F9A86909EB65
:10EBB0000003AB6142F211708342C0F0E6802A6923
:10EBC00041460FF27430F5F769F8FF2000F037F98D
:10EBD0000120E871A8716870D7E0B8F1010F40F02A
:10EBE000D480E86909EB0003EB6168694844686117
:10EBF0004EF661208342C0F0C8802A6941460FF278
:10EC00005030F5F74BF8FF2000F019F90120E871BA
:10EC1000A87120466870B8E095F80280B8F1020F3C
:10EC200002D0B8F1030F15D1062000F008F9286AC8
:10EC30008345C0F0AA805B462A6941460FF228301E
:10EC4000F5F72CF8FF2000F0FAF80120E871A87120
:10EC500068709AE0B8F1040F2FD1042000F0EFF8AB
:10EC6000686909EB00036B61E878002801D001288E
:10EC700013D142F211708342C0F087802A69414665
:10EC80000FF2FC20F5F70AF8FF2000F0D8F8012079
:10EC9000E871A8710220687077E0FF2000F0CFF8DB
:10ECA0000120E871A8716B692A6941460FF2E820DA
:10ECB000F4F7F4FF0220687067E0B8F1010F64D147
:10ECC000E86909EB0003EB614EF6612083425CD3F7
:10ECD0002A6941460FF2D820F4F7E0FFFF2000F048
:10ECE000AEF80120E871A871204668704DE004205C
:10ECF00000F0A5F895F80280B8F1020F02D0B8F143
:10ED0000030F17D1A8694844A861022000F097F8C2
:10ED1000AA6941F28930824237D341460FF2A820D6
:10ED2000F4F7BCFFFF2000F08AF80120E871A87119
:10ED300068702AE0B8F1040F27D1686909EB000375
:10ED40006B61E878002801D001280DD14EF66120D2
:10ED500083421AD3BAF1000F0FD12A6941460FF24C
:10ED60007C20F4F79BFF08E0BAF1000F05D12A6977
:10ED700041460FF28020F4F791FFFF2000F05FF88A
:10ED80000120E871A871022068706879012809D112
:10ED90002046687101242046A87001460FF26C20BD
:10EDA000F4F77CFFA87901280CD1686BA96A884226
:10EDB00008D301240020E8712863A9780FF26020AD
:10EDC000F4F76CFFE87901280CD1286B2E498842B2
:10EDD00008D30020E87128630124A9780FF260208D
:10EDE000F4F75CFF012C10D1287940F00100287164
:10EDF00005202872FF2000F022F80020E8620FF2C0
:10EE00006020F4F74BFF0020A871304639465822A5
:10EE100003B0BDE8F04FFBF729BA1249086270470A
:10EE20001049486291ED090AB8EE400ADFED0C0A7C
:10EE300020EE200ABCEEC00A81ED0A0A7047C10725
:10EE400002D5084900228A61810702D505490022BE
:10EE50004A61400702D503480021C16170470000A4
:10EE60006666663F544F012000408F405C5501208C
:10EE700035E60008E7E6000841E90008A5E50008D6
:10EE80004DE70008C0270900603D0800CC4C012078
:10EE9000244D0120C05301204C5420436D64415443
:10EEA000440000004C54204F70656E206661696C10
:10EEB000000000004C54204154204F70656E2066C5
:10EEC00061696C004C542053544F50004C54204105
:10EED000502053746179696E67205374617475733F
:10EEE000202564004C542053657457542025640039
:10EEF0004C54205365745341522025640000000097
:10EF00004C54205365745352202564005B4C524589
:10EF1000515D205472616E73204D6F6465202564CD
:10EF2000000000005B4C5245515D205245512D566A
:10EF300031202564202564005B4C5245515D2052F0
:10EF400045512D563320256420256420256400007A
:10EF50005B4C5245515D205245512D56342025645D
:10EF600020256420256400005B4C5245515D2052F1
:10EF700045512D573120256420256420256400004B
:10EF80005B4C5245515D205245512D57322025642E
:10EF900020256420256400005B4C5245515D2052C1
:10EFA00045512D5733202564202564202564000019
:10EFB0005B4C5245515D205245512D5734202564FC
:10EFC00020256420256400005B4C5245515D205291
:10EFD00045512D5331202564202564005B4C52455A
:10EFE000515D205245512D53322025642025642047
:10EFF000256400005B4C5245515D205245512D5314
:10F000003320256420256420256400005B4C524594
:10F01000515D2041504453542C20256400000000D1
:10F020005B4C5245515D20466F726365642072658A
:10F030007175657374322121212025640000000060
:10F040005B4C5245515D20466F726365642072656A
:10F050007175657374312121212025640000000041
:10F060005B4C5245515D2052657365740000000091
:10F070000FB410B5DFF83C4500206081082201463E
:10F08000F4F7C8FA08220B210020F4F7C3FA02288B
:10F0900001D102200EE000202070E0806070A0818D
:10F0A0001E206071002020616061A061A070E0708E
:10F0B0002071012010BC5DF814FB80B5DFF8F4046A
:10F0C00000210170418190F90100002804D108223B
:10F0D0000B210120F4F79EFA082200210120F4F709
:10F0E00099FA012002BD000070B52DED028BA6B08B
:10F0F000012413A8F4F7EDFADFF8B85495F901608C
:10F10000002E05D0022E2ED009D3032E51D075E04B
:10F110001398009014980190159802906EE09DED60
:10F12000140A8DED010ADDED150ACDED020A9FED01
:10F13000561A00EE401A00EEE01AB5EE401AF1EE53
:10F1400010FA0DDD11EE100AFCF7C0FB41EC100BBC
:10F1500007F0DCFC51EC100BFCF7B2FC00904DE02A
:10F16000002000904AE013980090DDED150ACDEDE7
:10F17000020A9DED130ADDED131A9FED431A00EE0E
:10F18000611A00EEE01AB5EE401AF1EE10FA0DDD4C
:10F1900011EE100AFCF79AFB41EC100B07F0B6FCDD
:10F1A00051EC100BFCF78CFC019027E00020019043
:10F1B00024E0139800909DED140A8DED010A9FED57
:10F1C000321A00EE401A9DED130ADDED130A00EE2F
:10F1D000601AB5EE401AF1EE10FA0DDD11EE100ACC
:10F1E000FCF774FB41EC100B07F090FC51EC100B9A
:10F1F000FCF766FC029001E000200290B5F90A00DD
:10F20000012801D120460BE195F90000002871D1B9
:10F210002889401C288195F905104A1C00B28242B9
:10F2200037DB1398FCF752FB21F000414FF02042EE
:10F23000DFF8843306F062FE03D8A878401CA8707B
:10F2400001E00020A8701498FCF740FB21F0004179
:10F250004FF02042D84B06F051FE03D8E878401C0E
:10F26000E87001E00020E8701598FCF72FFB21F012
:10F2700000414FF02042D04B06F040FE06D82879DE
:10F28000401C2871CBE000BF3D57C04200202871D0
:10F29000C5E095F90200884202DB204668700FE065
:10F2A00095F90300884202DB0220687008E095F9B6
:10F2B0000400884202DB0320687001E000206870CF
:10F2C00095F90100002808D008220B212046F4F708
:10F2D000A1F9032801D10220A2E095F901100FF253
:10F2E0002430F4F7DBFC20462870002028810DF044
:10F2F00045FB94E001283AD1E888401CE88030467C
:10F3000000A991EC030A0DF03DFB002817D00098EE
:10F310002861019868610298A86195F901000028A8
:10F320000AD1082200212046F4F774F9032800D1FD
:10F3300003240220287072E0032028706FE0B5F9E2
:10F34000060064286BDB0020E88000F003F995F9E3
:10F350000100002804D108220B212046F4F75AF9B5
:10F36000052028700FF2AC20F4F798FC57E0032832
:10F3700055D1002E5DD12889401C288100B2652816
:10F3800052DA95ED040ADDED000A30EE600A10EE67
:10F39000100AFCF79BFA21F00041FCF791FB08EE04
:10F3A000100A95ED050ADDED010A30EE600A10EE57
:10F3B000100AFCF78BFA21F00041FCF781FB08EE04
:10F3C000900A95ED060ADDED020A30EE600A10EEB5
:10F3D000100AFCF77BFA21F00041FCF771FB00EE0C
:10F3E000100ADFED720AB4EE608AF1EE10FA04DA68
:10F3F000F4EE608AF1EE10FA06DBDFED6D0AB4EE92
:10F40000600AF1EE10FA57DA0020A881B5F90C0075
:10F41000052804DB04202870204600F08CF82046E4
:10F4200026B0BDEC028B70BD002028812870A88119
:10F43000F5E795ED040ADDED000A30EE600A10EE06
:10F44000100AFCF743FA21F00041FCF739FB08EE03
:10F45000100A95ED050ADDED010A30EE600A10EEA6
:10F46000100AFCF733FA21F00041FCF729FB08EE03
:10F47000900A95ED060ADDED020A30EE600A10EE04
:10F48000100AFCF723FA21F00041FCF719FB00EE0B
:10F49000100ADFED460AB4EE608AF1EE10FA04DAE3
:10F4A000F4EE608AF1EE10FAAEDBDFED410AB4EE65
:10F4B000600AF1EE10FAA7DBA889401CA881A5E735
:10F4C00080B5F4F7A5F83B49C8613C49C0F804127F
:10F4D00000F501703A4941603A4981600FF20D012F
:10F4E000C1600FF2E9010161012002BD38B50024BD
:10F4F000304DE96991F8E111002901D1204632BD72
:10F50000012802D100F013F80446012C07D100F0C5
:10F5100021F80120688108220B21F4F77BF82046AE
:10F5200032BD80B5002000F006F8012002BD26485B
:10F5300090F90000704724490870704780B5082290
:10F5400000210846F4F766F8022801D1022002BD26
:10F55000012002BD80B5174800210181C180082229
:10F560000120F4F757F8032801D1032002BD012040
:10F5700002BD38B501240F4D95F90000022812D1C3
:10F58000FFF7DCFF022805D10FF29400F4F786FBA9
:10F59000022032BD032800D10324032028700FF27B
:10F5A0008C00F4F77BFB204632BD000001002040B8
:10F5B0000100404064A900209999274071F000089B
:10F5C000BBF00008E9F00008ED56012018B440F245
:10F5D00049120B7812FB030301241C700B7812FBF9
:10F5E00003035C700B7812FB030308249C700B78F8
:10F5F00012FB03000122C2700878401C087011BC85
:10F600008FE7000053535020534D41204D6F6465E8
:10F610002025640053535020534D41204E46000096
:10F62000534D20414420464C00000000494E5620D6
:10F63000534149000FB480B57F4801210170052274
:10F6400000210846F3F7E6FF022801D102200DE071
:10F65000052207210020F3F7DDFF022801D1022057
:10F6600004E000F0E1F80DF051FA012002BC5DF871
:10F6700014FB38B50124052207212046F3F7CAFF01
:10F68000032800D103246C4D95F90000032801D014
:10F69000012807D1052200210120F3F7BBFF032831
:10F6A00000D103240020287000F0BEF80DF0D9FA34
:10F6B000204632BD80B5002000F03DF8022801D17F
:10F6C000022002BD032801D1032002BD012002BD9A
:10F6D00010B5594CF3F79CFF2061F3F7ABF9A0602C
:10F6E000F4F773FAE06020695449C0F8501100F54E
:10F6F000A87053494160534981600FF21101C16004
:10F700000FF249110161012010BD000001460020E7
:10F71000494A126992F82D21002A02D0012900D10C
:10F7200002E07047002003E0474890F9000070476E
:10F7300045490870704770B582B0064601253E4CB9
:10F7400094F90000012823D1A088401CA08000B2B9
:10F750004C280BDB0020A080022020700522002115
:10F760002846F3F757FF032800D10325012E59D16E
:10F77000E068007E012807D1B4F904001F2851DB9E
:10F780006078401C60704DE0A078401CA07049E09B
:10F7900002281CD1012E0AD1E068007E012803D185
:10F7A0006078401C607002E0A078401CA07094F962
:10F7B0000100012836DB052200210846F3F72AFF65
:10F7C000022801D1022076BD032020702AE0032800
:10F7D00028D100208DF8000000A9A0680DF0BAF92A
:10F7E000C0B202280DD1052200212846F3F712FFEE
:10F7F000032800D103250120FFF79AFF0420207081
:10F8000010E003280ED1052200212846F3F702FF5D
:10F81000032800D1032500206070A0700220207012
:10F820000DF074F9284676BD0348002181804170AF
:10F8300081707047000000005454012035F6000824
:10F8400073F60008B5F60008DE56012010B50C4628
:10F8500040F24911227811FB020201231370227831
:10F8600011FB02025370227811FB020205239370F0
:10F87000227811FB02000121C170FFF753FF2078AD
:10F88000401C207010BD00000FB480B50222012181
:10F890000020F3F7BFFE022801D102200EE0022271
:10F8A00007210020F3F7B6FE022801D1022005E06F
:10F8B0000DF0E8F94C4800210170012002BC5DF810
:10F8C00014FB80B5022201210846F3F7A3FE0328AA
:10F8D00001D1032002BD022207210120F3F79AFE85
:10F8E000032801D1032002BD3F48002101700120FF
:10F8F00002BD00B593B000A8F3F7EBFE03A890ECAF
:10F90000030A0DF0F5F938490870012013B000BD65
:10F9100010B5354CF3F77CFEA060F4F756F9606043
:10F92000A0683249C0F89C109C303149416031498F
:10F9300081600FF22101C1600FF2690101610120B4
:10F9400010BD80B528484068007E0DF0CAF901203E
:10F9500002BD0000002024498A6892F87920002A1C
:10F9600004D091F90010002900D0012070471E48F2
:10F97000002101700120704710B50024012804D037
:10F9800007D303280BD002D303E0012407E00224AD
:10F9900005E0032401460FF26000F4F77FF92046EA
:10F9A00010BD000038B50C4640F24911227811FB19
:10F9B000020201231370227811FB02025370227895
:10F9C00011FB020202239370227811FB0205064804
:10F9D00090F90000FFF7D0FFE8702078401C2070FD
:10F9E000BDE83140C3E700004455012089F8000814
:10F9F000C3F80008F3F800084C4D43505320312061
:10FA0000256400000FB410B5B14CB248C069E06085
:10FA10009DF80A10A1619DF80B20E2619DF80C3061
:10FA200023620FF2D020F4F739F92F220021084683
:10FA3000F3F7F0FD022805D10FF2CC20F4F72EF9F0
:10FA4000022020E02F2207210020F3F7E3FD022807
:10FA500005D10FF2BC20F4F721F9022013E00EF0DB
:10FA600003F80C2200212046F4F72AFE4FF0FF3065
:10FA7000E0622063E068407A022803DB00F0D0F8FF
:10FA8000E06A6060012010BC5DF814FB80B50FF2E5
:10FA90008820F4F703F92F2200210120F3F7BAFDA3
:10FAA000022805D10FF27C20F4F7F8F8022002BDFD
:10FAB0002F2207210120F3F7ADFD022805D10FF217
:10FAC0006C20F4F7EBF8022002BD012002BD804853
:10FAD00000218160C1698269012A2BD1002903D0EC
:10FAE00002291BD009D37047016805294DD0416810
:10FAF00002294AD10121816070470168026A012A06
:10FB000007D1052941D0416802293ED101218160F8
:10FB10007047052939D0012181607047016A0129A8
:10FB200033D10168052930D0416802292DD1012146
:10FB300081607047002903D0022916D009D370478D
:10FB40000168052902D0416802291ED10121816086
:10FB50007047016A012918D10168052902D041685E
:10FB6000022912D10121816070470168026A012ACD
:10FB700007D1052902D04168022906D101218160FF
:10FB80007047052901D101218160704730B593B0DC
:10FB900000A8F3F79EFD00A890EC030A0DF06FFF9C
:10FBA0004B4C606A401C6062032806DB03200DF0AA
:10FBB00083FF010001D021632060E06A10F1010F92
:10FBC00011D0206B10F1010F0DD0A56A002D04D1CA
:10FBD000FFF77DFF012000F04AF8681CA0620328AF
:10FBE00001DB0020A062012013B030BD10B5384CFD
:10FBF000F3F70EFD6061F3F7E8FF206160693649B5
:10FC0000C0F8281B00F6283034494160344981602F
:10FC10000FF23501C1600FF25D010161012010BDDD
:10FC200010B52B4C2069007EE062002802D1012033
:10FC3000606001E002206060FFF749FF012000F0F2
:10FC400016F80120606210BD2148406990F8050B4C
:10FC5000002801D10020704705E080B5002000F0A9
:10FC600006F8012002BD1F4890F9000070471D49A9
:10FC7000087070473CB440F249120B7812FB030342
:10FC800001241C700B7812FB03035C700B7812FBD1
:10FC900003032F249C700E4B0C7812FB04049D6808
:10FCA00025720C7812FB04041D6825710C7812FB78
:10FCB00004005A6842710878401C087033BCCCE7D5
:10FCC0000349086201460FF26C00F3F7E7BF00003A
:10FCD000DCA80020AC49012005FA00088DFA0008D4
:10FCE0008DFB0008E956012001460FF25800F3F79A
:10FCF000D5BF000050533A5245472825642C25644F
:10FD00002C2564290000000050532D414F45000070
:10FD100050532D504F45000053414E473A554E52D7
:10FD20004547000050532D414345000050532D508E
:10FD30004345000053414E473A5345542825642912
:10FD40000000000053414E473A43616C6C5F696E9E
:10FD5000666F5B25645D000080B55A490978491CCF
:10FD6000584A1170017A491E0172C9B2002901D1A5
:10FD70000DF08EFFF5F75AFF01BD38B5040052486B
:10FD800005680BE0287A002807D06868A04204D1F3
:10FD9000012028722800FFF7DFFFED68002DF1D168
:10FDA00031BD38B5040049480078002802D0A120B0
:10FDB000F5F7DCFBF5F7F9FE4348056805E0A542D9
:10FDC00002D1AF20F5F7D2FBED68002DF7D1404806
:10FDD00040490160142200212000F4F771FC6920E1
:10FDE0002074802080F3118800BF00BF364800686F
:10FDF000E0603548046033484078F021084202D082
:10FE00009920F5F7B3FB2F484078002802D1002055
:10FE100080F3118831BD38B504002C4800780028E3
:10FE200002D0A120F5F7A2FBF5F7BFFE207C6928E0
:10FE300002D08520F5F79AFB22480078401C214922
:10FE40000870207A002804D11E488068606001256F
:10FE500010E060681B498968884209D010212000A1
:10FE600001F094FA207A0028F8D116488068606082
:10FE7000207A451C2572F5F7D9FE280032BD10B551
:10FE8000040012480078002802D0A120F5F76EFB8C
:10FE9000F5F78BFE207C692802D08520F5F766FBFC
:10FEA000207A002802D19620F5F760FB60680549AA
:10FEB0008968884202D09C20F5F758FB2000FFF7A4
:10FEC0004BFF10BD28A80020B4560120FB5601208E
:10FED000C85601207BFD000800F5E07002689142E1
:10FEE00003D343689A18914202D380680028F5D161
:10FEF0007047DFF82007016899B94FF480318160BD
:10FF000004224FF4805141604FF0FF31C160016124
:10FF100004214161DFF80017C1F8BC21DFF8FC16AD
:10FF200001600120704701F1080313F0070305D0B9
:10FF300001F10803C3F1080303F007035918D21AAB
:10FF40008161C26042F001034B60511828224A606F
:10FF5000DFF8C0160969C16170472DE9F84F044602
:10FF600001F1080010F0070005D001F10800C0F110
:10FF7000080000F0070000EB010B02F1080010F090
:10FF8000070005D002F10800C0F1080000F00700EA
:10FF90008618A6EB0B00A0EB030803EB0B0743F05E
:10FFA0000300CBF80400B74228BF0DF093FE307970
:10FFB000C00758BF0DF08EFEB8F1100F38BF0DF01E
:10FFC00089FEA069864207D1E0684044E060A761ED
:10FFD00040F0010078605AE16069864208D1A0686B
:10FFE0004044A060676140F001017960C0514EE17A
:10FFF000706800F00301012940F0AD80C0084FEAAD
:020000021000EC
:10000000C00920283BD2D6F808A0F5680090AE427F
:1000100008BF0DF05FFE564508BF0DF05BFE70682F
:100020000099C008C000B0EBC10F18BF0DF052FE20
:10003000009804EBC00000F128018A4508D021692E
:100040008A45C0F08480DAF80C10B14240F07F801D
:10005000554506D1009A20680121914088432060CF
:1000600077E02830854205D0206985426FD3A868A3
:10007000B0426CD1CAF80C50C5F808A069E0F56828
:10008000D6F818A0B5420CD0B0682169884223D3B5
:10009000C168B14204BFA968B1421DD1C560A86062
:1000A0001CE006F11400056835B906F1100005687A
:1000B000A5B101E00846056805F114010A68002AA7
:1000C00002BF05F110010A68002AF3D121698842B4
:1000D00002D30021016001E00DF0FCFDBAF1000F38
:1000E00037D0F06904EB800000F5987001688E420B
:1000F00009D10560280014D1F2696068012191409E
:100100008843606025E02069824508D3DAF8100052
:10011000B04214BFCAF81450CAF8105001E00DF0F4
:10012000D9FDB5B12069854211D3C5F818A0316950
:1001300029B1814226BF29618D610DF0CBFD706927
:1001400038B12169884202D36861856101E00DF010
:10015000C1FD4E44C84470684008400070604FEADA
:10016000D80548F00100786048F80780202D21D29A
:1001700004EBC50000F12806B146B8F1100F38BFF6
:100180000DF0A8FD206820FA05F1C90704D401216B
:10019000A9400843206006E0B068216988422CBF6E
:1001A00081460DF097FDB760C9F80C70C7F808904C
:1001B000FE606CE05FEA182008BF002123D0B0F594
:1001C000803F28BF1F211ED2A0F58071090C01F0CD
:1001D00008018840A0F58052120C02F00402904001
:1001E000A0F580431B0CC1F10E0103F00203891A34
:1001F000C91A984001EBD030C11D28FA01F101F075
:10020000010101EB4001F96100227A613A6104EBDE
:100210008100626822FA01F300F59870DB0706D4CA
:10022000012303FA01F11143616007601CE01F29FB
:1002300000680EBF00214908C1F1190108FA01F157
:1002400000E010464268D208D200424510D0CA0FE2
:1002500000EB820202F1100349001A68002AF0D173
:1002600021698B4211D31F60B861FF60BF600EE04F
:1002700022698168904228BF914206D3CF6087608F
:10028000B960F8600020B86101E00DF023FD0BF1CA
:100290000800BDE8F28F2DE9F04F0546DFF8740342
:1002A000006883B0884608B9FFF723FEDFF86403CF
:1002B000806800EB08012F31401E21EA00008045D4
:1002C00080F0A581D5F8B81141B1D5F8B0218018DA
:1002D000824280F09C818142C0F099810DF0FEFC49
:1002E00000281EBF0446076814F1010F00F08F813B
:1002F000D5F8B0013818C5F8B001D5F8B41181426D
:1003000038BF0146C5F8B411A86968BB286908B1AF
:10031000844200D22C61C5F8C041C5F8C4710020E8
:10032000C5F8CC012021BB48006868624FF0FF305F
:100330002862284600F128020830D2609260491EE7
:10034000F8D1B548854203D1A7F12802214625E01E
:1003500055F8040CC00805EBC000A0F108013819DD
:10036000401AA0F1280219E005F5E071084600E006
:100370008068B8B142680368D2189442F8D1027B11
:1003800012070FD4AA699A420CD3466833449A42A2
:1003900008D2B9194160E868A9693A182846FFF7F8
:1003A000C2FD1FE12869844238BF2C610846391913
:1003B00000E0806880B102688A42FAD1017B0907B7
:1003C0000AD40460434641687918416028462146B2
:1003D00003B0BDE8F04FC0E5AE6931462846FFF7EF
:1003E0007BFD41680068081801902F3800F1080172
:1003F00011F0070105D000F10801C1F1080101F079
:10040000070101EB000906F11000814538BFB14634
:1004100009F10800009004F1080109F1180A4FF0F1
:10042000000BA7F1280011F0070105D004F1080125
:10043000C1F1080101F007010A19401AAA61E86038
:1004400040F0010151608018282141607148006925
:10045000E861009810F0070018BF0DF03BFC1B206E
:10046000C9F8040005F5E071B1E80C500098A0E867
:100470000C50C5F8C041C5F8C471C5F8CCB100989E
:10048000C5F8C801019800E08A460722CAF804208E
:100490000AF104010A1D0BF1010B8242F4D3BBF1F6
:1004A000020FB8BF0DF016FCB14500F09B80A9EB20
:1004B000060081194FEAD0094A68520852004A6082
:1004C00040F0010171608051B9F1200F1FD205EB9E
:1004D000C90101F128042746102838BF0DF0FAFBA6
:1004E000286820FA09F1C90705D4012101FA09F1A8
:1004F0000843286006E0A068296988422CBF0746A7
:100500000DF0E8FBA660FE60B760F4606AE0010AE7
:1005100008BF002223D0B1F5803F28BF1F221ED282
:10052000A1F58072120C02F008029140A1F58053EF
:100530001B0C03F004039940A1F58044240CC2F184
:100540000E0204F00204D21A121BA14002EBD131B8
:10055000CA1D20FA02F202F0010202EB4102F2612E
:1005600000237361336105EB82016B6823FA02F4A7
:1005700001F59871E40705D40120904018436860A4
:100580000E601CE01F2A09680EBF00225208C2F14B
:10059000190200FA02F200E019464B68DB08DB00A2
:1005A000834210D0D30F01EB830303F110045200F8
:1005B0002368002BF0D12869844211D32660B161F1
:1005C000F660B6600EE02A698868914228BF9042C2
:1005D00006D3C6608E60B060F1600020B06101E0BB
:1005E0000DF078FBE868804511D2A0EB0800E860C8
:1005F00040F00100A96908EB0102AA61506048F0CF
:100600000300486003B001F10800BDE8F08F00204E
:1006100000F02BBCD8530120343601206859883CA7
:100620002DE9F84F044688460026C8F1000B5FEA22
:10063000182008BF002123D0B0F5803F28BF1F211C
:100640001ED2A0F58071090C01F008018840A0F5C8
:100650008052120C02F004029040A0F580431B0C63
:10066000C1F10E0103F00203891AC91A984001EB87
:10067000D030C11D28FA01F101F0010101EB400168
:1006800004EB8100D0F8300130B31F290EBF0022E7
:100690004A08C2F1190208FA02F2002300E05200EF
:1006A0004568ED08ED00A5EB08055D4503D206465B
:1006B0005FEA050B0CD045694FEAD27E00EB8E0055
:1006C000002D00691CBF85422B460028E7D1184643
:1006D00000283AD1002E3AD1012088404000414202
:1006E00008436168084000F05F8141420840411EB4
:1006F000080B00F0100021FA00F2510901F0080186
:10070000CA40930803F00403DA40550805F00205D7
:100710000818EA401818C2F3400E2844704422FA20
:100720000EF1081804EB8000D0F830010DE0084607
:100730004168C908C900A1EB080159453CBF8B4677
:10074000064601690029F2D140690028F0D1002E47
:1007500000F02A81A068A0EB0800834580F0248186
:1007600020698642C0F01E817068C00808EB0B0942
:10077000C00008EB0605484518BF0DF0ABFAAE42C5
:1007800080F01081F768D6F818A0B7420CD0B06896
:100790002169884223D3C168B14204BFB968B1421C
:1007A0001DD1C760B8601CE006F11400076837B9B6
:1007B00006F110000768A7B101E00846076807F1D5
:1007C00014010A68002A02BF07F110010A68002A12
:1007D000F3D12169884202D30021016001E00DF0CC
:1007E00079FABAF1000F38D0F06904EB800000F517
:1007F000987001688E4209D10760380014D1F269FF
:100800006068012191408843606026E0206982454C
:1008100008D3DAF81000B04214BFCAF81470CAF84E
:10082000107001E00DF056FABFB12069874212D373
:10083000C7F818A0306930B12169884226BF3861F5
:1008400087610DF047FA706938B12169884202D397
:100850007861876101E00DF03DFABBF1100F09D21C
:1008600049F00300706009EB0600416841F00101A6
:10087000416096E048F0030070604BF00100686052
:100880004BF805B04FEADB0020281DD204EBC00175
:1008900001F12807216821FA00F2BB46D20705D4EE
:1008A000012202FA00F00843206006E0B8682169DE
:1008B00088422CBF83460DF00DFABD60CBF80C507A
:1008C000C5F808B0EF606CE05FEA1B2008BF0021AC
:1008D00023D0B0F5803F28BF1F211ED2A0F5807124
:1008E000090C01F008018840A0F58052120C02F0BA
:1008F00004029040A0F580431B0CC1F10E0103F0EF
:100900000203891AC91A984001EBD030C11D2BFA95
:1009100001F101F0010101EB4001E96100226A618E
:100920002A6104EB8100626822FA01F300F59870F5
:10093000DB0706D4012303FA01F11143616005606E
:100940001CE01F2900680EBF00214908C1F11901F0
:100950000BFA01F100E010464268D208D2005A4575
:1009600010D0CA0F00EB820202F1100349001A688E
:10097000002AF0D121698B4211D31D60A861ED607E
:10098000AD600EE022698168904228BF914206D393
:10099000CD608560A960E8600020A86101E00DF0ED
:1009A00099F907E10DF096F901E12DE9F84F0446B8
:1009B0008846606841420840411E080B00F0100064
:1009C000C1404A0902F00802D1408B0803F0040339
:1009D000D9404D0805F002051018E9401818C1F378
:1009E000400628443018F140081804EB8000D0F885
:1009F00030014168C908C9000646A1EB080A09E0B0
:100A000008464168C908C900A1EB080151453CBF2F
:100A10008A46064601690029F2D140690028F0D1D2
:100A200020698642C0F0C1807068C00808EB0A09DE
:100A3000C00008EB060B484518BF0DF04BF95E45AA
:100A400080F0B380F768B569B7420CD0B06821690F
:100A5000884223D3C168B14204BFB968B1421DD1F5
:100A6000C760B8601CE006F11400076837B906F1EA
:100A700010000768A7B101E00846076807F11401F4
:100A80000A68002A02BF07F110010A68002AF3D1A0
:100A90002169884202D30021016001E00DF01AF9BA
:100AA000002D34D0F06904EB800000F598700168E7
:100AB0008E4209D10760380011D1F26960680121C6
:100AC00091408843606022E02069854205D328690F
:100AD000B04214BF6F612F6101E00DF0FBF8B7B1B8
:100AE0002069874211D3BD61306930B121698842E4
:100AF00026BF386187610DF0EDF8706938B1216962
:100B0000884202D37861876101E00DF0E3F8BAF121
:100B1000100F09D249F00300706009EB060041682C
:100B200041F0010141603FE048F0030070604AF08D
:100B30000100CBF804004AF80BA0D4F808804FEA73
:100B4000D805202D28BF0DF0C5F8B8F1000F27D02B
:100B5000D4F81490009504EBC50000F128052F4649
:100B6000B8F1100F38BF0DF0B5F82068009920FAE1
:100B700001F1C90705D4009A012191400843206082
:100B800006E0A868216988422CBF07460DF0A2F84C
:100B9000C5F80890C7F80C90C9F80870C9F80C504F
:100BA000C4F808A0C4F814B004E00DF093F80020D5
:100BB000BDE8F28F06F10800BDE8F28F2DE9F04F95
:100BC00083B00546C046C046DFF8B847F52D80F033
:100BD00001810B2D31BF102705F10B00C008C700A4
:100BE0002068FE08F04010F0030F42D0C04300F030
:100BF0000100861904EBC60000F12808F700D8F8B8
:100C000008506868C008C000B84218BF0DF062F80C
:100C1000D5F80890454508BF0DF05CF84D4508BF74
:100C20000DF058F86868C008C000B84218BF0DF051
:100C300051F8C84505D120680121B14088432060A2
:100C40000DE02069814508D3D9F80C00A84204D1F1
:100C5000C8F80890C9F80C8001E00DF03BF847F0A7
:100C60000300686078190835416841F0010141606E
:100C7000F8E0A168B94280F0BF80002800F0A180B0
:100C8000012505FA06F149004A42B04011430840E7
:100C900041420840411E080B00F01000C1404A09C3
:100CA00002F00802D1408B0803F00403D9404E083B
:100CB00006F002061018F1401818C1F34008301869
:100CC000404421FA08F101EB000804EBC80000F1F0
:100CD00028094FEAC80AD9F808607068C008C0003F
:100CE000504518BF0CF0F6FFD6F808B04E4508BFC7
:100CF0000CF0F0FF5E4508BF0CF0ECFF7068C00818
:100D0000C000504518BF0CF0E5FFD94505D120685B
:100D100005FA08F1884320600DE02069834508D377
:100D2000DBF80C00B04204D1C9F808B0CBF80C9045
:100D300001E00CF0CFFF47F003007060AAEB07085A
:100D4000B819019048F001014160019848F800800D
:100D5000A7684FEAD70ABAF1200F28BF0CF0BAFFF4
:100D600047B3CDF800A004EBCA00D4F8149000F10A
:100D7000280AD346102F38BF0CF0ACFF206800992A
:100D800020FA01F1C90705D4009905FA01F10843D9
:100D9000206007E0DAF80800216988422CBF83460A
:100DA0000CF098FFCAF80890CBF80C90C9F808B07E
:100DB000C9F80CA0C4F8088006F108050198606124
:100DC00050E06068C0B339462046FFF7EEFD0500ED
:100DD00012D047E015F1400F28BF4FF0FF370BD27C
:100DE00005F10B00C008C700606828B139462046ED
:100DF000FFF716FC050035D1A168B9421CD3CA1B08
:100E00006069102A0AD339186161A26042F00103B7
:100E10004B60525047F0030141600AE00022A2609B
:100E2000626141F00302426009184A6842F001021F
:100E30004A6000F1080515E0E06887420DD2C01B4A
:100E4000A169E0607A18A26140F00100506001F1F0
:100E5000080547F00300486004E039462046FFF7E4
:100E60001AFA0546C046C046284603B0BDE8F08FD2
:100E700000B970472DE9F047A0F10804C046C0460C
:100E8000DFF8005528698442C0F07582616801F07E
:100E90000302012A00F06F82CA084FEAC20808EB79
:100EA0000409CA0737D4226811F0030F00F06582E5
:100EB00051420C1990448442C0F05D8269698C42B1
:100EC00000F0D880D608202E70D2D4F80CA0A768E5
:100ED000544508BF0CF0FEFEBC4208BF0CF0FAFE01
:100EE0006068C008C000B0EBC60F18BF0CF0F2FE7F
:100EF00005EBC60000F128018F4205D029698F4219
:100F000051D3F968A1424ED1BA453DD1286801219B
:100F1000B140884328604C4580F02D82D9F8040008
:100F2000C10740F12882810700F17A81A9698945CA
:100F300040F0B580E868AC614044E86040F00101F1
:100F4000616069698C4202D100216961A960E96927
:100F5000814280F01282DFF83004006808B9FEF7A1
:100F6000C8FFA969002900F00882E868292824BF81
:100F70002846FEF7B1FFE869E968884280F0FD8104
:100F80004FF0FF30E861F8E12830824506D028694B
:100F9000824508D3DAF80800A04204D1C7F80CA0B3
:100FA000CAF80870B7E70CF095FEB4E7E768A669E1
:100FB000A7420BD0A168814222D3C868A04204BFD7
:100FC000B868A0421CD1CF60B9601BE004F11401E5
:100FD0000F6837B904F110010F689FB101E01146A5
:100FE0000F6807F114021368002B02BF07F110020B
:100FF0001368002BF3D1814202D30020086001E086
:101000000CF068FE002E86D0E06905EB800000F54C
:10101000987001688C4209D10760380011D1E269EB
:101020006868012191408843686074E728698642B6
:1010300005D33069A04214BF7761376101E00CF03D
:1010400049FE002F3FF467AF28698742ABD3BE61EA
:10105000216929B1814226BF39618F610CF03AFEC6
:10106000606900283FF457AF296988429BD37861B3
:10107000876150E799F8040000F0030003287FF42B
:101080004AAFC5F80880D9F8040040084000C9F804
:10109000040048F00100606048F804806DE169696F
:1010A000894508D1A8686C614044A86040F00101FE
:1010B0006160005161E1C008C0004FEAD00A80447D
:1010C000BAF1200F36D2D9F80C70D9F80860B945BA
:1010D00008BF0CF0FFFDB14508BF0CF0FBFDD9F8CF
:1010E0000400C008C000B0EBCA0F18BF0CF0F2FD3E
:1010F00005EBCA0000F128018E4206D029698E4214
:10110000C0F08180F16849457DD1B74206D1286899
:10111000012101FA0AF18843286076E028308742ED
:1011200005D0286987426ED3B86848456BD1F7600F
:10113000BE606AE0D9F80C70D9F818604F450DD040
:10114000D9F808002969884223D3C168494504BFFA
:10115000B96849451DD1C760B8601CE009F11400A9
:10116000076837B909F110000768A7B101E0084620
:10117000076807F114010A68002A02BF07F110018D
:101180000A68002AF3D12969884202D3002101604C
:1011900001E00CF09FFD002E37D0D9F81C0005EBC4
:1011A000800000F59870016889450AD10760380011
:1011B00012D1D9F81C2068680121914088436860E9
:1011C00023E02869864205D33069484514BF77611A
:1011D000376101E00CF07EFDBFB12869874212D370
:1011E000BE61D9F8101029B1814226BF39618F61E3
:1011F0000CF070FDD9F8140038B12969884202D387
:101200007861876101E00CF065FD48F001006060E5
:1012100048F80480686984420BD1C5F80880ACE0C6
:1012200040084000C9F8040048F00100606048F838
:1012300004804FEAD807202F22D205EBC70000F127
:1012400028094E46B8F1100F38BF0CF043FD28684E
:1012500020FA07F1C90704D40121B94008432860E6
:1012600007E0D9F80800296988422CBF06460CF02F
:1012700031FDC9F80840F460A660C4F80C907CE029
:101280005FEA182008BF002123D0B0F5803F28BFB7
:101290001F211ED2A0F58071090C01F008018840C1
:1012A000A0F58052120C02F004029040A0F5804399
:1012B0001B0CC1F10E0103F00203891AC91A9840F0
:1012C00001EBD030C11D28FA01F101F0010101EB61
:1012D0004001E16100226261226105EB81006A68E0
:1012E00022FA01F300F59870DB0706D4012303FA14
:1012F00001F11143696004601CE01F2900680EBF02
:1013000000214908C1F1190108FA01F100E0104675
:101310004268D208D200424510D0CA0F00EB8202C8
:1013200002F1100349001A68002AF0D129698B42A2
:1013300011D31C60A061E460A4600EE02A6981689A
:10134000904228BF914206D3CC608460A160E060E7
:101350000020A06101E00CF0BDFC286A401E28625C
:101360000BD1D5F8C80100E080680028FCD14FF00F
:10137000FF30286201E00CF0ADFCC046C046BDE87D
:10138000F087000034360120D853012000B585B025
:10139000029001900E4A92680392802282F3118893
:1013A00000BF00BF0268009200AA026000980028F7
:1013B00002D0009800AA42600548806800AA8260B6
:1013C000034880680174F4F711FD05B000BD00BF4B
:1013D00028A8002038B5028BC3684469E318046963
:1013E000A34201D304691B1B534384680D781D5528
:1013F000491C5B1C521E002AF7D1C168491CC16000
:10140000012902D10CF044FC0EE027484078F0217D
:10141000084202D09920F4F7A9F823484078002820
:1014200002D1002080F3118831BD10B50400208B5B
:1014300062694243A368D35C0B70521C491C401E76
:101440000028F7D16069401C60612169884201D39E
:1014500000206061E068411EE1602169884212D18C
:1014600011484078F021084202D09920F4F77EF824
:101470000D484078002802D1002080F31188200018
:101480000CF006FC0EE008484078F021084202D03B
:101490009920F4F76BF804484078002802D1002026
:1014A00080F3118810BD000028A8002008B584B082
:1014B0000023029311B90093019302E00090481EAB
:1014C000019004AB00A90748784418300CF01CFCCC
:1014D000009909B100220A70002858BF029805B08F
:1014E00000BD00BF5F32FFFF00F10103810704D0A0
:1014F00010F8011B89B18107FAD10268B2F10131FC
:10150000914311F0803F04BF50F8042FF6E710F824
:10151000011B11B110F8011BFBE7C01A7047000056
:10152000506002604160086070470A68F8E74860F0
:101530000160704701684068F9E7F8B50600DFF818
:10154000EC5901D52846F2BD2C460020A96900E0DF
:10155000096805F11802914204D00C46A26896422F
:10156000F6D10120002840D1286AD0F888701820D0
:10157000F2F7A4FA0446A660002F05D0B74203D2C2
:10158000B6FBF7F0784300E03046E060002F02D071
:10159000B74200D23E46266100202075DFF89069F0
:1015A0003078401C30707078F021084202D09920C9
:1015B000F3F7DCFFF4F750F87078401C707005F119
:1015C00018012046FFF7B1FF7078F021084202D0E1
:1015D0009920F3F7CBFF7078401E7070C0B20028DE
:1015E00001D1F4F733F8F4F721FB2046F2BD38B50A
:1015F000044694F91400002829D1DFF834592878DA
:10160000401C28706878F021084202D09920F3F736
:10161000ADFFF4F721F86878401C68702046FFF7AA
:1016200089FF2046F2F762FA6878F021084202D07A
:101630009920F3F79BFF6878401E6870C0B20028BD
:1016400001D1F4F703F8BDE83140F4F7EFBA31BD4A
:10165000F8B5044608466FF00045FFF76EFF0646F2
:1016600094F9050094F90410814214D1C01C800043
:10167000F2F724FA074694F90500012807DB8200F7
:1016800021683846F2F742FA2068F2F72FFA27600D
:101690006079C01C607194F90400411C21712168BB
:1016A00041F82060DFF88408864202D0307D401C7B
:1016B0003075002008E0216851F820108A689542B2
:1016C00001DB1546A160401C94F904108842F2DB4E
:1016D000F1BDF8B504466FF00046DFF85028154616
:1016E00010464FF0FF33002704E0664501DB6646F5
:1016F00075467F1C94F904C067450DDAD4F800C024
:101700005CF827E0DEF808C0002BEED58C45ECD164
:1017100070463B465BB2ECE7002B11D4BCF1010FE5
:101720000EDB06E0216801EB8306766841F8236052
:101730005B1C94F904104E1EB342F3DB491E217169
:10174000904204D0017D491E0175FFF750FFA5604E
:10175000F1BD10B4C26A836B406C9C68002C02D54A
:101760006FF0004300E01B698468002C02D56FF025
:10177000004000E00069984200DD1846D2685143FD
:10178000884201DB012000E0002010BC70472DE9F9
:10179000F0410446DFF89457D5F82080D8E91C675B
:1017A0000120002194F9082000F0B4FC30433943B3
:1017B000C8E91C0105F124012046FFF7B6FE01200F
:1017C000BDE8F081F8B50446DFF86007056AD5E9A1
:1017D0001C670120002194F9082000F09BFC26EAF8
:1017E000000027EA0101C5E91C012046FFF7A2FE1F
:1017F0000120F2BD012070472DE9FC4104460D4651
:1018000016461F4604F12400FFF722FF07EB4700AE
:1018100004EB8008314608F13000FFF719FF01950D
:1018200098F9340000903B46627A94F908100FF260
:101830005070F2F733FABDE8F3812DE9FC4104461C
:101840000D4616461F4604F12400FFF742FF07EB42
:10185000470004EB8008314608F13000FFF739FFFC
:10186000019598F9340000903B46627A94F908108B
:101870000FF22070F2F712FABDE8F381C16A8A68AC
:10188000012A09DB0969012906DA006D002801D562
:1018900000207047022070470020704701EB410292
:1018A00000EB8201896B8A68012A09DB0969012939
:1018B00006DA006D002801D500207047022070472D
:1018C00000207047002900D5D8E7E7E7012900DAB2
:1018D000012113460A468FE7012900DA0121134648
:1018E0000A46AAE7DFF84C06C06A417A481E8041E2
:1018F000C00F704713464FF0FF3211467CE7134686
:101900004FF0FF32114698E780B5DFF828060068EF
:10191000417A002903D1D0F8200140688047012096
:1019200002BD80B5FFF74EFFDFF808060068417A78
:10193000002903D1D0F8200180688047012002BD32
:10194000DFF8E825126AD2F8882050325242026548
:101950001DE7DFF8D825126AD2F8882050325242AB
:10196000026514E7B1F57A7F01DC4FF47A71134612
:101970000A464FF4FA713FE7B1F57A7F01DC4FF484
:101980007A7113460A464FF4FA7156E710B50446C9
:10199000002922D5E06A816801291CDB0069012841
:1019A00019DA02212046FFF7D4FE002813D194F95A
:1019B000540010F1010F04D1002084F854000120DC
:1019C00010BD002807D1012060774FF0FF3084F868
:1019D0005400022010BD002010BDBDE810405DE79E
:1019E0004FF0FF3280F85420D1E6DFF84025126A2C
:1019F000D2F88820A03252420265C8E600290AD5F2
:101A0000C06A8168012904DB0069012801DA02202B
:101A100070470020704741E7B52900DAB42113462A
:101A20000A463C21E8E6B52900DAB42113460A4605
:101A30003C2102E710B50446002927D5E06A8168F9
:101A4000012921DB006901281EDA03212046FFF766
:101A500080FE002818D194F95400014611F1010FBD
:101A600004D1002084F85400012010BD002803D1C7
:101A7000012084F8540010BD012905D14FF0FF303A
:101A800084F85400022010BD002010BDBDE81040B5
:101A900004E74FF0FF3280F85420DFF89024126AF8
:101AA000D2F88820B4325242026570E6DFF87C2416
:101AB000126AD2F8882046325242026567E6DFF8A1
:101AC0006C24126AD2F888204632524202655EE6E1
:101AD00013463C2211468FE613463C221146ACE6E3
:101AE000002918D5C16A8A68012A14DB096901290D
:101AF00011DA90F85410491C80F8541049B20029AA
:101B000001D101207047012905D14FF0FF3180F844
:101B10005410022070470020704713464FF0FF32E8
:101B2000114669E613464FF0FF32114685E680B54F
:101B3000FFF72DFEF2F749F800210176012002BDE2
:101B400080B5FFF73FFEF2F740F800210176012053
:101B500002BD000070B50C46DFF8D81351F82050D4
:101B6000287205F590710FF240424A601B2800F27E
:101B70006681DFE810F01C00300045006D00590060
:101B8000810090009E00D600AC00C800E400F20086
:101B9000FE000901170123012E0139013901390124
:101BA000390139016401BA0044014F015A01DF488B
:101BB000026A072382F88C3005F108020623537667
:101BC0000A2393762C30506040F2DC5090600FF284
:101BD000F430486033E1D548026A8C3203235370F5
:101BE00005F10802062353760A23937600F2086073
:101BF00050604FF4967090600FF2004048601EE114
:101C0000CA48026A8C320023937005F108020C2343
